:100000000C94F7290C94F7290C94F7290C94F729F0
:100010000C94F7290C944B0F0C944D120C947B17F5
:100020000C94F7290C94F7290C94F7290C94F729D0
:100030000C94F7290C94F7290C94F7290C94F729C0
:100040000C943D0F0C94F7290C94F7290C94F72984
:100050000C94F7290C94F7290C94F7290C94F729A0
:100060000C94F7290C94F7290C94040E0C94F7299E
:100070000C94F7290C94F7290C940E0D0C94300D68
:100080000C94F7290C94F7290C94F7290000000030
:100090003D3D3D3D3D3D3D3D3D3D3D3D3D3D3D3D90
:1000A0002020546573742653657276696365202039
:1000B0003D3D3D3D3D3D3D3D3D3D3D3D3D3D3D3D70
:1000C000202020202020202020205A582045766FF4
:1000D0006C7574696F6E20546573742653657276FF
:1000E000696365200000160F18687474703A2F2F2A
:1000F0007777772E4E65646F50432E636F6D2F00B8
:10010000040126010D0A0A8FE0AEA2A5E0AAA020F4
:10011000A2EBA2AEA4AEA22041544D4547413132DC
:10012000382E2E2E20000D0A0A41544D45474131EC
:1001300032382070696E7320636865636B2E2E2ED3
:10014000200046015E018FE0AEA1ABA5AC20ADA5BD
:1001500020AEA1ADA0E0E3A6A5ADAE2E00004E6F8F
:100160002070726F626C656D7320666F756E642EA1
:10017000000076019C010D0A8EA1ADA0E0E3A6A5CA
:10018000ADA020AFE0AEA1ABA5ACA020ADA020AF4C
:10019000AEE0E2E3282DA0E5293A20000D0A4861EF
:1001A000766520612070726F626C656D20617420CD
:1001B000706F72742873293A200050417820000033
:1001C00050427820000050437820000050443520F1
:1001D0000000504578200000504778200000E201E0
:1001E000FC010D0A8FE0AEA3E0A0ACACA020AEE114
:1001F000E2A0ADAEA2ABA5ADA02100000D0A5072E9
:100200006F6772616D2069732068616C7465642129
:1002100000001A0228021B0229020A0D91AEE1E237
:10022000AEEFADA8A52000000A0D5374617475737C
:10023000206F66200000504F574552474F4F443DB6
:1002400000002C20564343353D004E026A020D0A41
:1002500082AAABEEE7A5ADA8A520AFA8E2A0ADA805
:10026000EF204154582E2E2E0A000D0A41545820DA
:10027000706F7765722075702E2E2E0A0000820234
:10028000A6020D0A87A0A3E0E3A7AAA020AAAEAD0C
:10029000E4A8A3E3E0A0E6A8A820A2204650474196
:1002A0002E2E2E2000000D0A536574204650474123
:1002B00020636F6E66696775726174696F6E2E2E4A
:1002C0002E200000C802F00287A0A2A5E0E8A5AD9C
:1002D000AE2E0D0A8FE0AEA2A5E0AAA020AEA1AC82
:1002E000A5ADA020E120465047412E2E2E20000033
:1002F000446F6E652E0D0A4650474120646174615B
:100300002065786368616E676520746573742E2E4E
:100310002E2000004F6B2E001C032A0385E1E2EC27
:1003200020AEE8A8A1AAA821000057652068617640
:100330006520736F6D65206572726F7273210000A6
:1003400044036E030D0A8AAEABA8E7A5E1E2A2AEB4
:1003500020ADA5AFE0A0A2A8ABECADEBE520A1A03D
:10036000A9E220A8A7203530303030202D000D0A1A
:100370005175616E746974792077726F6E6720624F
:100380007974652066726F6D203530303030202DE5
:1003900000009603B6030D0A8FE0AEA2A5E0AAA066
:1003A00020AAABA0A2A8A0E2E3E0EB2050532F329A
:1003B0002E2E2E0D0A000D0A50532F32206B657918
:1003C000626F61726420636865636B2E2E2E0D0A66
:1003D0000000D603E803202E2E2EADA5E220AEE2CB
:1003E000A2A5E2A00D0A0000202E2E2E6E6F207214
:1003F0006573706F6E73650D0A00FE031604202E80
:100400002E2EADA5AEA6A8A4A0A5ACEBA920AEE269
:10041000A2A5E20D0A00202E2E2E756E77616E7455
:10042000656420726573706F6E73650D0A00320427
:100430004A04202E2E2EE1A1AEA920AFE0A820AFC5
:10044000A5E0A5A4A0E7A50D0A00202E2E2E66612A
:10045000696C20746F207472616E736D69740D0A1B
:10046000000006031C089FF0CD25E803CC100418FB
:10047000B112ED18A2252B299709B11EC4C4C4C41A
:10048000C4C4C4C4C4C4C4C4C4C4C4C4C4C4C4C42C
:10049000C4C4C4C4C4C492A5E1E220AAABA0A2A86B
:1004A000A0E2E3E0EB2050532F3220202020202038
:1004B00092A5E1E220AAABA0A2A8A0E2E3E0EB2093
:1004C0005A5820A820A4E02E202092A5E1E220ACDA
:1004D000EBE8A82020202020202020202020202001
:1004E0002020202092A5E1E220424545502F544192
:1004F00050454F55542F434F564F5820202092A51A
:10050000E1E220A2A8A4A5AE2020202020202020C7
:10051000202020202020202092A5E1E22052532DEF
:100520003233322020202020202020202020202094
:10053000202084A8A0A3ADAEE1E2A8AAA020534445
:100540002F4D4D4320202020202020208FE0AEA3DF
:10055000E0A0ACACA8E0AEA2A0ADA8A520466C611E
:1005600073682D524F4DC4C4C4C4C4C4C4C4C4C4ED
:10057000C4C4C4C4C4C4C4C4C4C4C4C4C4C4C4C43B
:1005800050532F32206B6579626F617264207465FD
:10059000737420202020202020205A58206B657959
:1005A000626F617264207465737420616E6420658B
:1005B000746320204D6F75736520746573742020FB
:1005C00020202020202020202020202020204245E4
:1005D00045502F544150454F55542F434F564F5877
:1005E0002074657374202020566964656F207465DB
:1005F0007374202020202020202020202020202054
:10060000202052532D323332207465737420202001
:1006100020202020202020202020202053442F4D47
:100620004D4320646961676E6F7374696320202095
:10063000202020202020577269746520466C617349
:10064000682D524F4D2020202020202020202020C7
:100650005406180716050E8EE1ADAEA2ADEBA5202F
:10066000AAABA0A2A8E8A820E3AFE0A0A2ABA5ADEA
:10067000A8EF3A16050F3C183E2C203C193E1605F3
:10068000103C456E7465723E202D202284A0222CE1
:1006900020A2EBA1AEE01605113C4573633E202D70
:1006A00020228DA5E2222C20AEE2ACA5ADA02C200C
:1006B000A2EBE5AEA42016051283AEE0EFE7A8A5F5
:1006C00020AAABA0A2A8E8A82028E2AEABECAAAE74
:1006D00020A220ACA5ADEE293A201605133C5363A9
:1006E000726F6C6C4C6F636B3E202D20E0A5A6A84A
:1006F000AC2054562F5647411605143C4361707385
:100700004C6F636B3E202D20EFA7EBAA20A8ADE233
:10071000A5E0E4A5A9E1A00016050E557361676583
:100720003A16050F3C183E2C203C193E1605103C8D
:10073000456E7465723E202D2022596573222C204F
:1007400073656C6563741605113C4573633E202D1B
:1007500020224E6F222C2063616E63656C2C206515
:1007600078697420160512486F742D6B65797320B3
:1007700028696E206D656E75206F6E6C79293A2040
:100780001605133C5363726F6C6C4C6F636B3E20A9
:100790002D20746F67676C652054562F5647412093
:1007A0006D6F64651605143C436170734C6F636B29
:1007B0003E202D206C616E677561676520737769D7
:1007C00074636800C807F007161A0A83E6160A0C55
:1007D0003C183E2C203C193E202D20A8A7ACA5ADEE
:1007E000A5ADA8A520E7A0E1E2AEE2EB150F000061
:1007F000161A0A487A160E0C3C183E2C203C193E5C
:10080000202D206672657175656E6365150F000099
:1008100014083008160E078AABA0A2A8A0E2E3E0F5
:10082000A0205A5816230784A6AEA9E1E2A8AA0080
:10083000160F075A58204B6579626F617264162350
:10084000074A6F79737469636B00160B09312032A4
:1008500020332034203520362037203820392030EE
:10086000160B0A512057204520522054205920555C
:100870002049204F2050160B0B4120532044204686
:1008800020472048204A204B204C2065160B0C6343
:10089000205A2058204320562042204E204D2073BD
:1008A000207316260A1816240B1B2046201A16261B
:1008B0000C19160E0F536F66745265736574161E0D
:1008C0000F547572626F4B6579001605076520201D
:1008D0002031203220332034203520362037203874
:1008E00020392030203120322020702073207020C9
:1008F0002007200720071605096020312032203309
:100900002034203520362037203820392030202D43
:10091000203D201B2020692068207520206E202F7C
:10092000202A202D16050A742051205720452052D8
:100930002054205920552049204F2050205B205D15
:10094000205C202064206520642020372038203956
:1009500016050B63204120532044204620472048A1
:10096000204A204B204C203B20272020206520209F
:10097000202020202020203420352036202B160552
:100980000C73205A2058204320562042204E204DE0
:10099000202C202E202F20202020207320202020DB
:1009A0001820202020312032203316050D632077B7
:1009B00020612020202020202073202020202020A3
:1009C00020612077206D206320201B2019201A2011
:1009D00020302020202E20651605105261772064DB
:1009E0006174613A16040F00EC091C0A1605139293
:1009F000E0F1E5AAE0A0E2ADAEA520ADA0A6A0E2A0
:100A0000A8A5203C4553433E202D20A2EBE5AEA4F3
:100A100020A8A720E2A5E1E2A02E0000160A1350AC
:100A200072657373203C4553433E2074687265655C
:100A30002074696D657320746F20657869742E0069
:100A4000440A5C0A0D0A92A5E1E2A8E0AEA2A0ADBC
:100A5000A8A520ACEBE8A82E2E2E20000D0A4D6F85
:100A600075736520746573742E2E2E200000720A33
:100A7000880A8EA1ADA0E0E3A6A5ADA8A520ACEBA9
:100A8000E8A82E2E2E202000446574656374696EDC
:100A900067206D6F7573652E2E2E20200000A20A30
:100AA000B00A8DA0E1E2E0AEA9AAA02E2E2E200071
:100AB000437573746F6D697A6174696F6E2E2E2E33
:100AC0002000C60AD00A8FAEA5E5A0ABA821000081
:100AD0004C6574277320676F2100DE0AF80A202016
:100AE000202020208DA5E220AEE2A2A5E2A020AE2B
:100AF000E220ACEBE8A82E002020202020204E6F22
:100B0000206D6F75736520726573706F6E73652EDF
:100B10000000160B360B20202088ACA5EEE2E1EF9A
:100B200020ADA5AAAEE2AEE0EBA520AFE0AEA1AB52
:100B3000A5ACEB2E000020202020546865726520B3
:100B400061726520736F6D652070726F626C656D88
:100B5000732E0000580B780B20203C456E74657294
:100B60003E202D20AFA5E0A5A7A0AFE3E1E2A8E2DB
:100B7000EC20E2A5E1E22E0020202020203C456E62
:100B80007465723E202D20726573746172742074D6
:100B90006573742E00009A0BD60B1623122092A5B3
:100BA000E1E2204452414D201620138FE0AEA2A571
:100BB000A4A5ADAE20E6A8AAABAEA2162014A1A5AE
:100BC000A720AEE8A8A1AEAA162015E120AEE8A89D
:100BD000A1AAA0ACA800162312204452414D2074B3
:100BE000657374201620134C6F6F707316201450A9
:100BF0006173731620154661696C0000000C0C0CC3
:100C000016170C90E3E1E1AAA8A9000016170C45FD
:100C10006E676C69736800001C0C5E0C1602028221
:100C2000EBE5AEA416020382E1F120E1ADAEA2A095
:100C300016020491E2A5E0A5E2EC20AC2FE1E52E3E
:100C400016020584AEA1A0A22EA7A0A4A0ADA8A5BF
:100C500016020682EBAFAEABADA8E2EC20001602A6
:100C600002457869742016020352657472696576CC
:100C70006520616C6C201602044572617365206307
:100C800068697020160205416464206A6F6216026A
:100C90000645786563757465206A6F627300A20CFF
:100CA000B20C159F208DA5E220E4A0A9ABAEA22036
:100CB0000000159F20204E6F2066696C6573202010
:100CC0000000C60CEA0C16020A159E97E2A5ADA814
:100CD000A520466C617368159F16020B3C45534373
:100CE0003E202D20A2EBE5AEA40016020A159E526E
:100CF00065616420466C6173682E2E2E159F160266
:100D00000B3C4553433E202D206578697400120D3D
:100D1000260D16020B159F88ADA8E62E534420AA77
:100D2000A0E0E2EB000016020B159F5344636172D2
:100D30006420696E69742E2000003E0D4E0D208DDA
:100D4000A5E220534420AAA0E0E2EB2120002020CD
:100D50004E6F2053442D6361726421202000620D88
:100D6000720D208EE8A8A1AAA020E7E22E2053440D
:100D700020002053442072656164206572726F7296
:100D80002000860D960D2020208DA5E2204641549E
:100D900020212020200020464154206E6F20666FC5
:100DA000756E64212000AA0DBA0D20208EE8A8A13E
:100DB000AAA0204641542021200020204641542052
:100DC0006572726F722021202000CE0DDE0D208E04
:100DD0002C20A3ABEEAAA0ADE3ABAE2120002047B0
:100DE0007265617420676C69746368212000F20D7C
:100DF000060E16020C159E2093A2A5E0A5AD3F207D
:100E00003C593E20000016020C159E596F75207348
:100E10007572653F203C593E00001E0E320E1602D0
:100E20000C159E91E2A8E0A0ADA8A52E2E2E2020A4
:100E3000000016020C159E45726173652E2E2E2041
:100E40002020202000004A0E5E0E16020C159E8700
:100E5000A0AFA8E1EC2E2E2E2020202000001602AC
:100E60000C159E57726974652E2E2E20202020208E
:100E70000000760E8A0E16020C159E8FE0AEA2A51B
:100E8000E0AAA02E2E2E2020000016020C159E5641
:100E900065726966792E2E2E202020200000A20E79
:100EA000B60E16020C159E87A0A2A5E0E8A5ADAE71
:100EB0002E202020000016020C159E436F6D706CD2
:100EC0006574652E202020200000CE0EEE0E160D3B
:100ED0000687A0AFA8E1EC20A220466C617368529F
:100EE0004F4D20A7A0A2A5E0E8A5ADA000001612D6
:100EF000064A6F6228732920636F6D706C65746594
:100F0000642E0000080F180F161507A1A5A720AE24
:100F1000E8A8A1AEAA2E00001611074E6F20657238
:100F2000726F72732064657465637465642E00006B
:100F3000340F440F161507E120AEE8A8A1AAA0AC13
:100F4000A8210000160E07536F6D65206572726F41
:100F500072732061726520646574656374656421D1
:100F60000000660F740F20202084A0E2E7A8AAA842
:100F70003A20000020202053656E736F72733A2070
:100F80000000860F9A0F20202020208DA5E220AAA5
:100F9000A0E0E2EB202020202000202020202020A4
:100FA0004E6F206361726420202020202000B20F49
:100FB000C60F208AA0E0E2A020E3E1E2A0ADAEA24D
:100FC000ABA5ADA020002020204361726420696E93
:100FD00073657274656420202000DE0FF20F2020FC
:100FE00087A0E9A8E2A020AEE220A7A0AFA8E1A8D0
:100FF0002000202020202052656164206F6E6C79D3
:101000002020202020000A101E10202087A0AFA83A
:10101000E1EC20E0A0A7E0A5E8A5ADA020002020FD
:1010200020577269746520656E61626C656420206A
:1010300020003610501088ADA8E6A8A0ABA8A7A045
:10104000E6A8EF20AAA0E0E2AEE7AAA82E2E2E0086
:101050004361726420696E697469616C697A617454
:10106000696F6E2E2E2E00006C10881053442F4D89
:101070004D4320AAA0E0E2A020ADA520AEA1ADA0E6
:10108000E0E3A6A5ADA02E004E6F2053442F4D4D9A
:1010900043206361726420666F756E642E00A21037
:1010A000B6108EA1ADA0E0E3A6A5ADA020AAA0E059
:1010B000E2A03A200000466F756E6420636172649E
:1010C0003A200000C810FE1016100B8DA0E7A0E219
:1010D000EC20A4A8A0A3ADAEE1E2A8AAE320160CE0
:1010E0000C5B205D208FAEA4E0AEA1ADEBA920AEDD
:1010F000E2E7F1E220A22052532D323332001611E2
:101100000B537461727420646961676E6F737469E4
:101110006320160C0C5B205D2044657461696C656E
:1011200064206C6F6720746F2052532D323332006D
:10113000341144118EA1ADA0E0E3A6A5ADA02046D8
:1011400041540000466F756E6420464154005211B0
:101150006C118FAEA8E1AA20E4A0A9ABAEA2AEA903
:1011600020E1A8E1E2A5ACEB2E2E2E0044657465CB
:101170006374696E67206F662066696C6520737999
:101180007374656D2E2E2E008C11A61197E2A5ADFD
:10119000A8A520E2A5E1E2AEA2AEA3AE20E4A0A9FC
:1011A000ABA02E2E2E0052656164696E67206F66BB
:1011B00020746573742066696C652E2E2E00C21132
:1011C000DA1184A8A0A3ADAEE1E2A8AAA020A7A04E
:1011D000A2A5E0E8A5ADA02E0000446961676E6F8E
:1011E0007374696320697320636F6D706C657465D7
:1011F0002E000D0A6F75742000002C20696E2000EF
:101200000D0A3B434D4400000D0A3B41434D44341D
:1012100031000D0A4353207570000D0A43532064BA
:101220006F776E004D4D4300534420763100534498
:101230002076322B205374616E64617264204361A6
:10124000706163697479000053442076322B204822
:1012500069676820436170616369747900004F4376
:10126000523A20004353443A20004349443A200074
:101270004D616E75666163747572657220494420B4
:10128000202020004F454D2F4170706C69636174C0
:10129000696F6E204944200050726F64756374203A
:1012A0006E616D65202020202020200050726F6428
:1012B000756374207265766973696F6E20202000F3
:1012C00050726F647563742073657269616C20235A
:1012D000202020004D616E75666163747572696EC1
:1012E00067206461746520002E3230002E31390091
:1012F0004352433D00000D0A3B5265616420736513
:1013000063746F7220000D0A3B353132206F7065B7
:10131000726174696F6E7320697320736B69706595
:1013200064000A0A20049F0100023516DF0064975A
:101330004C7F44600E945715A0E0B1E00E9408175E
:1013400000E21FE725E30E944717E2E2F3E10E9473
:101350007B15E4ECF0E10E941517FB8A99D206D3C5
:101360000E94FC0FE1F30537C1F3023749F00A355B
:1013700049F011FDF4CF063791F7477F6496089541
:10138000EB8AECCF0B89002319F008E04027E6CF69
:101390004A7F4260DBD2DAD2E0ECF0E00E94FD143A
:1013A0000E94D414D3D24660E1D2E8E2F3E10E9475
:1013B0007B15A1E0B3E0BB8B0E940817C7D2E2E324
:1013C000F0E10E94F814F0922601FA8AA9D212EAFA
:1013D0000FEF0E946F1710E20E948617ACD211EA3D
:1013E0000FEF0E946F172FEF00E080D2EEEFF2E3D5
:1013F0000E949B172A9531F4AED2E8E6F0E10E94F4
:10140000F8143AC2013081F708E070D2E4E0F3E367
:101410000E949B1780E002FF80E4898B14E00E9409
:10142000861773D207E70E948B1712E00E94861777
:1014300009E60E94E31709890E94E3170E949217A8
:10144000002379F002FFEDCF01E050D201E40E94C9
:101450008B170023C9F742D238D210E1E4E2F2E15F
:101460001DC03CD232D211E0E8E2F2E1098900234A
:10147000A9F00AE33BD20AE70E948B17DE0126E0BF
:101480000E94E2170D932A95D9F712E0EEE2F2E1FD
:10149000088106FF03C016E0E8E4F2E1109326019C
:1014A0001A8BEF93FF9357D2EEE9F0E10E94F81404
:1014B000FF91EF910E94FD141A8911FF0CC04BD2CD
:1014C000EEE5F2E10E94FD14DE0124E00D910E94A0
:1014D0004D152A95D9F711EA0FEF0E946F1709E011
:1014E00005D209E40E948B170023B9F40E94A217C9
:1014F0000F3F99F0DE0121E10E94E2170D932A953A
:10150000D9F729D2E4E6F2E10E94FD14DE012FE0D2
:101510000D910E944D152A95D9F711EA0FEF0E94FF
:101520006F170AE0E3D10AE40E948B17002321F42D
:101530000E94A2170F3F09F49FC1DE0121E10E9422
:10154000E2170D932A95D9F706D2EAE6F2E10E9456
:10155000FD14DE012FE00D910E944D152A95D9F75B
:10156000FAD1E0E7F2E10E94FD1408810E940F1514
:10157000F2D1E4E8F2E10E94FD143A89098134FFD6
:101580000E94531534FD0E940F150A8134FF0E94FA
:10159000531534FD0E940F15DED1E8E9F2E10E94F7
:1015A000FD14DE01139625E034FD26E00D910E9426
:1015B00018152A95D9F7CFD1ECEAF2E10E94FD1473
:1015C000088534FD098502950E9413150EE20E94DC
:1015D0001815088534FD09850E941315BCD1E0EC6F
:1015E000F2E10E94FD14DE01199634FD119624E00B
:1015F0000D910E940F152A95D9F7ADD1E4EDF2E1D6
:101600000E94FD140E8534FD02950F700E94031593
:10161000E8EEF2E10E8534FD0CC01D85007F1F70E1
:10162000012B02950F930E94FD140F910E94031548
:101630000CC00F70035018F40C59ECEEF2E10F934C
:101640000E94FD140F910E94031585D1EEE4F1E193
:101650000E94F8141DB7109305011EB710930601E0
:10166000C0930701D0930801E9E1FCE0E0935C013D
:10167000F0935D0111EA0FEF0E946F170E94CE19DF
:10168000AF93BF938F939F9366D1E0E3F1E10E9404
:10169000F8141091270102E1112321F006E11A95B7
:1016A00009F002E30E940F159F918F91BF91AF91B6
:1016B00080E090E00E94761B07C00196B096F8305B
:1016C00019F40E94761B01F51081153EB1F3112328
:1016D000D9F00385087D89F7EF93DF01EAE0F7E1B0
:1016E0000591002331F01D910117D1F3FB2FEF91EC
:1016F000E4CFFB2FEF91848D958DA68DB78D082FAC
:10170000092B0A2B0B2B39F4B7C0544553544649C7
:101710004C4542494E006FEF71E00E946B1C8C8378
:101720009D830E94491C0197AF09BF0900912901BF
:101730000A950823039500935601009129010E9400
:10174000521C8093570190935801A0935901B09374
:101750005A01F0925101828D938DA489B5898093AD
:10176000520190935301A0935401B0935501F3D0CB
:10177000E8E8F1E10E94F814F092040102E0C02EC2
:1017800014E50E946F170E946A260E947A1C0023AB
:1017900031F1E0E0F4E0A0E0B2E00E949C2600918C
:1017A0000401002391F3F0920401AEE1BB89BB8BED
:1017B0000E9408174F934C7F446000915A010E9489
:1017C0000F15009159010E940F15009158010E94B8
:1017D0000F15009157010E940F154F91D6CFE0E0F1
:1017E000F4E0AC81BD81B17011960E949C260E94EC
:1017F0008F26CC24002714E50E946F17AEE1BB8929
:10180000BB8B0E94081700E228E00E944C17A3D06F
:10181000E0EFF2E10E94FD140B810E940F150A8196
:101820000E940F1509810E940F1508810E940F1553
:1018300023C0F894109105011DBF109106011EBF31
:10184000C0910701D091080178940F9384D00F9133
:10185000EAE3FDE0013071F0EEE5FDE0023051F029
:10186000E2E8FDE0033031F0E6EAFDE0043011F09B
:10187000EAECFDE00E94F8146ED0EEEBF1E10E947C
:10188000F8144C7F446072D00E94FC0FE1F350CDFD
:101890002227B22FB55FABE00E9408172F930B8968
:1018A0001FE9201709F410EF2EE10E9451172F9124
:1018B0002395223071F7ADE0BCE00E94081700E2EA
:1018C00043FD0BEF0E944217089500E10FD0EAE0BC
:1018D000F3E30E949B170023C1F708950BE306D0A2
:1018E0000BE70E948B170023C9F7089543FF089563
:1018F0004F934A7F42600F93E0E0F2E10E94FD14B3
:101900000F910E9403154F91089543FF08954F933F
:101910004A7F4260E8E0F2E10E94FD144F91089591
:1019200043FF08954F934A7F4260E2E1F2E10E9453
:10193000FD144F91089543FF08954F934A7F4260ED
:10194000EAE1F2E10E94FD144F910895F4D043FFC3
:1019500008950BE3ADC0A1E0BB89B395BB8B0E949A
:101960000817E9D043FF08950BE3A2C0A0E0B1E05F
:101970000E9408171FE70E940517E2E6FFE00E9499
:10198000F8141AE7E2E8FFE0B59903C01CE7EEEAB5
:10199000FFE00E9405170E94F8141AE7EAEDFFE045
:1019A000B49903C01CE7E6E0F0E10E9405170E942D
:1019B000F814089510D018E010939A004D7F4160FC
:1019C00008950DE001D00AE000909B0005FEFCCFD9
:1019D00000939C000895F092980015E010939900F0
:1019E000F0929B001EE010939D000895F4DF18E92B
:1019F00010939A004E7F426010E0109309011093FB
:101A00000A01F0920B0110E810930C0110930D01E4
:101A1000F0920E0195988D9ABE9808951F931FB766
:101A20001F930F9300919C0010910E01103898F4B1
:101A3000AF93BF93B3E0A0910C010D93AF77A06873
:101A4000A0930C01BF91AF91139510930E011C361A
:101A500010F044FD959A0F911F911FBF1F9118958B
:101A60001F931FB71F9310910B011123C1F044FF67
:101A700002C0B69914C0AF93BF930F93B3E0A09187
:101A80000A010D9100939C00AF77A060A0930A011A
:101A90001A9510930B010F91BF91AF9105C0109152
:101AA0009A001F7D10939A001F911FBF1F911895D8
:101AB0001F93AF93BF9344FD87D010910B01103853
:101AC000D0F7B3E0A09109010D93F89410910B01A8
:101AD000139510930B017894AF77A060A093090140
:101AE00044FF02C0B69905C010919A00106210938D
:101AF0009A00BF91AF911F9108951F9310910E010D
:101B00001123B9F0AF93BF93B3E0A0910D010D91F4
:101B1000F89410910E011A9510930E0178941B36CB
:101B200008F49598AF77A068A0930D019894BF91A1
:101B3000AF911F9108950DE0BBDF0AE0B9CF4F933D
:101B4000427F4260EF93FF93E0E9FBE156D7FF91BC
:101B5000EF91A0E0B0E0EFDF0B2F61D70A2F5FD746
:101B600000E2A6DFA5DFEF93FF9380E1019195D717
:101B70008A95E1F700E29CDFFF91EF9180E101910E
:101B800092D78A95E1F75096B23029F74F91089590
:101B90000D0A3B20202020202E30202E31202E32F6
:101BA000202E33202E34202E35202E36202E372086
:101BB0002E38202E39202E41202E42202E43202E3A
:101BC00044202E45202E4600B69908951F9310916B
:101BD0000B01112329F010919A00106210939A00C2
:101BE0001F91089510E010938B0019E010938A0064
:101BF0001BE21093870012E31093860010917D0082
:101C0000106110937D0008951F931FB71F931091CB
:101C10000F0114FDC798139510930F0131F4C79A63
:101C2000109110011395109310011F911FBF1F9168
:101C30001895AF93BF93F894A0910F01B091100144
:101C40007894A80FB91FB068A083B183BF91AF91FA
:101C500008959F93918197FF12C08F938081AF93D6
:101C6000BF93F894A0910F01B09110017894A81B34
:101C7000B90BB6FD07C0F182BF91AF918F919F91D3
:101C800008940895BF91AF918F919F918894089582
:101C90001127939A000000000000000000000000DF
:101CA00000000000839B116093988B9A0000000055
:101CB000839912608B98112361F0BF9A0E942E269F
:101CC000C79A00FDC798A0E0BCE6A150B040E9F774
:101CD000F5CF0E94DA0C75DE74DE73DEE0ECF0E026
:101CE0000E94FD140E94D414E0E0F1E00E94F81478
:101CF00015E51BBB1AEA1ABB12E818BB15E017BBA7
:101D000015E115BB1AE014BB959A8D98189A109896
:101D10001998119A15E1109365001AE01093640068
:101D200084E191E00197F1F7002719B3153509F027
:101D3000016016B31778103809F0026013B31F71F1
:101D4000153109F00460859B086011B113701130E2
:101D500009F00061109163001F71153109F00062F4
:101D60001AEA1BBB15E51ABB15E018BB12E817BB36
:101D70001AE015BB15E114BB95988D9A1898109A26
:101D8000199A11981AE01093650015E110936400F8
:101D900084E191E00197F1F719B31A3A09F0016073
:101DA00016B31778153009F0026013B31F711A309B
:101DB00009F004608599086011B11370123009F0C0
:101DC0000061109163001F711A3009F00062002356
:101DD00029F4E2E4F1E00E94F81408950F930E94C0
:101DE0004F26E2E7F1E00E94F8140F9106950F9359
:101DF00020F4EAEBF1E00E94FD140F9106950F9399
:101E000020F4E0ECF1E00E94FD140F9106950F9391
:101E100020F4E6ECF1E00E94FD140F9106950F937B
:101E200020F4ECECF1E00E94FD140F9106950F9365
:101E300020F4E2EDF1E00E94FD140F9106950F935E
:101E400020F4E8EDF1E00E94FD14EEEDF1E00E94D7
:101E5000F8140E944F26FFCF1AB712601ABF19B7A5
:101E6000106119BF12E013BFF0921601F092110138
:101E7000F0921501F092170108958E98969A1F938B
:101E80001FB71F9317B71E7F17BF1F911FBF1F914B
:101E900014981C9A18951F931FB71F932F930F9395
:101EA00000911201209111011091160117FD64C0DB
:101EB000293081F02A30A0F4222329F4869959C0D0
:101EC0001E7F239580C00695869B02C000681E2554
:101ED000239579C086991E2510FF4BC0239573C0AA
:101EE000869B47C020931301009314011C98149AF9
:101EF00020E822BF21E026BF27B7216027BF20911D
:101F000015012223D1F4013E51F10A3A89F10B3A2D
:101F100001F10E3E69F10A3F59F10E3F49F1003ED1
:101F200041F0003F41F01068109317010093180131
:101F30001FC012601EC014601CC02A95209315019A
:101F4000C1F4009118010E37A1F416E8109317019F
:101F50000FC0F092180121E02093150109C012E88A
:101F6000109317010EE70093180127E02093150145
:101F700011270027222727C02930A1F02A30E1F0BD
:101F80002B30F0F4222319F4116023951CC007951F
:101F900028F48E98969A1E25239515C096988E9AA9
:101FA000239511C010FD04C096988E9A23950BC0FE
:101FB0008E98969A239507C08E98969A239503C07B
:101FC00018E000272227209311010093120110939B
:101FD00016010F912F911F911FBF1F9118950E94FD
:101FE0002E261091170117FFFACFF092170112FD5C
:101FF000F6CF0091180108950E942E261091170126
:1020000017FF08C0F092170112FD04C000911801DB
:1020100098940895189408958E98969A17B71E7FED
:1020200017BF14981C9A11270C9BF6CF1A95E1F74D
:10203000F8941C98149A96988E9A0093120110E8BE
:1020400010931601F0921101F0921501F092170110
:10205000F0921301789484E191E00197F1F796985A
:102060008E9A86E695E00197F1F7E9E1F1E08FE0DD
:1020700090E00E94190E14981C9A10911601187085
:1020800041F4E9E1F1E00E94290EB8F78E98969AA2
:1020900018940895F0921301E9E1F1E084E190E0F1
:1020A0000E94190E10911301112341F4E9E1F1E0AE
:1020B0000E94290EB8F70027189408950091140182
:1020C0000895219714981C9AE2E9F3E091D4F092D4
:1020D0001301E9E1F1E084EF91E00E94190E109103
:1020E0001301112331F4E9E1F1E00E94290EB8F760
:1020F00003C000911401D1D40FEF31D0F09213013D
:10210000E9E1F1E088EE93E00E94190E10911301CD
:10211000112339F4E9E1F1E00E94290EB8F736D035
:1021200006C000911401B9D40A3A09F02CD002EF8C
:1021300016D029F40BEA1CD011F403E819D000EFF3
:102140000ED011F402E00BD003EF09D031F400E01F
:1021500006D0E7E9F5E50E94FD14219608959DD487
:102160005BDF71F097DF91F098D40A3F61F4089536
:10217000088390DF59F091D41881011721F4089554
:10218000EEE2F4E005C0EAEFF3E002C0E2EDF3E0D6
:102190000E94F814989408952597FB82E6E5F3E2EF
:1021A0000E947B15E8EEF9E040D610E81C83EAECCB
:1021B000F8E040D604EC2DE26FD6E0E1F8E0F292D0
:1021C000EE23E9F7F0921301F88200911301002346
:1021D00019F00091140171D00C8107FF15C0077030
:1021E0000C830DEE6AD018DF79F054DF69F065D00A
:1021F0000A3F51F40C8161D00FDF31F04BDF21F049
:102200005CD00A3F09F492D01091170117FFDDCF7F
:10221000F09217010091180119832B8112FF0CC055
:1022200011FD09C0063739F423952B83233020F0A4
:10223000E0D525960895FB8211FD17C012FD11C04F
:10224000AC81B1E00E3711F4AB27A068BB0F0737A4
:1022500011F4AB27A068BB0F083511F4AB27A068B9
:10226000AC83033811F4A8E410C0043811F4A8E7D3
:102270000CC0003808F5000F11FD0160ECE5F3E239
:10228000E00FFF1DA491AA23B9F0BA2FB770BB23AA
:1022900009F0B395A695A695AE73A43208F0A39560
:1022A000AE3108F0A395AD5FB95FB2D509811EEAE2
:1022B00002FD11ED21E0F5D588CF0F93F0921301C7
:1022C000E881F8E00193EF70E8834C7FA5E0B1E18D
:1022D0009FD5E881E3952DE02A83F8E0E395EF7040
:1022E000E98300810F931EE0003E61F0013E51F052
:1022F0001DE0003F39F01BE00D3E21F01AE00538EB
:1023000008F41FE082D500E2BDD50F912A81222377
:1023100029F085D3E9812A812A95DECF42600E9487
:102320000F1500E20E9418150F910895A9E2B7E079
:102330006FD50C811CED01FF10ED22E0B2D50C81B0
:102340001CED02FF10ED22E0ACD50C811CED00FF6E
:1023500010ED22E0A6C503052F10DF010000580094
:102360000000380028001800200070000000600005
:102370005000400030000A000900000000001D5D10
:102380000C0000000D75120011000000000000009C
:1023900014001B0013001A0019000015000024008F
:1023A0001C002300220029002100006500003D00E0
:1023B0002C002B0032002A003100006D00003C0090
:1023C00034003B0033003A003900000000000000F8
:1023D00044004300420041004900000000004C005E
:1023E0004B004A0052005900510000000000540008
:1023F0005C9953005B005A0061000000000000007F
:102400006300000062006900000000000B0074001F
:1024100073AD6A00000072000000000000000000C0
:102420000000000000000000710000000000948225
:102430000000937D92810000000000009579A57A4C
:102440009C859B00A38D9A84080091006800AB00D6
:10245000A48AA900A178A2898088000016250F57B8
:102460006865656C203D16250C4C2020204D2020F1
:1024700020521625115820203D1625125920203DA6
:10248000000016040A15DF0003022F13DF01090AFA
:102490002204AF01230A0D0ADF001F931FB71F9309
:1024A0002F930F9300911C0120911B0110911F018C
:1024B00017FD22C0293081F02A30A0F4222329F40C
:1024C000879917C01E7F239540C00695879B02C041
:1024D00000681E25239539C087991E2510FF09C065
:1024E000239533C0879B05C020931D0100931E01D7
:1024F00011270027222729C02930A1F02A30E1F036
:102500002B30F0F4222319F4116023951EC0079597
:1025100028F48F98979A1E25239517C097988F9A1D
:10252000239513C010FD04C097988F9A23950DC072
:102530008F98979A239509C08F98979A239505C0ED
:102540001127879B12E00027222720931B0100936D
:102550001C0110931F010F912F911F911FBF1F91FD
:1025600018954B7F4260E0E4FAE00E94F814446062
:102570002A97F8948F98979A15981D9A1AB7186009
:102580001ABF19B7106219BFF0921F01F0921B0118
:10259000F0921D017894E8E8F4E20E947B15A4E033
:1025A000B3E036D4C8DAEEE6FAE00E94F814A4E00C
:1025B000B4E02ED4C0DAF0921D01E0E2F1E082E056
:1025C00090E00E94190E10911D011123A1F7E0E285
:1025D000F1E00E94290EB8F70FEF5FD29FD1B9F05A
:1025E000CBD1A9F05AD20A3F91F4F0921D01E0E25A
:1025F000F1E088EE93E00E94190E10911D01112365
:1026000039F4E0E2F1E00E94290EB8F76EC070C024
:1026100000911E0142D20A3AC9F700E05CD0A4E062
:10262000B5E0F6D388DAEEE9FAE00E94F814A4E007
:10263000B6E0EED380DA03EF45D008EC43D003EFE9
:1026400041D004E63FD003EF3DD000E53BD0A4E00D
:10265000B7E0DED370DA02EF35D0F0921D01E0E290
:10266000F1E084E190E00E94190E10911D01112308
:1026700031F4E0E2F1E00E94290EB8F736C0009193
:102680001E0109870AD2002319F0033009F02DC07A
:10269000A4E0B8E0BDD34FDA08EE14D002E012D0C7
:1026A00006EE10D003EF0ED004E60CD004EF0AD0F3
:1026B000A4E0B9E0ADD33FDAE2ECFAE00E94F8140E
:1026C0003ADA4EC0EAD12AD171F056D161F0E5D1A3
:1026D0000A3F49F408950B834FD129F0DED11B81C5
:1026E000011709F40895FF91EF91E2E1FBE002C0C8
:1026F000EAEDFAE0EF93FF931EDAEEE8F4E20E94CF
:102700007B15AAE0BBE084D3FF91EF910E94F814FF
:10271000AAE0BCE07DD3E4E5FBE00E94F8140E944F
:10272000EF0F063719F00A35D1F723CF00E0C02E9E
:1027300014E50E946F17002710EAD1D300271DEA85
:10274000CED300271EEACBD3F8948F98979A15988A
:102750001D9A19B71F7D19BF789442602A96089573
:102760004C7F02E0C02E14E50E946F17E4E9F4E20A
:102770000E947B15E6E6F4E21985112311F0ECE5E1
:10278000F4E258D316E91C83FD8218E71E83FF820A
:10279000F886F0921D011985112331F0ADE2BFE0FA
:1027A00037D30F810E941315A9E2B1E131D3AC8177
:1027B000BD810E942215A9E2B2E12AD3AE81BB27D6
:1027C0000E942215BBE0BF93A4E222D31FED08852F
:1027D00000FD1EEA23E065D31FED21E062D31FED6B
:1027E000088502FD1EEA23E05CD31FED21E059D3EA
:1027F0001FED088501FD1EEA23E053D3BF91B39579
:10280000BE3008F3009104010023B9F0F0920401F6
:10281000AC81BD81D196D196AF930B2F10EA5FD3D7
:102820000F911DEA5CD3AE81BB279B96AF930B2F14
:1028300010EA55D30F911EEA52D30E94FC0F19F0F3
:10284000063709F473CF00911D010023D9F2F092ED
:102850001D0100911E0103FFD5CF08838DD091F299
:1028600009838AD079F20A831985112319F084D05B
:1028700049F20B83088107700887AC81BD8189818B
:102880009927188114FD08C0A80FBF1DAE33BE05DF
:1028900050F0ADE3B1E007C080950196A81BB90BDD
:1028A00010F4AA27BB27AC83BD83AE81BB278A81E6
:1028B0009927188115FF0AC080950196A80FB91FA6
:1028C000BB2311F4AA3F30F0A9EF04C0A81BBF0935
:1028D00008F4AA27AE831985112329F00B81AF8153
:1028E000A00FAF70AF83E2E8F4E2A4D242600881A7
:1028F00096D000E29DD0098192D000E299D00A8161
:102900008ED000E295D01985112321F00B8187D05C
:1029100000E28ED000E28CD04C7F3DCF11270D9B82
:10292000FDCF1A95E1F7F89400931C0110E810937D
:102930001F01F0921B01F0921D011D98159A7894C9
:1029400087E691E00197F1F797988F9A89E48A9545
:10295000F1F7E0E2F1E08FE090E00E94190E1598A7
:102960001D9A10911F01127031F4E0E2F1E00E9413
:10297000290EB8F718940895F0921D01E0E2F1E0F5
:1029800087E090E00E94190E10911D01112339F487
:10299000E0E2F1E00E94290EB8F718940895009142
:1029A0001E01F0921D010895ECEFFFEDEBBEA79123
:1029B000B6910A2F0F71D9F01B2FAA0F111FAA0F62
:1029C000111FAA0F111F1F7091F01D3080F42B2FC3
:1029D00026952F73293058F00F9308E229D0022F43
:1029E00012D0012F10D00F910ED009E221D00895FE
:1029F000EB0DFF1D85919591FC010591002311F0D0
:102A000017D0FBCF0895005D07FF0053085E06FF57
:102A10000851045F05FF0C500A5F04FF06500F9336
:102A2000029501D00F910F700A3008F0095F005D28
:102A300040FD0E94E40C41FD0E94580D42FD0E94A1
:102A400042170895E2E9FAE224E000278591959182
:102A5000A81BB90B10F00395FBCFA80FB91F0023DB
:102A600021F400E20AD0002703C0006306D000E38F
:102A70002A9561F70A2F0063DBCFEF93FF93AF93A3
:102A8000BF932F93D5DF2F91BF91AF91FF91EF911E
:102A900008951027E80364000A000F93C0DF00E2E6
:102AA000C7DF0F910895003208F40EE2C1CFA0E015
:102AB000B1E0AED117E783EC94E007C2A0E0B0E04C
:102AC000A7D100E210EF25E3E2D100EB17E783EC9A
:102AD00094E0F1D100E210EF25E3D9D14C7F4460BE
:102AE000A0E0B0E095D1E0ECF0E0A4D10E94D414D5
:102AF000E6EEF0E09FC12897A591A883B591B98330
:102B000015911A8312501B8315911C8312501D833B
:102B100015911E8315911F837BD11E8176D10AEDFD
:102B2000B1D104EC2B81B8D10FEBACD1A881B98124
:102B3000B395B9836DD11E8168D103EBA3D100E2B7
:102B40002B81AAD103EB9ED12F8120FF03C011E07E
:102B500021E0A7D12D812A952D8341F7A881B98144
:102B6000B395B98355D11E8150D100EC8BD104ECC3
:102B70002B8192D109ED86D12F8120FF03C011E076
:102B800021E08FD12F8120FF08C0A881A395B981B2
:102B9000B3953ED111E02A8184D11E8136D1289689
:102BA00008956197EA83FB83FC82F98287DFEA81DB
:102BB000FB81A591AD83B591BE83BF831591188725
:102BC000159119871A8715911B8715911C871591E7
:102BD0001D8715911E8715911F871591188B1985D3
:102BE000110FE10FFF1D0885025019851395019FF4
:102BF0001B2D169521F0E00DF11D1A95E1F708D176
:102C00001B8503D10AED3ED104EC3CD1288522502E
:102C100030D104EC37D10FEB35D1AD81BF81B39505
:102C2000BF83F6D01B85F1D003EB2CD100E22AD173
:102C3000288522501ED100E225D103EB23D111E0DB
:102C400021E02FD12A852A952A8739F7AD81BF81C6
:102C5000B395BF83DDD01B85D8D000EC13D104EC35
:102C600028851AD109ED0ED111E021E01AD1AD81EC
:102C7000A395BF81B395CCD011E028852E5F11D1EB
:102C8000ED85FE8500E00995AD81A395BE81B395E4
:102C90001C81B10FBDD01C85288503D10E94FC0F7B
:102CA000C1F00A3559F10537B1F10237E9F10D37B5
:102CB000F1F00C36E1F00A37D9F00936C9F011FD10
:102CC00008C00637C9F00835A1F00E3799F0053075
:102CD00091F0FE010E94290E08F7ED85FE8501E0C6
:102CE0000995FE018F8598890E94190ED7CF27C0BC
:102CF0002BC03EC067C02EC061960895D8DEEA8121
:102D0000FB813A961C81110FE10FFF1DA591B59132
:102D1000FD0109954ACF1C81112309F4BFCF60D072
:102D20001C811A951C83B0CF1C8109850A95101748
:102D300008F0B4CF55D01C8113951C83A5CF1C81FE
:102D40004FD011271C83A0CF1C814AD019851A951A
:102D50001C839ACFACDEE8E6FDE2CDDEE0E5F6E0EE
:102D600064D00E94EF0F21CF030D2509CF012296D9
:102D70000B2D0E5F043008F00027B02E069583E07F
:102D80009FE00E94602693DEEEEBFDE2B4DE1EE9DA
:102D90003CD0ECEFFBE049D02297FE0180ED97E0BC
:102DA0000E94190EFE010E94290E38F00E94FC0FAD
:102DB000C9F311FD02C00835D1F22296F6CE0D0BF3
:102DC0001B039F0110E8A1260A2D00781FEA0E942C
:102DD0006F170A2D82E09FE00E9460260AD0E5CEA0
:102DE000AD81A395BE81B395B10F12D01B85288507
:102DF00058C00DEE11D941F04DD931F00A3F21F400
:102E000000E0A7FE01E008D90895012F1AEA67C083
:102E100015E3B19FBB27A00DB11D1197B77018EA3C
:102E20000A2F5DD019EA0B2F5AC0EB0DFF1D8591BB
:102E30009591FC01C09A1CEA1FB958D00591002356
:102E400071F0053121F0063131F04ED0F7CF059108
:102E50001AEA45D0EFCFA591B591DADFEBCF08950F
:102E6000C09A1CEA1FB942D001913ED02A95E1F7E1
:102E70000895C09A1CEA1FB939D0059135D02A951A
:102E8000E1F708951F931CEA2AD01F9108950F932C
:102E9000012F1AEA24D00F911CEA21D02A9531F48F
:102EA0000895012F1BEA1BD02A9521F0C098C09AE3
:102EB0002A95E1F708950F93012F1AEA10D00F9188
:102EC0001CEA0DD0019731F40895012F1BEA07D0B9
:102ED000019721F0C098C09A0197E1F708950F93E8
:102EE000C09A1FB903D00F91C0980FB9779BFECF3E
:102EF0000FB1C09A08953F933FB7C0FC0E943619A6
:102F0000C1FCE09204013FBF3F9118950FEF5BD0E9
:102F10001A95E1F708950F9312E0F8DF0F9153D05F
:102F2000002751D000274FD000274DD000274BD08D
:102F30000FEF49D007C012E0E9DF16E0059143D05A
:102F40001A95E1F710E20FEF3ED00F3F11F41A95FA
:102F5000D1F708950091260102FD07C0880F991F3F
:102F6000AA1FBA2FA92F982F88270FEF2CD001E581
:102F70002AD00B2F28D00A2F26D0092F24D0082F93
:102F800022D00FEF20D08FEFDDDF8A95D1F00E3FFA
:102F9000D9F74F9343FF0AC0427F4260EF93FF93FC
:102FA000E6E0F3E10E94FD14FF91EF9180E092E0F2
:102FB00009D001930197E1F74F9113E0A7DF9894AF
:102FC000089508950FEF43FF8FCF4F934A7F4260DC
:102FD000EF93FF930F93E2EFF1E10FDD0F910F936A
:102FE0001EDD0F91C0980FB9779BFECF0FB1C09A2D
:102FF0000F93EAEFF1E101DD0F910F9310DD0F91D7
:10300000FF91EF914F910895ECEBF1E374DDE2EC69
:10301000F1E371DDE8ECF1E36EDDEEECF1E36BDDA5
:10302000E4EDF1E368DDE0E1F8E0FFDEEAE4F8E09A
:1030300001DFE0E3F8E0F292EE23E9F7FABADBBA57
:10304000F4BAF5BAE0E0F8E0A09AA9D0A098A19A65
:10305000A6D0A198A29AA3D0A298A39AA0D0A398F0
:10306000A49A9DD0A4980091630025E09DD003B35D
:10307000001F001F001F22E097D0E0E0F8E0ABE067
:10308000B9E0C6DE03817FD003857DD003897BD084
:10309000038D79D003A177D004A175D0048D73D0AE
:1030A000048971D004856FD004816DD0ABE0BAE0A3
:1030B000AFDE028168D0028566D0028964D0028DBD
:1030C00062D002A160D005A15ED0058D5CD00589DB
:1030D0005AD0058558D0058156D0ABE0BBE098DECC
:1030E000018151D001854FD001894DD0018D4BD048
:1030F00001A149D006A147D0068D45D0068943D00D
:10310000068541D006813FD0ABE0BCE081DE008186
:103110003AD0008538D0008936D0008D34D000A157
:1031200032D007A130D0078D2ED007892CD007854B
:103130002AD0078128D0A6E2BAE06ADE03A523D010
:10314000A4E2BBE065DE01A51ED004A51CD000A54D
:103150001AD0A6E2BCE05CDE02A515D0AEE0BFE06E
:1031600057DE06A529E010D0AEE1BFE051DE05A58F
:1031700028E00AD00E94FC0F11F0063709F062CF58
:10318000F4BAF5BA089521E01FED037021F01EEAAC
:10319000033009F011ED85DE1FED21E082CE00271E
:1031A0000A95F1F709B328E010811E7F079508F012
:1031B000136011932A95C1F7989408950706260C79
:1031C000DF0109081706DF0022090905DF000C0EE0
:1031D0000D03DF001C0E0C03DF002197ECEBF2E384
:1031E0000E947B15E4ECF7E00E94151701E014E55E
:1031F0000E946F1707E00883A4E1BAE00E94081755
:103200000881000F000FE2ECF2E3E00FFF1DA59133
:10321000B591EF93FF930E942215FF91EF910591D5
:103220000093240105910093250113E5C09A1FB96D
:103230000E94761701E0C02E0E94EF0FCC240637C3
:1032400079F0053719F0023731F0F4CF08810E30EC
:1032500088F70395D0CF0881002361F30A95CBCF7F
:1032600000E014E50E946F17219608950F93BF9315
:103270008F939F93EF93FF93FFEFB0912201E09123
:1032800023018091240190912501B80FE91F049139
:10329000C0980FB9779BFECF0FB1C09A0C30A8F33E
:1032A000B0932201E0932301FF91EF919F918F91C1
:1032B000BF9100E4009358000F910895080820067C
:1032C000DF014B002D006B00400098005B00D60032
:1032D00080002E01B500AB0100015C026A015603BB
:1032E0000002B804D402AD0600047109A8055A0D05
:1032F0000008E112500BB41A0010C425A1164000BA
:103300000000009548000001AA875000000200FF5D
:10331000E0935C01F0935D0112EA0FEF0E946F17DA
:1033200010E2F4DD11EA0FEF0E946F172FEFEEEFBE
:10333000F2E301DE2A9511F401E09AC10130B9F7F8
:10334000E4E0F3E3F8DD80E002FF80E414E0DEDD9A
:1033500007E7E1DD12E0DADD09E635DE082F33DECE
:10336000E1DD002351F002FFF3CF01E4D4DD0023BF
:10337000E1F74FD153D110E10FC04BD14FD111E044
:10338000882351F00AE7C7DD1DDE0F9315E0BEDD8F
:103390000F9112E006FD16E010932601EEE5F1E034
:1033A000D192D192D192D08280E090E0A0E0B0E0C2
:1033B00064D13AD111F003E05BC1EEEB00810F77ED
:1033C000A1F4E2EC0081013051F0043041F006300C
:1033D00031F00B3021F00C3011F00E3031F4E6EC0E
:1033E00081919191A191B0812CC0E0E0F6E035850A
:1033F00000E010E028E037950F1D2A95E1F70A95C7
:1034000009F4139506850784002909F013950389AB
:103410000488002909F4139500A101A0002902A045
:10342000002903A0002909F413950589007F003FB6
:1034300009F41395143009F0BECF80E090E0A0E0CD
:10344000B0E08093340190933501A0933601B0939E
:10345000370113D1E9D009F0AECFE0E0F6E0038503
:10346000002319F40485023011F004E001C1A0E04A
:10347000B0E086899789092F082B21F484A195A1B2
:10348000A6A1B7A180932E0190932F01A0933001A4
:10349000B0933101A0E0B0E083899489092F082B13
:1034A00021F480A191A1A2A1B3A180933C019093AA
:1034B0003D01A0933E01B0933F0181899289A0E034
:1034C000B0E0092F082B19F000E1ECD1DC01BF932B
:1034D000AF9300890093280180912E0190912F01D4
:1034E000A0913001B09131010A95880F991FAA1F50
:1034F000BB1F0A95D1F76F917F91EDD166857785D6
:103500006093320170933301E6D180933801909338
:103510003901A0933A01B0933B01ECE3F1E0C5D14E
:10352000E0E0F6E00585013408F09FCF0093290123
:10353000B9D18093400190934101A0934201B0938F
:10354000430102E0BB2359F4AA2349F4853F9D05BA
:1035500030F401E01FE0853F910708F400E000939C
:10356000270180E090E0A0E0B0E0002331F00A9570
:1035700021F084A595A5A6A5B7A580932A019093CF
:103580002B01A0932C01B0932D0180934C019093BB
:103590004D01A0934E01B0934F0180913201909163
:1035A0003301A0E0B0E0E4E3F1E08CD1809344018A
:1035B00090934501A0934601B0934701EEE2F1E0FC
:1035C00081D18093480190934901A0934A01B0931F
:1035D0004B0180912A0190912B01A0912C01B09177
:1035E0002D018F939F93AF93BF9311E0082E092A6B
:1035F0000A2A0B2A39F01F93C4D0B1D01F9110F4BE
:103600001395F9CF10935001BF91AF919F918F9176
:1036100008950BE780DC0023E1F70895EAE0F3E387
:103620008ADC0023D9F70895EEEFF7E00191053524
:10363000008109F40A3A089543FF14C04F93427F72
:103640004260E6EFF2E10E94FD140B2F0E940F157D
:103650000A2F0E940F15092F0E940F15082F0E9494
:103660000F154F91E0E0F4E075DC09F0089502E0F9
:10367000E0915C01F0915D010994EEE5F1E00191CA
:10368000081749F40191091731F401910A1719F447
:1036900001910B1741F180935E0190935F01A0931C
:1036A0006001B093610143FF14C04F93427F4260B9
:1036B000E6EFF2E10E94FD140B2F0E940F150A2F76
:1036C0000E940F15092F0E940F15082F0E940F1539
:1036D0004F91E0E0F6E03EDC51F2E0E0F6E043FF3F
:1036E00008950E949F0DE0E0F6E008958F939F9368
:1036F00011EA0FEF0E946F17A0E0B0E000E1D2D016
:103700008F93009129010F93CDD0009150010A951C
:10371000081738F40F910F919F918F910FEF0023AD
:103720000895A0914E01B0914F01082F0023809180
:103730004C0190914D0129F00F9323D00F910A95E0
:10374000D9F785D00F900A940F910021800F9F1D0B
:10375000AF1DBF1D92DF9F918F91002708951FE03D
:1037600000912701002319F4873F910708950A95D6
:1037700019F4873F9D050895873F9D05AD05B10765
:10378000089511EA0FEF0E946F170091270100239F
:1037900039F10A9579F0880F991FAA1FBB1F082FCE
:1037A000892F9A2FAB2FBB270AD03196A191B081D8
:1037B000BF700895A0E0B0E0082F892F99270F93DC
:1037C000AF93BF93E4E4F1E07DD057DFBF91AF91B9
:1037D0000F91E00FFF1DE00FFF1D81919081089573
:1037E000FC01EE0FFF1FE80FF91FF695E795082F74
:1037F0008F2F9927AA27BB2786950F93EF93FF93C7
:10380000E4E4F1E05FD08F939F9337DF9F918F9136
:10381000BF91AF91B170EA0FFB1FA191F83031F465
:10382000AF93A0E0B0E0019628DFAF910F919081B7
:103830008A2FA0E0B0E0069540F49695879596957E
:10384000879596958795969587959F7008950B2FE8
:103850000A2B092B082B59F4E8E4F1E080912E01A2
:1038600090912F01A0913001B09131012BC00297AE
:10387000AF09BF090091290104C0880F991FAA1F31
:10388000BB1F0695D0F7E4E3F1E01CD0E8E3F1E0DC
:1038900019C0892F9A2FAB2FB0E001E0B695A795FC
:1038A000979587950795D0F708950191081B802F6C
:1038B0000191090B902F01910A0BA02F00810B0B96
:1038C000B02F08950191800F0191901F0191A01FC9
:1038D0000081B01F0895860F971FAF1DBF1D08956B
:1038E000D8DFEEE2F1E0E1DF082F007F092B0A2BA1
:1038F0000B2B089511EA0FEF0E946F17E7E5F1E037
:1039000001911191012B1191012B1191012BE1F1E9
:103910008091520190915301A0915401B0915501B1
:1039200096DF00915101800F9F1DAF1DBF1D84DEEA
:103930008091520190915301A0915401B091550191
:103940000091510103950093510110912901101725
:10395000C9F4F092510115DF809352019093530105
:10396000A0935401B0935501E7E5F1E000810150C7
:10397000019300810F09019300810F0901930081D8
:103980000F0901930FEF0895809152019091530117
:10399000A0915401B09155015ADF00915101800F5F
:1039A0009F1DAF1DBF1D48DE00915101039500937F
:1039B000510110915601011B0895E0936201F093AB
:1039C0006301E4E6F1E010E8118310E0128318E0EF
:1039D0001383D6820895E4E6F1E0008111816281CB
:1039E0007381A481B5810680E0916201F091630149
:1039F000002012F0C1F062C00790E0936201F093E2
:103A00006301E4E6F1E0F68200831183A483B583C9
:103A1000A62FB72F0D92B850B770B85FA283B383AB
:103A2000002D9894089592E08FEF110F11F41791E3
:103A3000111F881FD0F79A9549F402E0859580F010
:103A40000395839551F093E08FE3EFCF9A95B1F40E
:103A5000869590F29395E9CF080F94E08FEFE5CF2C
:103A60008395D1F49395879560F1991F110F11F407
:103A70001791111FC0F7090F96E0D7CF9A9511F44F
:103A800001E00BC09A9529F4839531F495E08FE11C
:103A9000CCCF9A9509F7982F87919A95A82FB92F8F
:103AA000A60FB71FB850B770B85F0D90E0936201D2
:103AB000F0936301E4E6F1E0E682A6CF0A9591F780
:103AC000B2CF18940895160209159F4368697000D3
:103AD00049443A2000003A204D3239463034300013
:103AE0003A416D3239463034300016020A159F4390
:103AF00052433A20000016020B5344636172643A49
:103B000020464154000016130E159F205BFB5D20DC
:103B100045726173652063686970200016010B159A
:103B2000AE00000111079F00000811069F0011015F
:103B3000240D9F00000E350A9F000B041F06CF01C5
:103B40000B041F06AF01202020203F3F3F3F2020D5
:103B50002000202020656D70747920202000A802AC
:103B6000990C7A7820626173696334382000C859EF
:103B7000C0837A78206261736963313238007106DC
:103B80007A7A74722D646F73202020202000446F95
:103B9000D787616C636F676C756B70656E004845A5
:103BA000474C6865676C756B2020202020004556C7
:103BB0004F4465766F646F732020202020004144BD
:103BC000444F6164646F6E732020202020005253A4
:103BD000545F7273745F30382020202020005052D0
:103BE0004F4670726F662D726F6D2020200051431A
:103BF00020337163332E78782020202020001E652A
:103C00001EB361746D325F63706D20202000BCA410
:103C10002C297862696F732073746D6E7500272E7E
:103C200023687674722D646F732020202000203C5E
:103C30004449523EB30042D000E949D017EA03E0BC
:103C40004ED980E090E060E070D0E02F81E06DD050
:103C5000F02F34C0E0E0F4E0A0E0B2E000810F3FDC
:103C6000E1F000EA34D017EA01E039D913EA082F6D
:103C700036D914EA092F33D916EA008130D917EA68
:103C800005E02DD901E030D903E02ED916EA27D975
:103C90002BD91081012707FDFBCF31960196119793
:103CA000E9F6089500E813D000E111D017EA03E027
:103CB00016D916EA14D918D907FFFDCF00EF07D09F
:103CC00082E18A95F1F717EA03E009D908950F9385
:103CD00017EA01E004D913EA05E501D914EA05E57C
:103CE000FED816EA0AEAFBD817EA05E0F8D801E0A0
:103CF000FBD813EA0AEAF3D814EA0AE2F0D816EA83
:103D000005E5EDD817EA05E0EAD801E0EDD813EAB9
:103D100005E5E5D814EA05E5E2D80F9116EADFD803
:103D200017EA05E0DCD801E0DFC815EA062FD7D88E
:103D300014EA092FD4D813EA082FD1D816EA0FEFC6
:103D4000CEC817EA0BE0CBD88827EFDF01C0CCD86C
:103D5000019320230E946F2601966F1D1197B9F7DA
:103D6000089566974C7FFB8AFC8A02E80D8BA0E0E1
:103D7000B8E020E200E80D931FE0FD921A95E9F704
:103D80002A95C1F7E2E2FBE30E947B15E8E2FBE340
:103D90000E947B15EEE2FBE30E947B15E4E3FBE36C
:103DA0000E947B15E8E1FCE00E941517CAD40FE0E1
:103DB0000C8BE6ECFAE30E941A173DDFE13029F4A0
:103DC000F43A19F4E0EEFAE306C0E03239F4F23ED8
:103DD00029F4E6EDFAE30E941A1711C0EF93FF935E
:103DE000E0EDFAE30E941A17FF91EF910E2F0E9467
:103DF0000F1500E20E9418150F2F0E940F15E2EC1C
:103E0000FCE00E941517D98AFA8A61D663D7222767
:103E1000992766272E839C836D83E6E4FBE3E0937A
:103E20006B01F0936C01E0E0FAE0A0E0B4E02FEF6A
:103E300088DF20936D012497E6E9FAE0AFE6B1E070
:103E40006CD7EEE5FBE336D621F1E0E8FAE0A0E836
:103E5000B0E063D7EEE6FBE32DD6D9F0E3E6FDE074
:103E6000A8E0B0E05AD7EEE1FCE324D691F0E0E020
:103E7000FAE0A7E0B0E051D7EEE0FCE31BD649F052
:103E8000E0E0FAE0A8E3B0E048D7EEEFFBE312D6BB
:103E900021F4E0936B01F0936C01249688279C81B8
:103EA0009C5F6D81A0E0B8E317EA0BE018D8209181
:103EB0006D013BDF01C018D8202311D7019611975F
:103EC000D1F720936D019C81945C6D81E0E0FAE074
:103ED000A0E0B4E036DFE2E5FBE3239521F4E093D4
:103EE0006B01F0936C012497E8EFFDE000801180F6
:103EF00022803380EEE9FBE3DDD561F1EEEAFBE3FE
:103F0000D9D541F1EEEBFBE3D5D521F1EEECFBE3A6
:103F1000D1D501F1EEEDFBE3CDD5E1F0EBE9FBE02E
:103F20000080118022803380EEEEFBE3C3D591F058
:103F3000EFE2FBE0A9E0B2E0F0D6EEE8FBE3BAD5B1
:103F400049F0E0EBFDE0A0E4B0E0E7D6EEE7FBE30C
:103F5000B1D521F4E0936B01F0936C012496E091CC
:103F60006B01F0916C01A5E0B8E00E8110E1019FBA
:103F7000A00DB11D2BE005910D932A95E1F7A7D572
:103F80000E94FC0F29F011FD03C0063709F472C02E
:103F90009C816D8110E4910F6F1D2E81239525FF6B
:103FA00039CFBDD6EAEEFAE30E941A170B810E94C0
:103FB0000F150A810E940F1509810E940F150881B3
:103FC0000E940F15EEE0FDE00E9415171DB710933B
:103FD00005011EB710930601C0930701D093080195
:103FE000EDEDF1E295D9AF93BF938F939F93E6EFF9
:103FF000FAE30E941A176091270101E312E3662396
:1040000029F016E36A9511F003E312E31F930E946F
:1040100042170F910E9442179F918F91BF91AF91CC
:10402000B1D3DC862CD4FC860D890F710D8B89D31E
:104030000E94EF0F053741F0023779F00A35A1F001
:104040000637B1F701E0F2CF0D89069588F31C8998
:10405000102309F4FACF0D8BE7CF0D89000F40F341
:104060001C891023C1F7FACF0D891C89012301F3A4
:10407000069510F466960895069508F473CE069595
:1040800008F4C5C1069528F40D8900680D8B59D335
:10409000E0C1069508F0CCCF0D8900680D8B51D397
:1040A000EEEEFDE00E9415170E94EF0F11FD02C019
:1040B000053351F0A2E0BCE00E94081700E21FE9BE
:1040C0002DE00E944717B0CF1EE00E9405170B8914
:1040D00020E0069518F50F932F93220F220F2F93B0
:1040E00024D505E42CE00E944C172F9123952F93A3
:1040F0001CD505E42CE00E944C172F9123952F939B
:1041000014D505E42CE00E944C172F9123950DD572
:1041100005E42CE00E944C172F910F912395283035
:10412000C1F6EAE1FEE00E9415170B890F3F11F47A
:10413000B9DD2DC06FEF63950695E8F70F936F9388
:1041400000E8C5DD15EA0F910F930E946F1700E399
:10415000BEDD6F910F916395683068F40695D8F7CE
:104160000F936F9315EA062F0E946F1700E3D6DDB9
:104170006F910F91F0CF17EA03E00E946F1716EAD4
:104180000E946F170E94741703FFFCCF8FDDE6E4D7
:10419000FEE00E9415171AE00E94051720E02E830A
:1041A000E0E0F8E010E1129FE00DF11D80818F73D7
:1041B00011F0813208F055C08A8B9927AA27BB27B6
:1041C000108116FD80960197009129010A95082318
:1041D0000395009356010091290164DB80935701F8
:1041E00090935801A0935901B0935A01F092510154
:1041F00081819281A381B481809352019093530174
:10420000A0935401B0935501108116FF06C020E21F
:104210002F9370DB2F912A95D9F72E8186D4992779
:104220006E81669597956695979515EA062F0E947B
:104230006F17A5E5B5E0AD87BE879F935BDB9F91C8
:10424000882708DDAD85BE85B25038F407E50E94A9
:10425000421715E5A10F15E0B11F1A891A951A8B9F
:1042600051F72E81239525FF9ACF28DD17EA03E029
:104270000E946F17E2E7FEE00E94151720E02E83F0
:10428000E0E0F8E010E1129FE00DF11D80818F73F6
:1042900011F0813208F071C08A8B9927AA27BB27B9
:1042A000108116FD80960197009129010A95082337
:1042B00003950093560100912901F4DA8093570188
:1042C00090935801A0935901B0935A01F092510173
:1042D00081819281A381B481809352019093530193
:1042E000A0935401B0935501108116FF06C020E23F
:1042F0002F9300DB2F912A95D9F72E8116D4992779
:104300006E81669597956695979515EA062F0E949A
:104310006F17FF86F88AA5E5B5E0AD87BE879F9346
:10432000E9DA9F918827E0E0F4E0A0E0B2E017EA44
:104330000BE00E946F17FCDC02C00E947417119101
:10434000011711F0EF86E88A01961197B1F7AD8554
:10435000BE85B25070F40F851CE000FD1EEA0E947D
:10436000051706E50E944217FF8615E5A10F15E027
:10437000B11F1A891A951A8B81F62E81239525FF74
:104380007ECFEEE9FEE00E941517EAE3FBE3088921
:10439000002311F0E0E4FBE30E947B15EAECFEE071
:1043A0000E941517E4E0FFE0088911F0E0E3FFE068
:1043B0000E9415170E94EF0FD5CCF89410910501BB
:1043C0001DBF109106011EBFC0910701D0910801C9
:1043D00078940F93ECE1FBE30E941A170F91EAE344
:1043E000FDE0013071F0EEE5FDE0023051F0E2E871
:1043F000FDE0033031F0E6EAFDE0043011F0EAECD4
:10440000FDE00E94151707E00C8B02E00FCEA0E044
:10441000B8E011E00B89012399F40B89012B0B8B78
:1044200024E0FD92FD92FD92FD92FD92E2E5FBE318
:104430008BE005910D938A95E1F72A9591F702C0DB
:1044400090969096110F30F70C8900610C8B3FD33A
:10445000EBCD15D20E94EF0F0537D1F0023739F1BD
:104460000D37A9F10A37D9F10C36A1F1093671F0EF
:104470000A3569F0063771F7BC85BE5FA2E10E947C
:1044800008171FE922E20E945117CECD3CC04BC055
:104490000B850023F9F20A950B870C85002319F090
:1044A0000A950C8703C00A850A950A87D2CF0B8527
:1044B00019850395011770F60B870C850A3018F4DF
:1044C00003950C8703C00A8503950A87C2CF0B8525
:1044D0000A5008F400270B870A87FC86BACF198593
:1044E0001C3028F40AE00B87FA860C870BC00B857A
:1044F000065F011710F0012F0A950B871AE01C8741
:10450000011B0A87A6CF19851C3028F40AE00B8707
:10451000FA860C8707C0012F0A950B871AE01C87C3
:10452000011B0A8796CF0B85E0E0FAE010E2019FBD
:10453000E00DF11D03850023E1F0828D938DA489A8
:10454000B589182F192B1A2B1B2B41F480912A01A6
:1045500090912B01A0912C01B0912D0180934C01E1
:1045600090934D01A0934E01B0934F010BD1FC8667
:1045700070CFEF83F887848D958DA68D0FEF1FE3A5
:10458000800F911FAF1D990FAA1F990FAA1FAA8B09
:10459000F98ABC85BE5FA2E10E9408171FE122E2F2
:1045A0000E94511794D20E94EF0F0537C9F00237CD
:1045B000E9F00B3639F0043759F00A3509F10637BE
:1045C00091F76DC00989002371F30A95098BEACF31
:1045D00009891A89100F103230F70395098BE2CF41
:1045E0000989045008F40027098BDCCF09891A894E
:1045F000010F0C5F003208F000E2011B098BD2CFE3
:10460000E0E0F8E0098910E1019FE00DF11DEC8385
:10461000FD831091290110935101EF81F885828D5E
:10462000938DA489B5898093520190935301A093EF
:104630005401B0935501848D958DA68DB78D6FEF84
:1046400071E049D926D920E2809730F129F18D8790
:104650009E8729D020E22E83009151010A95A1F472
:104660008091520190915301A0915401B091550154
:104670000E94C11B8093520190935301A093540157
:10468000B093550100912901009351012E812A9583
:1046900011F78D859E85D7CF8096282F04D0D98A93
:1046A000FA8A15D2C1CC2F9311E009890695069597
:1046B000002319F0110F0A95E9F70B890123D1F4B2
:1046C0000B89012B0B8BA0E0B8E009890C7110E17C
:1046D000019FA00DB11D24E0FD92FD92FD92FD927F
:1046E000FD92E2E5FBE31BE005910D931A95E1F7DE
:1046F0002A9591F72F9100912901109151010117ED
:1047000009F02064AC81BD812D93009152010D937D
:10471000009153010D93009154010D9300915501A7
:104720000D93EF81F8852BE001910D932A95E1F728
:10473000AC83BD830C8900610C8B09890395098BBF
:104740000895222711E02E831D87B22FBE5FA1E0BE
:104750000E9408170D85AC891FE9A02309F417E909
:10476000AD890A2329F0AA0F10F010EF01C01F71C4
:104770002FE00E9451172E8123951D85110F15FFE3
:10478000E2CF0895E0E0FAE0EF83F887F986FA8651
:10479000FB860E94F11A80E090E00E94761B07C021
:1047A0000196B096F83019F40E94761B81F41081BE
:1047B000153EB1F3112359F01E3219F411811E3246
:1047C00079F703850E7D21F0003151F71FC031C00C
:1047D0000085023549F0023419F70185093401F7E3
:1047E00002850E3439F0DCCF01850F34C9F602851D
:1047F0000D34B1F6078D002399F6068D158C048CC7
:104800000E181F080F0960F2083050F6AF81B88506
:1048100020E2EF93FF9301910D932A95E1F7FF9129
:10482000EF91AF83B887298523952987203350F4EA
:10483000B7CF2985213081F0222321F40C8907701C
:104840000C8B0AC0E0E0FAE0662779857A95008152
:104850000E3209F46395CDD0E0E0FAE029850385B6
:104860000E7D038741F41BE0008188D001931A95E7
:10487000D9F7759601C0B0962A9589F70895222731
:104880002F93B22FBE5FA2E10E9408170C851FE98B
:10489000021709F410EF0E9405170A85020F198507
:1048A000011768F0212B31F4EEE9FCE00E941517A6
:1048B00026E101C022E200E20E944C1759C0E0E06C
:1048C000FAE010E2019FE00DF11DEF9328E00E9455
:1048D000301700E20E94421723E00E94301703EBDA
:1048E0000E944217EF91EF93FF930385002329F075
:1048F000EEE2FCE30E941A1707C0848D958DA68D09
:1049000051D003EB0E944217FF91EF91008D0F7180
:104910000E9403150EE20E944217008D118D17951B
:10492000079502950F700E9403150EE20E94421730
:10493000018D0695005B043610F00456FCCF0E94F2
:10494000031503EB0E944217078906950695069505
:104950000E9403150AE30E94421716890789111F56
:10496000001F111F001F111F001F0F730E9403154E
:104970002F9123952B3008F483CF0895013488F0CC
:104980000B3570F0003868F0003950F0003A30F024
:10499000003F38F0083F28F401600895005B089557
:1049A000005E0895E8EEF9E425E02E2C002705903E
:1049B000159080199109A20910F00395FACF800D86
:1049C000911DA21D002329F400E20E944217002736
:1049D00004C000630E94421700E322242A9539F79D
:1049E000082F00630C944217A0861027E803640088
:1049F0000A0067170CF00895962F970F9695862F4B
:104A000027D0262E2394372E3214B4F0721534F0AA
:104A1000862F922D33D010F02394F8CF361634F031
:104A2000862F932D2BD010F43A94F8CF23141CF436
:104A3000822D932D0DD0E8CF862F932D09D03F9254
:104A40007F93732D7A95D5DF7F916F916395D1CF49
:104A5000891709F40895EF93FF93DF0120E2829F05
:104A6000A00DB11D929FE00DF11D0C9110811D93C1
:104A700001932A95D1F7FF91EF910895EF93FF935A
:104A8000DF0100E2909FA00DB11D809FE00DF11DA0
:104A900013851E7DA55F0C910E7D011741F4AB506F
:104AA0002BE00D911191101711F42A95D1F7FF9178
:104AB000EF9108950591001549F40591011531F420
:104AC0000591021519F40591031501F40895E0E02C
:104AD000F8E022272F8729D000811EE007FD17E08C
:104AE0002F850989201728F0BA890B0F201708F4A1
:104AF00010EFBF8500E1B2FD10270E940517359623
:104B000028E00E94301700E20E94421723E00E9432
:104B100030172F8523952032E8F20B890F3F21F4BF
:104B2000E6E0FBE30E941A170895A22FA3701DE090
:104B3000A19FA02DA395B22FBC71B695B695B15F7C
:104B40000C9408172197A0E0B0E00E94081700E03D
:104B500010E08DE295E00E945B17AFE0B4E00E94A8
:104B60000817E9EEF0E00E941A170A2D0078039565
:104B700008831FEA0E946F170E94EF0F063731F07B
:104B80000881102F1F70163090F3EFCF0A2D007898
:104B90001FEA0E946F172196089525970C834F9363
:104BA0004C7F11E50E946F17088310EA0E946F176F
:104BB000098312E50E946F170A8310EA0E946F179B
:104BC0000B831A81012B51F41C81112321F017E76B
:104BD0000E9405170BC0E6E2FCE402C0ECE2FCE434
:104BE0000E947B15E6E9FBE00E941517ABE2B4E1F9
:104BF0000E940817A881B9810AD0ABE2B5E10E94F2
:104C00000817AA81BB8103D04F9125960895AF93D1
:104C1000BF93119600E209F40EE30E944217BF9180
:104C2000AF910C9422151E12150577001E12150562
:104C3000AE0021E20027111BAA1FBB1FEE1FFF1FA2
:104C40002A9559F0001F111F081B190B20F4080F9B
:104C5000191F8894F1CF0894EFCF08958F939F93F5
:104C60001F93809102019091030180930301881F9B
:104C7000991F092F881F991F881F991F881F991F27
:104C800009278091010180930201809100018093A6
:104C90000101009300011F919F918F910895E0E21F
:104CA000F0E0F192EC33E9F7E1E6F192E636E9F76C
:104CB0000895E199FECF9FBB8EBBE09A0DB3089596
:104CC000102FF7DF101729F09FBB8EBB1DBBE29A98
:104CD000E19A0895D882D982DA82DB820895EF932F
:104CE000FF93188101271127000F111F000F111FBB
:104CF000E2E4FDE4E00FF11F05911981012708832B
:104D000005911A810127098305911B8101270A83D7
:104D100004910B83FF91EF910895DCDF0DD00880A3
:104D2000009408821980109419822A8020942A8283
:104D30003B8030943B8208950191D1DF1197E1F7D8
:104D4000089500000000963007772C610EEEBA51EE
:104D5000099919C46D078FF46A7035A563E9A395A5
:104D6000649E3288DB0EA4B8DC791EE9D5E088D9D0
:104D7000D2972B4CB609BD7CB17E072DB8E7911DAB
:104D8000BF906410B71DF220B06A4871B9F3DE41DC
:104D9000BE847DD4DA1AEBE4DD6D51B5D4F4C78559
:104DA000D38356986C13C0A86B647AF962FDECC982
:104DB000658A4F5C0114D96C0663633D0FFAF50DEB
:104DC000088DC8206E3B5E10694CE44160D572715D
:104DD00067A2D1E4033C47D4044BFD850DD26BB5EB
:104DE0000AA5FAA8B5356C98B242D6C9BBDB40F922
:104DF000BCACE36CD832755CDF45CF0DD6DC593DD9
:104E0000D1ABAC30D9263A00DE518051D7C81661FB
:104E1000D0BFB5F4B42123C4B3569995BACF0FA52A
:104E2000BDB89EB802280888055FB2D90CC624E92F
:104E30000BB1877C6F2F114C6858AB1D61C13D2DA4
:104E400066B69041DC760671DB01BC20D2982A1050
:104E5000D5EF8985B1711FB5B606A5E4BF9F33D4E0
:104E6000B8E8A2C9077834F9000F8EA809961898F7
:104E70000EE1BB0D6A7F2D3D6D08976C6491015C5E
:104E800063E6F4516B6B62616C1CD83065854E0033
:104E900062F2ED95066C7BA5011BC1F4088257C434
:104EA0000FF5C6D9B06550E9B712EAB8BE8B7C8859
:104EB000B9FCDF1DDD62492DDA15F37CD38C654C1E
:104EC000D4FB5861B24DCE51B53A7400BCA3E23068
:104ED000BBD441A5DF4AD795D83D6DC4D1A4FBF41E
:104EE000D6D36AE96943FCD96E34468867ADD0B839
:104EF00060DA732D0444E51D03335F4C0AAAC97CB4
:104F00000DDD3C710550AA41022710100BBE862012
:104F10000CC925B56857B3856F2009D466B99FE4DD
:104F200061CE0EF9DE5E98C9D9292298D0B0B4A816
:104F3000D7C7173DB359810DB42E3B5CBDB7AD6CDF
:104F4000BAC02083B8EDB6B3BF9A0CE2B6039AD2CA
:104F5000B1743947D5EAAF77D29D1526DB048316A5
:104F6000DC73120B63E3843B64943E6A6D0DA85AB4
:104F70006A7A0BCF0EE49DFF099327AE000AB19E1B
:104F8000077D44930FF0D2A3088768F2011EFEC28A
:104F900006695D5762F7CB67658071366C19E70665
:104FA0006B6E761BD4FEE02BD3895A7ADA10CC4A8A
:104FB000DD676FDFB9F9F9EFBE8E43BEB717D58E47
:104FC000B060E8A3D6D67E93D1A1C4C2D83852F23D
:104FD000DF4FF167BBD16757BCA6DD06B53F4B3647
:104FE000B248DA2B0DD84C1B0AAFF64A0336607A6A
:104FF0000441C3EF60DF55DF67A8EF8E6E3179BEE5
:1050000069468CB361CB1A8366BCA0D26F2536E2A9
:10501000685295770CCC03470BBBB91602222F269A
:105020000555BE3BBAC5280BBDB2925AB42B046AD3
:10503000B35CA7FFD7C231CFD0B58B9ED92C1DAEA4
:10504000DE5BB0C2649B26F263EC9CA36A750A9394
:105050006D02A906099C3F360EEB85670772135750
:105060000005824ABF95147AB8E2AE2BB17B381B9B
:10507000B60C9B8ED2920DBED5E5B7EFDC7C21DF5E
:10508000DB0BD4D2D38642E2D4F1F8B3DD686E8371
:10509000DA1FCD16BE815B26B9F6E177B06F774790
:1050A000B718E65A0888706A0FFFCA3B06665C0BA1
:1050B0000111FF9E658F69AE62F8D3FF6B6145CF2A
:1050C0006C1678E20AA0EED20DD75483044EC2B318
:1050D0000339612667A7F71660D04D476949DB772A
:1050E0006E3E4A6AD1AEDC5AD6D9660BDF40F03B41
:1050F000D83753AEBCA9C59EBBDE7FCFB247E9FF10
:10510000B5301CF2BDBD8AC2BACA3093B353A6A350
:10511000B4240536D0BA9306D7CD2957DE54BF67DD
:10512000D9232E7A66B3B84A61C4021B685D942BFA
:105130006F2A37BE0BB4A18E0CC31BDF055A8DEF4F
:10514000022D161403C2160B0470632F77696E3399
:10515000322016170454455354434F4D160905C3C6
:10516000160B064269742072617465203131353244
:1051700030302020204E6F20706172697479160BD8
:10518000074461746120626974732038161D0746F4
:105190006C6F7720636F6E74726F6C20160B085300
:1051A000746F7020626974732032161E08FB2052DF
:1051B00054532F435453161D09445352202D204954
:1051C000676E6F72656416150A53746172742042BB
:1051D0004552542016190BC216190CB3434F4D20DB
:1051E000706F727416190DB316130E52532D32339D
:1051F00032B3160C0FC216190FC11605105A5820DB
:1052000045766F1610104C61737420736563162613
:1052100010736563160311C3160512527842756642
:1052200066162D125254531605135478427566664D
:10523000162D13435453000002023114DF010903F9
:105240002209DF0009030C03DF00030F2F06DF0034
:10525000030F0A03DF004C7F44602A97E8E3F2E57E
:105260000E947B15EEE3F2E50E947B15E4E4F2E593
:105270000E947B15EAE4F2E50E947B15E0E5F2E589
:105280000E947B15E2E4F1E50E941A17DA82DB82C4
:1052900040619DD0FE0167D00E94FC0F51F00932A1
:1052A000A9F311FD06C0063721F491D04F7E2A964E
:1052B0000895FE010E94290E08F455D01CD00E94CA
:1052C000E40D10910B01103838F70E947D0D21F389
:1052D0000E94580DAE81BF81E885F9851196EF1DBA
:1052E000FF1DAE83BF83E887F987AC81BD8111962E
:1052F000AC83BD83E4CFACE0B2E10E9408172091FB
:105300000E012695239526951CD01EEA959B10EC40
:1053100023E00E9451171FED0E940517ACE0B3E196
:105320000E94081720910B0126952395269509D0F8
:105330001EEAB69B10EC23E00E9451171FED0C945F
:10534000051700E2021B222329F00F930BED0E94A8
:105350004C170F91002321F0202F00EB0E944C17D7
:1053600000E20C94421788EE93E00E94190EA0E22E
:10537000B0E10E940817AA81BB81119631F4FC822A
:10538000FD82FE82FF82F886F986AA83BB830E9493
:105390002215A2E1B1E10E940817AC81BD810E94F3
:1053A0002215FC82FD82A3E2B1E10E9408178A81E6
:1053B0009B81882321F4992311F4DC0106C0AE817E
:1053C000BF81E885F9850E9419260C942215F8946E
:1053D0001091090110930A01F0920B0110910C0138
:1053E00010930D01F0920E01959878940895F89419
:1053F0000024E1E0F0E00192EE31E9F7E0E2F19221
:10540000F131E9F7E394DA941FEF1DBF10E11EBFFD
:10541000A0E0B1E01D93DD92ED92DD9282E09FE08D
:105420000E945926A02E83E00E945926023008F0DF
:105430000027000FB02E0E94480E1FEF109365004A
:1054400010E01093640018E0109362001093610064
:1054500013EF13B910E012B91FEF12BB10E011BB2C
:105460001FED15BB10E014BB19EF18BB17E817BBF5
:105470001FEF1BBB10E01ABBE2E1F2E00E94CD2A55
:10548000009B03C09D9B0CC014C0EAE4F2E00E94A4
:10549000F814009905C0E6E1F2E00E94CD2AF9CFA8
:1054A0002AEA2F93E6E1F2E00E94CD2A2F912A9575
:1054B000C1F7EEE7F2E00E94F81411E01EB910E720
:1054C0001DB91091610011601093610083E98A9504
:1054D000F1F7109161001E7F10936100019BFECFD8
:1054E000E0E0F0E0EBBE0E94DD1C0E94EB1C21F02E
:1054F0000FB9779BFECFF9CF029BFECF10E51DB908
:10550000C0E0D3E0E4ECF2E00E94F81420E00E9456
:105510002E261AEA0E946F170E942E260E947417E8
:10552000009510910101011709F04BC02A95A1F7D0
:105530000FE70E947417E4E1F3E00E94FD1488E293
:1055400092E00197F1F70E94F60C0E942C0F0E9446
:10555000F20D1AB710621ABF19B7106419BF789408
:105560000A2D00781FEA0E946F1700E014E50E94E0
:105570006F170E94611001E010E50E946F17E4E9C7
:10558000F5E50E94FD140E94F916E2E6F4E00E949F
:10559000D115FBCF2D2D2D0D0A000E94F814E6E346
:1055A000F2E00E94FD1400E39D9901E30E941315AF
:1055B000E2E4F2E00E94FD1400E3009901E30C94A0
:1055C0001315E8E1F3E00E94F81480E593ECA0E005
:1055D000B0E00E942E260E947417009510910101E0
:1055E000011709F011960197A1F7E0E4F3E00E949A
:1055F000F8140E942215E9CFFFFFFFFFFFFFFFFF16
:10560000FFFFFFFFFFFFFFFFFFFFFFFFFFFFFFFFAA
:10561000FFFFFFFFFFFFFFFFFFFFFFFFFFFFFFFF9A
:10562000FFFFFFFFFFFFFFFFFFFFFFFFFFFFFFFF8A
:10563000FFFFFFFFFFFFFFFFFFFFFFFFFFFFFFFF7A
:10FF00007F8386898C8F9295989B9FA2A5A8ABAE84
:10FF1000B0B3B6B9BCBFC1C4C7C9CCCED1D3D5D894
:10FF2000DADCDEE0E2E4E6E8EAECEDEFF0F2F3F44E
:10FF3000F6F7F8F9FAFBFCFCFDFEFEFFFFFFFFFF02
:10FF4000FFFFFFFFFFFFFEFEFDFCFCFBFAF9F8F7E9
:10FF5000F6F5F3F2F0EFEDECEAE8E6E4E2E0DEDC01
:10FF6000DAD8D5D3D1CECCC9C7C4C1BFBCB9B6B31A
:10FF7000B1AEABA8A5A29F9C9995928F8C898683E0
:10FF8000807C797673706D6A6764605D5A575451EE
:10FF90004F4C494643403E3B383633312E2C2A27BE
:10FFA0002523211F1D1B1917151312100F0D0C0BE4
:10FFB0000908070605040303020101000000000010
:10FFC0000000000000000101020303040506070809
:10FFD000090A0C0D0F1012131517191B1D1F2123D1
:10FFE00025272A2C2E313336383B3E404346494C98
:10FFF0004E5154575A5D6063666A6D707376797CB2
:020000021000EC
:10000000FF1F627FC23C006088FFFF8008900122D2
:10001000400688C60011FC0304024410014841292F
:10002000F32026F5E61035009AFFD30C10D3040810
:1000300019B1E0EFC6982003644FF301F8FF00F018
:1000400014C00250FF0B400128800481600A0F0297
:100050003028FBF31E05A060E680339AB31280605F
:10006000D30AC0363DE0C6340305B04EF30298FD16
:10007000130486FF98FFC141B380B040D9BF804BC5
:10008000FC4057C290FF026122CB40C216A870FD0F
:1000900098FB10C67C4218030E6041290704308685
:1000A000021061C648C108C00120D93006CCD03149
:1000B0000454E033D363E0208024D9F360A40CD34C
:1000C000846DF0FE96D39604BD1C7ECD083DFA38B3
:1000D000FB800721531EB878406D373C089EACFF6B
:1000E00046F36BD0E0417BF91EC420382FB6E050B8
:1000F000F378F9F0392050FB10531B10DCE9024073
:100100002886F3881ED5F03E6CEFD1AF209021E019
:1001100043CDA00E01C7CF2BD341C94FD302341515
:10012000FAAD0B40C02121A7BF8C88098F0246E1A0
:10013000C00818612360FB8C80110038B368CC3094
:10014000E0EFFDB060044C8005B0F3CCC62CD310BA
:100150007D88FF39339007F453981019401EE00151
:100160003CA01FF1201ECFC083460FE281D93C2066
:10017000CE19013D88E7E0D0037AE5100FE4E0B244
:10018000F3407ED3412C0038FB81666106C24C18D7
:10019000F860090C444AF3C065F30362F319E6DF23
:1001A000CC7AE0C4E6E06040DDD30434F320F39B76
:1001B00010D1FE94B346ED9E05B3110C9052E003AE
:1001C000404AD3FA6E442830FA24FBEFDCFF0618CD
:1001D00080C9B385E6E79C40D30B0272935CF0D3F1
:1001E000819823D76104FD9C302248FBFF445E9830
:1001F0008143090349041C93EB04DF489E086C21EA
:10020000A00189E6E120E95C6030F8C6F023914066
:10021000382E843BE0FF871220244804B5890DF373
:100220008CFD21483006E0FC1AD97D191E7AFA5F50
:10023000AF69DBDA825F748CEE7FE40D034FD4D7B5
:1002400080029F3BF68FE6FF5BF320FF7FC1F65EE7
:1002500098B582EFCB06C120356E83C645BF350306
:10026000EE5FB9EAB3EDF545DC7006F1B92EC25088
:10027000C0607FA3F3D344B30FF8863C08D8FAA834
:10028000BD92048029BB112849F3208344D8F36A26
:10029000A3FA14EC7CF40A70F80D04016F055D3CC0
:1002A00004F9AF114836D222ACF380810C44841D8E
:1002B000B9F83CA00906C018FC500360020C81721A
:1002C0009317424098E30801614704DC20B08BFBA0
:1002D000D8AF5EF00A9F83B0302A85058E109EE06D
:1002E00058000B203C8C3B1157F31360019380FFA7
:1002F000C7F948B33C0EF498D00D7A10DE98AD9053
:10030000FCCA1EC0027840B4D0ECB1843B1CFF3064
:10031000D6FD030B4AE0412C6DAA77BE835830A36B
:10032000642D2D0EF3F48B68F2C620E0F859D3C586
:10033000D29BA7A898209393586144842DF37EA262
:10034000F2B3FC834AA5E0734124E003669BD3E843
:1003500008D4D303C6F782803010FC3224B332961F
:100360005103BC985AB9784B04D346F39CF1B5308D
:10037000FC18090B80FC6BBF2D614D8691301AD3A0
:100380007E204CEF6B3ED8FCD5B208C330ECA0EB1E
:10039000604149953006F5F8DD13610CDC5070B30F
:1003A0001E442A30EFC0CC75F537592508E399D3A0
:1003B000828444B93D80E931B020D382E4006308EF
:1003C00052A5F3E6FF97A47E9B66715D3DFC9644C3
:1003D00076D6DE42898D99AFA9355FE35F73D8CBBE
:1003E000F0AEF6ED46FD7E3290B8300DC0B71F304E
:1003F000E24CF351E146CFB3B64C54D829D01C029D
:10040000F799ED8241FA4C18160379EEBD0AD3181C
:10041000D7C483F9CCE40108EFDBFE04FC9EAFE611
:10042000579884DDA9E56D90AC6F207B8006DC7465
:10043000D699ABD913665981B5804DD3127B50E163
:10044000D31D93B1D44838B770FD809D1440C07A55
:100450000113B930849F316F06C124980AA375F344
:100460000C82F245E99BEA36909FC10BA0B9098046
:100470001F300AF226C12008883F044C024B234655
:1004800082F398FF04F8103039F0F981AF2C2598E9
:100490001983B72F30F0DE76400F8FE6FFED0E02A6
:1004A00090A724F8511983CD4961E0802BE016C54F
:1004B00078E07223A0F6F3035A5096F3DD19F9C2DF
:1004C000777352D42410C9E23020F3026DBEA0FE2F
:1004D00065F3804928E3E00A815FD9AF88B8ACF3BF
:1004E0001D03296682C618A4FFC022BBA3F0FA64CC
:1004F000DDCB3009FDC5036BB6D6AAFF1440FC0561
:100500008B40816A93FF051360444080093269EC97
:100510006B13623E4C808975E628FDEB9880F930BC
:10052000128D0829B410CCC882159AF58CEB069D63
:100530006D20664EFDF7FC41FD596508047329C422
:100540009318D391149D81EAB480A6429BF3212095
:100550002444D3E4B4FFF3B26F31C51CFBC8B2CD61
:10056000544C9EDE85A04047CB56E00299536DD691
:1005700078FEE73370302B60FC988EEBF6C5781070
:10058000B85DF79AD2CC55BB42DF6D3930F4F545F2
:100590005E7D768ABCF9DD09047123BFA94C80D346
:1005A000C884FC79321210181825EECE79980659B5
:1005B000302E408C2F81D0D905D4F7E2ED744C3D1C
:1005C000F8C5A34F473510C010DB21044EEDF932BA
:1005D00001339B0C494F88EEBB73E332F306C80826
:1005E000A4237727F709F826C19722B5710FAF7DAD
:1005F000FE248C542070CEFFCB9050E18341300913
:10060000BB40B58B93FE3F84113111D3F6241804FF
:100610000B9CCAEF1269FCF798F0401EF0C0015A1B
:1006200000165AF5F9C566F528D10C848E0EFFFD2B
:100630003245094901EADE988AF2B3D5585EA569C8
:10064000E28BC6EE67306001D338FC460EBEA52FA4
:1006500093E330FCB8EE9C91093080BDFC2F405FE5
:10066000885FFAB481F5782011D345BF9F6BE5B858
:10067000ED7E61FADE9806C2B7E3534AED903BE0A7
:1006800032C811E02BF85D53BBA62210A784AF1629
:100690008040EB0882019E03C404980273C70A0CD1
:1006A000B2B0BF082F9BE2235DD3B8EA980AFA8361
:1006B000E2305DC6289CC8C182DFCA63CAE2041F5B
:1006C000ED99346610A04FB33FF75D78AD30EB3B4A
:1006D0001614D1A5883F2101A2098190E5101122AD
:1006E000C5C3D3E70413F0FD69E2CDC7E3338CFD46
:1006F000C2FF7B9BA822545C9CABF7A4C40651E5C7
:100700009FED6C0878C81988B0C09724301003AEEC
:10071000F34E8DF16EC083ED5E1381DCF70A225C2F
:10072000327B63172CC964FD7DD3AF0799B9D6110D
:1007300026EF840109CBC8D3D340E610F250FD88E0
:1007400005CCFFBFA2B7F72067BB24027F00595E2C
:100750003B20D1FD0E224C2C927F7A95B4D74E547B
:10076000B9C6812001B5447993AC09B9CCCC084B0A
:10077000D330BD89F87FA998402123FF60140C80F5
:10078000843004021F08580F2060FB212C8201B026
:1007900080A017B3B82F55E454FB8045B90322DD80
:1007A00098009EA8844130ED3962D3112BD33BAE23
:1007B000F0FFFD98B17F0330D70F62B1C505F05D42
:1007C000E2C5F3B2C81D05277C287F81024F19A519
:1007D0004544E0BB018B039D10027810FE9859C878
:1007E00068D359AE0E90B2C85E326602608346ACE2
:1007F000DAC8C2F8C596F1F35FF79E40041F39E0EE
:10080000A50EE0048240666F97C86EE999FF5A987A
:1008100006F030BF7E33C814E0A35FF2A584F30274
:10082000AE6F7B0134B3CDC80125C093C06424BF33
:10083000F39703538FD3B9B0FAA03AFA06C6EE4441
:100840004022B3E32815215712675850590C819B59
:1008500022F38AF74854B9D047EBFEDD4CF920501B
:10086000809075DF2802AE83218CA1222CD3DD9BE2
:1008700045C02333840461FF683E6830627E98F788
:10088000A08A5C743D66B9A0408998E3B3815ED3C9
:1008900020FD8081BB51C079F3A78598EBC0401E35
:1008A0008F17D0EFAEE730085C7A739C2942DD44A5
:1008B0007DC14AD1D3DB9EAF0F3F782FBBE52344E8
:1008C0003FDED8FB80110488AF40ACC29416DD49EE
:1008D00072A842B85046F23BF30905886366BD989A
:1008E0006BE0A4C80B2CAFE2BB2120A857216E57A8
:1008F000C0F26F3DD32540AF5B2E989F53FF180881
:100900001361D7004CBC980A464140C88F03DFF6FC
:100910008499C8F726027CF07F80BAD2D77049E963
:100920001208E018EB0503609F1051302106C1AD9D
:100930002803622043D3C6895E985C3D86B4B930F3
:1009400078BF20DD9807B00073507940BB0B29C8F1
:10095000BA8430F1106902870DED4309604BE0C69F
:100960006BD3E8DB2FBBE623813C1E98FBBCB2BCFB
:1009700098EF35D2F198F31618689362652ADB5E1A
:100980002B35C840942ED3B744F1A5F36B9BC81008
:10099000F92371A7FDFA1206C869E6D2BE98CA0407
:1009A000181FEBA45CCBC8049DFF6207A220B30212
:1009B000EDDB3DA8840902FE3E5C30DD020CCE1664
:1009C000F8FEA012F1C5A65FC8C06041E328080484
:1009D00042C65A7359C8D6202453C869860894C59C
:1009E000B219F0CF9B5D791649A891E0C5440399EF
:1009F00021C831E2EFC6C018CAC8F9CBC6D8E0F9A1
:100A00009F9198BCBBFF0E26BBB6EB08E0BFDB1B7B
:100A1000F23C02F3FC35FF58B6F9F1C5FFAF706246
:100A20009881309231460603784DD4F308DE88F77A
:100A30005626121A3CE06E8434BDC09438CF06228C
:100A4000E00883103419E0E35F7F6995C8C0303E49
:100A5000B0F884110675F30840E8980A2EDFEE8896
:100A600040113FFB42900812016A5FEF860CA07AAA
:100A7000F8AF194F50DD3609FF71AE13483C242002
:100A80009A2011E9A4A8779743CA76B3E24AFF5F98
:100A9000980009FB01048C8084B9502020E99BCA8E
:100AA0004C5FF77F8E0EC3FFFB0DC0DD5410E16B72
:100AB000FAC20408F87F810310AF30016D1839A61F
:100AC0006210C6C30911AF703498F4C5C8D7264068
:100AD0009F98C550E9C579F39222E680B6398E9C7D
:100AE0007FB3470D4540E0413CFAA005F02016F3E6
:100AF00098B3C83D41D37A1EC403DCF6E287C688AA
:100B0000B3F93C9812E450C1B692E3302BF473076A
:100B1000FC7153758FE5E0E40B96DBC220F030DE0C
:100B2000E9FD33A6C20E0B6473DC8191F3262BD34F
:100B30003BC862246F1B98BE90FF1C0900177B65A1
:100B400005463E9398040B6291C045351146E66B0D
:100B5000D9C8FB2268FCA085BC98BF18A04E2C28E1
:100B60001080BDC582D30241838CA15C1677B7FE8D
:100B7000AA55BFB3FC3E1D74803135ED10E5A59F2D
:100B8000A81120A40588B0BC983D037B6B8C21FA8A
:100B9000508010CCFFF3C62FD6982077BD9812A3B3
:100BA000FF6CCFF84FEA4824667A7B01CDCDC76051
:100BB0007130DE9878FDA203F3F2C5F3B8BC536F31
:100BC000F338F760AB574273F8DD3FD63AE988BC9B
:100BD000BD6B2BA8F3D9022638160767F31CF378F0
:100BE00010B90FC6588AF8EDC483085ED7774B7CDE
:100BF000F7BCC58752F84102103B08DBB3D5ECBD0A
:100C0000A55CFA22492F2840DA36C8A833803E0175
:100C1000134504E4894011F329A0CA29D34F9BACA2
:100C2000FEEBC012165D9C118B607BE884B0768C65
:100C3000A5FF0BA2F3A5F2AB7AFC9B7D40107D2FA4
:100C40005E521879087EA326BCA54FB5FF2C8209F9
:100C5000AF02570744914F8573B00241DAFCE0F9C7
:100C6000981F53CF308807F280779F98C050E907CC
:100C7000B310879690593CF3F8276F09ED3DEEA02D
:100C800007F1F5A55A64D59BE0F3F4B9037AE74080
:100C90000F68F308F0DAF980F998B657C8025D5E7C
:100CA000B85F0508EDE680053FA5D0295E0522C3A3
:100CB0000988DF3108CF8A0322200C5D3736D3C183
:100CC000B99B81883103C9FD2DB37C985D07C43081
:100CD000E0CAC4040CD3ECBAB1EE0A7DE20740B31B
:100CE0000A3B9B8411959342D7BE7B5809B0A41050
:100CF00086181E93602453D3E608F9158D9CFFB324
:100D0000EE54F7C07DB3CA01D868048DB7D370FB29
:100D10007DC2FCBC25A7369AF37BC48445EE76548D
:100D200010E73040882AB128B6D3D0F8C6CF9477E0
:100D3000B3C7764A3DF86C8DBFBD8E3BD6E8F92827
:100D40001E7B66948E7EF49FF8EC2B8A6920638B61
:100D500066FF081B660FDFFB6428EC50583971D61C
:100D600070D8FD20B9E4ABE60414BF169E30CA0566
:100D70000DC9C719B3E0FD6262E644676B0B0285DB
:100D80007AE08D361738FF34E267F9F68E2CD39867
:100D90007BF6CC10ABFC088CFCF3E2333BDF08FBAA
:100DA000533D0C0CFFE4C708968B660904FF19B38A
:100DB000408D40D7F0409685515BFCF9BAB3804C2A
:100DC00022D6C950F8DDC201635EE02C3DF5C310A8
:100DD0009ED4DB68F82DCF104CD3DF02E4E38ECF36
:100DE000E9318D4F52E403F3226BF3286D96459D54
:100DF000F397F6A639EB370112FE2470FEFFA5E744
:100E0000E484BA3A24F2CA0A93C45BB205044CB231
:100E1000B45B1604815FF396E8FE60FB80E1B404E6
:100E20001471D00A1893EEA0050E14E5E60DE6390C
:100E30007B8280057064288A77221A442DA750454A
:100E40003980E11908E97706AF150342DE307E4D9F
:100E500079FC0E9E19EE600402756A4A4008BDCF07
:100E60003126B3311235F230012220B3D853C4BD3C
:100E70002704635E58B808E1CAFE97B0F8D5DF08CA
:100E80007A2E88FFA3F207FE2B8CF7F266D5EA4094
:100E9000C8DB2145F76590909D41EA6FF9169DE901
:100EA000FE97659859EE99DF8E930888FADFF43F34
:100EB00001AF6BE3C386044694226765F1D2AF9C11
:100EC000B05E78670DA0FCEBDB14043EF664D8FE40
:100ED000103FA714ACDE024059CFDE5C5CFE8733C6
:100EE000D222807708BEE229F301F4224004884030
:100EF00084028CF3E51980ABE0029146E0A3F3C6CF
:100F00001134F344F31EFAC5566E083E2B2CA6EF9F
:100F1000EC5758FFF3463CF4C74C91864290FEC80C
:100F2000F375B84DCFEBC1C8E57AC4BB040166B612
:100F30008828FE597D8EFD728E6CE40DC8F89EE601
:100F400061B9B097A9620448A340460DB59E8003DD
:100F5000D0FC6E9B625F3C65667610CAFD6A808934
:100F6000FA4BF8C12F4C62EE309FE7FBC7F8FD1239
:100F7000E34E0D8C6685B3088FF9E69F96F06FF609
:100F8000BF88FE31EB17200B9BA6A8FD732A040532
:100F900010B81AB36591A852369C010EA0580C9750
:100FA00096FFEFFB10DAEE2DFB348A5AD384E66A03
:100FB00070DFCCE531EDAC029C19B0FF89CA10613D
:100FC000272C6808B5B30F1826C1B88FF71538F964
:100FD0006CCBB00240F79088FC206ECAB3804C6D99
:100FE0007FC5E5DE985FEDC0FB8054F544C0B304D7
:100FF000BD78086366B57315B0FC7B30802069E767
:101000007DA1A6105E08B9B1842F20588F8D179C42
:10101000049AC69F869E21D8FD4046F590A0C0A7A1
:10102000CAF130069420D6EA9DA0DD8A096D7A1AAD
:10103000F59BCB17C8919FFDAE6880C0B9DB652FCB
:10104000C93CE650FD80600F589CC0103F6C428840
:10105000020815D62120A00D1810F6B8A880889691
:101060005021DB759094A464BCD20C04AA06B34250
:101070002C2FF44087A0D160F82665D097E6F4FFC6
:101080006FB110AF592E08FECBD0D0FA50D7C31194
:10109000E9CC415682DA40201833B75BF8AF0A201A
:1010A00016E03DBD0E45EADC7CF810D0F780ED5728
:1010B0000AE5F039F3B8422CF4DD2306E0559988AF
:1010C000FD787F576BD25CF3C0F2F368E614FCBC8A
:1010D000C672348580C7A974B167929E62DD64369A
:1010E00061081BE90DBEEC49805F96EF801736B3AF
:1010F00090FD2DB6713C59B710169186BFFCD8688B
:10110000FBE9C08A9F48FBA62439A0FF709C2B40B6
:1011100023EDA77E55E3EE15F398CDE03CC1F3D364
:10112000FE1BEF6C6BF9FBA4D720ECD7040843A29D
:10113000323CBBDFF625012C36EC40FB8053EC142F
:1011400034FD7F409C9B62E6F03E9B5FCC619AFF42
:1011500008C4CC664DB30261A7BD43B8FB8031DF44
:1011600037AF429869BC011D84B0A0EBB4634FB3A4
:101170004F0DD3FE4970D36268748982C6BFC6F929
:101180002F600CD39D44F3D0F894D565FEEB0CC6CC
:10119000967B0124E0F740FCE001A5B9068DFF062F
:1011A000DC3C08ACD2C083EB60CF19D09981FDD371
:1011B00001F0E00378F3100CE041F3079201C6F16F
:1011C0005AF37F7FFC202BBF2E0DDD22086C479A3F
:1011D000391C1826ABC80C22C4FBBBC0293298119D
:1011E000F46C022C22F34AD7034C5B04E788E0CB73
:1011F00098FCF2503002EB9FBF2360088C805BD7D5
:10120000DD26C4E82C601E8C8101303339665138EC
:10121000D346C1BF1801130008C70C1038F340C0F3
:101220001C980013CC7D8CFDB00CB8FFA41926F0DF
:10123000F053C880787F0FE2013DA007D3F08039DA
:101240007A4017E0812CE6D2B34FD388E0401EC429
:10125000CC0312D3E09DD3F3F42032F37940C629B6
:10126000D3C970F873244E44180480BFDC883DF362
:101270000806C028CA83F38CE6E31A63D3DC24840F
:101280008130C07CC14D17601020D3316488FEFAD4
:1012900014042E0FF88F77802026C2210C17DE8CC5
:1012A00082B321306F800ADF9C1840058C8042D3C6
:1012B000ADC2C51293F0122C8011341026C78309D9
:1012C00061830284AD01482AF9E6072901421D32F3
:1012D000060221F4BCC5EF5FC663ABFC34DD71CE02
:1012E000A28AEFAA6751451835AD89CBF042F8C7FD
:1012F0008BD2CB8B497BF3219EA08606E0F9FEBF03
:10130000E4253873AF6D1740B884F7BC0C2081BB5F
:101310000EDCDC2790485B06334F5DE38141C13929
:1013200045FBA5AFF5D9EEA5C803114AC8B9F2C56A
:10133000F6E0C003C87BB31E02B8EA91B30F32CC0B
:1013400075B3530CCA188428FDBC80C670C0200633
:10135000DC8EBBC2F138F95766BA40E5882613081F
:1013600060B72225E201241888F47B0447B3D60134
:1013700003BB1EF9CB0B80B09905F98AFDAC22A501
:1013800047D3100EC6F8044AFC90E019F50211FC90
:101390007F12101FC2845820E3636004830199B157
:1013A000E5C2A4FA082060122C39BF291C8F605AAC
:1013B00073B31F301E2D63B310D016227F1360113C
:1013C0004CD28005F340398BCA0B62B66B070231F1
:1013D000D3982CEAF02B33BBDE200BFCB8F4F37A65
:1013E000316D083AB177EF161A3CF8C4030B0D9F24
:1013F000FAD3077120160F03723AE0E2411BF38320
:101400000EBBA40B3EAC3C20F8FB68731066BD9885
:101410000386608B66CFC5F5B860959B901A52F82D
:1014200057B310A5B8806634E00C82C6920666EF0A
:10143000E2C6F9ECEA97FF04A0C0586E0B61F058C1
:1014400026E0C4E6B301203B7E6D23801C39D740E3
:10145000420AD3123C86C08BC6EBECEBCA94520C0A
:10146000E60B08FEE2903180C020E8428A48290756
:101470002410049281B1D0EE655D8D02D0DFD4835B
:101480008CDCB9FCF8D4F310665623CD86CA14D28E
:10149000E018D359209180C4FCC0180209630842A7
:1014A000C67BD30160F9753403FE9D6BE68B4FB8A4
:1014B000B43E8C88B7053B1C54C086FC780B7E1468
:1014C0004082506CD035C6D0C230C1BD9818C5C45A
:1014D000832B2EB69E0885B8C650BE98F73281AAD7
:1014E000B83EB3195051E488BDB204AFF061F503C2
:1014F00078C30EA441C6F1D7C5C4756402E0DF2AE3
:1015000040FE2C505C738A12EE23B799BABA684B2E
:1015100003B05221AD419FBB92028A36094FF84970
:1015200011C982E6019084F7D1BD788B81688DA5C1
:1015300010DB206FFA40905E8F8CA07EC62AFE04DE
:10154000103062C2C2F85800A360384C80F110FD20
:1015500046C20498030CCB2C029B9E412650C874B3
:10156000E65E933A64DF84AAD7EAC1E40540735289
:10157000D383C68B108D01215CEA9D09D390FF7344
:101580006A80055C5DAFC875980F6201E8C5F0051B
:10159000F372300FBCABFE7B89229D140ABFDE8143
:1015A000FF4202E5413CA003E0E2001E80901925C5
:1015B000640C05C6F51ED00358C92341D3DD68FD70
:1015C000E7A57898BB7B883D73D3D0986216DE740C
:1015D000665EFDBF14C5DDB17DAC1CD3E05C035D70
:1015E0008F72F32082D30657C6B08BE9FDAD497CDC
:1015F00098FDE8F01131CABB5510292D693068BB40
:1016000068FF9F079608890531D721169378E01463
:101610002077391046C4040C2886C695B990C4308A
:101620007EAC02CEC803C98C21BB41C61A22B93098
:1016300060DA0C2DE7C8B8BAEE32C022CFA55D192A
:1016400068F220043086D27DB343600811659BE1C7
:10165000C6D72B9521279B9414FA6A88BB184C0F88
:10166000BC89028447DA3DEA11082C2422F89665E9
:10167000441AC299A69DE7D3B7D7A0F8F5D6FC3097
:101680005ADC4FE68007C1403A098378E81A0FEF29
:10169000175A3061B943BD2BE610B0A9813CEE75F5
:1016A000301EC483EB1B40C5C67917609736AB511B
:1016B000D06BE3F3AE10DA409D23F24102718BEF61
:1016C000601008128C1604F719A01316B42DE72821
:1016D000CB9A81AD04A449CE418C08E27E38C6B6CF
:1016E000EF4D2028D34B7F7FB008F526C04858D552
:1016F00044FA6045F038FA429863AE044C5F089FA4
:10170000C814742841773C2812329468F89C01026E
:1017100026C1A66FA36BFD8C3DBB0906C17F32437A
:1017200060F3104C8209C699AEFA193D26F26EBBE1
:10173000D05702E826F3B439D0EF4B98602C985A72
:101740008A12F70131AB4789F008E8353CA0E4780C
:10175000E0D63810529BD3F0950C039E8EC0813C8E
:101760001D2865C8FEE569F71FA5F341931E59447E
:10177000DF8002DE57815201FE4275C87EAE022034
:10178000E4034006C7C6F323804139F391F8EC5CCB
:101790003D59C870C0AF26737816C008B393E06097
:1017A000420CCA88F339BB169069FC140A82FDED1D
:1017B00011400208987484BBC82FD5F05E3361FDD8
:1017C000842719BCFF208544065D17F1825013025F
:1017D000FA018031D6E4C082ECD3C8112424064F2C
:1017E000B3B4E732D4BB817E9133196A3072E19091
:1017F00014D3BD6B680E29BFA88A0969AAF9C8CE9F
:1018000022013EC8FBD7C8DC39C9F5981092F9858A
:10181000822ABB3DFFCB4541841A1264FA980C59C9
:10182000CF28FF80E7FC38FF32063CDE4A5370F0D9
:101830009857E02BD4F03BC88360F9302048CFA6FE
:101840001D225311DCCAE641402BCC085CE38CB46A
:10185000035AE008E83ED3A662C608FC1A448B533C
:1018600023305D039AAA50FEC3182256466BB284F9
:10187000D0BD8193662072DD0D93CE2459A882BC21
:101880009869DF11378BF260018C02E585BFA8D91A
:10189000C8C640A03AE73AFD5660028802E0E7E099
:1018A0002C02E410B008965A993FF24EDC4357A23E
:1018B000DC2625F8FF11419212081031013F3C1837
:1018C00058042360F5020C90459DC8C12231F36293
:1018D000112B84D951E8FABD5EC5AFB2D71C801771
:1018E0003017239D8BE8985A720F86B20EB5AF0A57
:1018F0001F85017231650E42E07AED8803E1CAA8C6
:10190000F16BD37F1F03908EE80BE61F58FF845BBB
:10191000D0BF06AB2DDDD2888130C5A9E6988B6695
:10192000A04EF73B854004FE9B42136E3B30EEAC6D
:10193000C98ED346E8998E813159AFFB008578ED89
:10194000881020D2610AEC85C8C2A304D3BC8B12D4
:101950003FC692F815FD86B5FE0A60FC322E0530B2
:1019600008AE133F102BC8D7E70965C8CDC6A0FF46
:10197000726A8AB5E902A745CA812250E7040AC6FD
:10198000DF82447F0B5D909867A8FA57B53DAD564E
:101990005D8C7A16ED83DA39D3620893F13040B06A
:1019A000A07E1128520863351464C8DAC6C079983D
:1019B00019C73C302C80A7FF260410B955F819EF41
:1019C00008A28A22EF0D315617FF28FB405ED2266F
:1019D00019C0D0BFD60C5B760707215D914512F286
:1019E000F6F393CB7EE7BBA7C1D53DE826947CF008
:1019F000B49C32E0C002D6E00F57BBCD9FD6C47E68
:101A0000EC0281D3EEC0FFF204EB91FC1101FBC3A9
:101A1000018911FE7A4552C41B7A9BAAE41D9C776A
:101A20001F0EAA606684DC169CF445210A288113E7
:101A3000482620DC0122D7B9122508FAC2FA80050F
:101A400010D937B95EC5084A84FFEE40C024D74894
:101A500008255D2C79FA62F2AAE06098927DF8156B
:101A600058124C6BC90A1031E008EB8BF5EB82E79A
:101A70005E03C6779D6B9DC8E0FA680FF2B0B000B8
:101A80000E16BDD26077ABC5F48EC7E55DE465F593
:101A90003D66AE1E0718DF2AF7550D010CF203E272
:101AA00089E0980F779E5EC677836B4DD338FD1023
:101AB0008066975C2C7AD240BDC5C146F39C236BEF
:101AC00095C8E7A89AFFF11007E0765FE8982E40E6
:101AD000E7F30321699DC8B9FFA7381D8818214F76
:101AE000CBC84E031010B4603FC6BA3780092FAE82
:101AF0004238C0263CCC26EF7A4B23600A4CF85281
:101B0000D54690BB6D135ED328F9903102EF2E04B9
:101B100098209113701DF5CBE198E54183FF7FA7D5
:101B200010BBCE7633BBC9BEDE679B996447DFA688
:101B3000885140482C683C4180BBC630C882E06375
:101B4000F4218CA1F3BF384B15EBBCC2A25A1097FD
:101B500032DB72798E3DF71E48C00DDF7F3B69C8CE
:101B600026BC9FDCE396F820F9C84FE720F8FCE09C
:101B7000CF41085DC0401C0D65F875E466C830BCF7
:101B800098FEB4547BD9D048A45B9EF86A0CF82523
:101B9000BABE6B53C28410E30E03E001F74104C8E0
:101BA000033A7A0E8070F378FA2CDE96DD4248E72D
:101BB0009BF4D122CDE0784D5E7C1262D385E7F8AC
:101BC0000311CBA26256FA351E8BB30425221218DC
:101BD000DBB84A212CE48E8251E508FB9E103009C7
:101BE00026BDD205C2A020E50C824969FE985EDBC5
:101BF000F70C8145307FD46C908E25E7B335C098C3
:101C00008132909E10FFC402984D4CB388FC039023
:101C1000C0A76E20CF8E093002DF90F8CB3DB0B95F
:101C20006A180E0FBDB8887F9F98C250F3E7BBAE0D
:101C30005A8A7B66570DAECD3B30823DE11E8460F3
:101C400078103DC6F1AF207F987A100FE8813C08EC
:101C5000EE38FD84F5E540DA02B502F1B8395EC52B
:101C60009662C247AFE5050119C05935A511F0408C
:101C7000D9A80E08D0D3BCF6DB39C868FFD6BF316F
:101C8000DE98010B5082DBD56B18FEF5208090D1D9
:101C9000B30A2FBE04B3623502CE08262601B9105E
:101CA000534D269029A0863A8BE5038167C8D0FE64
:101CB0008820EC95C8D9F044F08C21F4B0A0B7AFDF
:101CC00042DD9F0CB7F07BD39865DCBAE5B3FAC868
:101CD00036DD7220CAC869E01843BD411784B0F3ED
:101CE00020C6C018516325D3C605B9B7F9CCC803BF
:101CF00047F1C8EBF304F8C8D1FF58E888010DA7F5
:101D0000BB81A2B1862E5B3718B5F6B0FC95C494A2
:101D1000C8C13F70100F82013859BE72E070DFDE1B
:101D2000714E23A083FD72F711504B54FFAFD6259F
:101D30006BE04433C607E0D3C84DF30F4029F3806E
:101D40006606A5896E02C97081C18C05BC48B72999
:101D50000CAC10BF4EDF984C10460D1177BC8B2891
:101D600081868837FBA58244F450080A20CF39C603
:101D7000112486FFA0081081A2290409D7CBF97E7F
:101D80003A02264840588322CA80FF47F3425E98B1
:101D900024CAB1BB48B8B94AA0F5A1E3374750926D
:101DA000D0BDED0616C1BF2B23E5600C285CFDCD30
:101DB000D09804AAC5C71107A9F8D6E08157C8A2D0
:101DC00098C4CE19536801E3F3F930405956943C56
:101DD0003914F40F0A0190F3E1800785C1E8CF3D83
:101DE0008826401E909E832603E2419DD3F4801EE8
:101DF0007B98400FCDC841D3D0A72E7D40FBD9BCE6
:101E00009806302047F37F9D9895C8E49EE90B81A2
:101E1000D0455E9235E7EF35D2CAC8F27842D3C2D8
:101E2000CA1810F3D2C2F698E1FF77ECB010799897
:101E30007FC8440CE6841131F8C2EF799860148CA5
:101E400002B35FCA44FD622FF4CABDC94ED93AE05D
:101E50009802C8C81790FB4B08585E3E99817909D3
:101E6000A69640B336FF4FB6C40330C073B3C60165
:101E7000EC1860046DD310BBF9E5C2F9FFB52C3640
:101E8000E3F3C6B07E1457EDBDF6C8A20A288DB69E
:101E9000D398FB3866731D0AAABC2AAB3E5596C779
:101EA0001BD680F81B3D934347DD419CEF088CA275
:101EB000804E638B3928081E669490242CE7B30C5F
:101EC0004811765C800F459E968362FF88BAB5C242
:101ED00007B3C40B0AB98CF8C2F61504C62036D66F
:101EE000F6D8FD040134447FEF2F8040B302CB408D
:101EF00046FA1A6CD3D8FA68E2CFF3F6CDE03C8DFF
:101F0000CD21D38BF4B1F85F22A2DAD9F1D8A05059
:101F1000F58D78BFBB2502622BD20A7FC032FA61F1
:101F200029FF7116E67032DDB1C8EFDB7F20792220
:101F3000C6FC6F997FCDD430FC99963A7F57DEEB83
:101F400089082EB8CAA335F8319F5687A0F9CB006F
:101F5000C5CA3334C5A2B38D801AD150FEC5B99617
:101F6000FF3CB880BBBE5CCC5B21089134AFE6EE91
:101F7000FF2F7AD308994F18FC39BC04B9C53E8F9E
:101F8000CF476504BC02F86CB008F61270FEF37916
:101F900094B081F84B240864880496B0CF7FEF7129
:101FA000114B9904F65590017CB144D9735FE8F95F
:101FB00076938FE3D442DF0A02E485DA599220F661
:101FC00025F3059C83FA60400D10A1459490256887
:101FD0002431D0148400AE503DA7A390726622072E
:101FE000842072D712486B53035354868E811A484B
:101FF00021ADE3545021339E04276056BC1E038854
:102000000602C0BC0581BE16FEBDF09B31B958CF9B
:10201000193C5A10E3211BFBC9C8E9298CBBFFD727
:10202000995C9A9817E6DF69F1CF511D0BA38B3F9E
:10203000CF5AEDAF10C6E0DEFEBC0879F58224363B
:1020400086C1FDA7DA198E4B73043C87F33F3D4CE4
:102050000164B7F2E0FEF50CAADF028F93E3E543DB
:102060006B125EB00896641A119E3EC6AFB8B3CC30
:10207000BADCCAE3E575A80297D61C29DD84F8FD11
:102080009C3862E6FF3AD74F9238FD4080DB08105B
:102090006FF802449084F32E425C4111560188751A
:1020A0002D11E068E713A5C62213C5D3E309F3C0D9
:1020B000B2FFD64740E28A09C265611091C67DFB36
:1020C000E3B282CCD9673645844FD975ABB3FE5F96
:1020D000D282300B08C6CC79F3983F7B8718F8334F
:1020E0008C32681FC7DB9AE8FE1631E5CDB3F8CF16
:1020F0007DCD78FF97D68B1E2CFF98734DAFFD1CBE
:10210000046856D9C0403E2AB301B5A6E8B0F8BD70
:102110008002672D9080D666FD21D5B197599873BE
:10212000F7AC0330E5E7B197967B1F7ECCFFD40B6D
:10213000DB813CB0E9B3FD637EC6614AB601BCE514
:10214000C5171940FD968F75669C8ED6B0FF59BE97
:102150003A36BF026DD43E5D23153699F3D275D35E
:1021600004FF4D5A7D686667A8C602E1C50C4C6540
:10217000ED40B1F9D3CFC2AB33C592F188B493C867
:10218000FBC57AD61296FB1011F67840FD31621F1E
:10219000E8BF58FCE78CDA48CB58155AFFD9A8FF9E
:1021A000FC8DB00A85C940671E0ABBDBB0FBFC4949
:1021B000B6F024FD66805639B2F319CA5BE808719F
:1021C0007DA69CE40A6CD509C90009F99784DB9BBC
:1021D0000CACCD40CCEDC782207CDCD4C917A1F972
:1021E000404BD1B4D3CF12F0424EF3A2048031144D
:1021F000811B01B428D57A1AB37302204C8B1028A6
:10220000C08A02A6909D2A28D7F47950F37BB39810
:10221000FC7379A2208F10159902DE44EEF848086D
:10222000B4C0183902E9FDEF0103216F7E0806EB07
:102230004BC7407580012594FBCCF50C0190F2E072
:10224000CEB64002ED05C168F70A98FF2091AB5366
:10225000AFDE4044BF802D107D401046C57FDB932C
:102260002CE1029F8B6CFF6BFBB002D7AE8024FD8C
:1022700041D3B982D8412DE04DB2FF984046F1BF1D
:102280009FA2047035EEEBAEBFA468D9F9303F6968
:102290002FACCDE910C6992BABA8042071F2D31D49
:1022A00097190880EDB06CFEE6DE13EA6AA6C692C6
:1022B000E3A019C2F5FF10E61923ED4B18FC871AAD
:1022C0001667F39058FB68290D8646B47F18CAB28A
:1022D0001901584B55A7EFB76E18FF6FDA06407912
:1022E00067FBCD657BB41008627FCF7926E695BB8E
:1022F000596BDE5730F808E3ED30048CE4FF94A30B
:10230000BB90679B739EC3BFB690FB7F7E37D6E8BA
:10231000F10D9777048B7AAD1BCB28FF7FFE6CF60F
:1023200062262E176FE238FC61666ECB04310A66B6
:10233000CE89FCD47AC2AFDE4A02F66693EB99F8F6
:10234000F9FF2048348014C10402E1402008BB7F1B
:10235000C00A1012840223F4F10121B06C04447B02
:10236000BF0F821CE7F94802D38004AF82FC0F0242
:10237000410A09814F900530017782E51B06C0763E
:10238000CD99E20CBF51F6CD75428CFFFD20104275
:10239000CE8C021BF7F3604E60DAB8F83B961CF067
:1023A000A443E3E48801C0FB55F9E70CB362BFE145
:1023B000B9808E1044E079378618FB93E041813C68
:1023C000785B96853142A1C2B8ADAD44C97D80F03D
:1023D000598248B55B881F0511627CC7AD4099479B
:1023E000990161862941698A42262122344003608D
:1023F00041F3A0FD8031131677E47F83927C901126
:10240000FF5746C10410020B609E12A909200AC59D
:102410003B26904066A58CFB2BD3C0BBCA11629FA4
:10242000060209A8F8603C308803323C1ED03250C6
:102430000660407FF307F08006C003F179000F6863
:102440006C1D491C07E670400EB0387FE0E2813C0D
:10245000A007F1A420C6783E0BE4017719F8FE8AA4
:1024600006DC57B640DD34B59DF4CCA9A310C813E3
:10247000FFCD0684402526667E528094F3C1CEA708
:10248000836F8201310FE0FBC38041EB124604F8F9
:10249000801364A8E7461ECFC822F3032001CD2C89
:1024A00004032291E57CA608AAB340018D60F802DE
:1024B0008C901130D31086981B1360D3424C6C055E
:1024C00088C4FA203F0A14D10042405AE29F415B7F
:1024D0003480401402822460D9F3213AE2A130FC16
:1024E000A7EF2A2038D5C682DA24CF0149EB24127F
:1024F000209ED07549084CBC8B1FA4007091FAAD8A
:10250000D790986D25F760110C19A659D03EA97F78
:10251000BD7FE73302069DA610AA904078C5102023
:1025200090F8691304A5C0348164A8E9EA3008E191
:102530001847391AF3B71E80093EB307F7E204863D
:102540006F9310F12EB41D786E02C3F5E060E0D8F1
:10255000FAF8FB88F2ADF0982B65F7AB78D2536DA3
:10256000884CD5021123A9B06A7ABB14DFDD0B7742
:102570003E7A05E51001029CFDDC028092639239EF
:1025800060D3094E401A042873AF73FC8930FF06EC
:1025900026C204180213604C6C503005E98B58AF0A
:1025A000E8601180F38FBB398CF88CFE472F58857B
:1025B000053009BEFFBE3981735349EAC01831F1B5
:1025C00022E7415D5020F11081F9E07C3C8003F06E
:1025D0005F16C08378AF402FA51CC50916C4087AC2
:1025E0006E32F3B75442EE040608E8CBFC70401696
:1025F000CF3A7809E8011C8B90F1030EC00238BC79
:10260000B543F3E128F9846E3020F6980803FDAF56
:102610002D068BD3E5CC067D2399C25F6D85D36EE5
:10262000E0E01A7664C0EF155E6BF1C203C241FFB1
:102630005EFDF046048298C0FF01084C80113022F4
:10264000463CE71809513C0A0C96C4F34EEEDB02F7
:10265000FE9505B2BF4504821943B3FF4C8451B0C7
:102660001046C140FF58080162024481099CB24DE6
:10267000FD307D24C22785020C08404C9534892901
:10268000986029FFA4A05C306AB3BB0ADC53231D09
:10269000305D0402DE98FF4250082A2140A00977ED
:1026A0001776B26B0A09D261D624EB68FCCD6E5660
:1026B0008601BE615C2396088656EE48057BF55F71
:1026C00023BF322F45EA0BE4957678D3EC1908F94D
:1026D00083B3C9FC74817F4B54E57CB47CCFB24B8F
:1026E000276EDB3002B8F06220032EED0AC0B87905
:1026F000FFEB30F80C043141A029F65704D38024B5
:10270000A60A10CEC014CCA008258C028B6A667372
:10271000F8436FEEBE72843B0895F301E5B8EAE535
:1027200085F97FBBEE11601209668884FA1DB1211C
:1027300071486E01834F6A90832680181F0120FB29
:10274000620C2C82452F9ED242E71F708FCC4176BF
:1027500003BB61F2C332FDBD9820E7116221A204E0
:1027600022F710E0FB607AA5325D26C0302664F3C4
:102770008804F10D1EC47AB80F6DE61CFCECE7BDB1
:10278000070D40B9E4067077A6A57819E21D0CDEA6
:10279000982E6322C6D3E9B0235ED27F133DCC8846
:1027A00081F4301004C4F32B8659FC4130BB657DA5
:1027B000B0DA8B19FFCD2BF3AD44FD7B83F56020A0
:1027C0000484EE9838FE8006302006C488791813F9
:1027D0002441A7CC05B0D8C02F40200960FD118C42
:1027E0001008300193EA4B065C938119FF40424880
:1027F000084160228CF80289B02040634080AF031A
:10280000048B4FF39AFC2049812440EB5002923F05
:10281000D54181A80410309E12DDB0DAB02D20DB46
:102820007998FBDBF81A232F38280BF17D1017A1BC
:10283000984A642128E5E7899002D30A49F4008187
:1028400022904D7EC0499444B5384C264010AED3FA
:10285000B7FE3D246980D31424F8C377B27374A003
:102860005A1971806D49D9C47BEC50FC7E6B23F002
:10287000EE6977E0E401389CDD322B60CD43171C14
:10288000133ED52D77B3898557E35D64FBCB42CEEC
:10289000DC220B8AE8578E75ACFD8021F3FB309863
:1028A000AC44C1A84CDC90045172921119A919B121
:1028B00066CBABD1D76612E9F2397E0A8010185C7C
:1028C0002059BBC509218348904E44FC804591198D
:1028D000A27F18022360120CCF5001DF4680245AD9
:1028E000DC770BDEA06FB94F885CFA672338904124
:1028F00024A0FD01E2720C2C9E642226C01F180841
:102900001187622CAC10F04829FEE0F91C9003A955
:10291000AE1E0630B56C24AE802F30438B1AED0FFF
:10292000E001BC980D14CF30070F88E926ED19702F
:102930002E0EC8B83DBD783DF580037240E598B9CC
:10294000F660A0326FF897B709A077165D686848FF
:10295000660238EABFEF5198886DEB16046E3B3083
:10296000E16036F5983065C8DE5E7F0E23B221FD4A
:1029700064D810528C0DBB0411BB44E3A56008144D
:10298000E404405C10179F98EE97221082D7BDF7A1
:102990008105127E9D020610110F208C04C38880D1
:1029A000C416608798833A694C84DF31D8F930FEC9
:1029B0001005821411021AFECE41307E81068B88EA
:1029C000BE86212DA0405AF2AEB3A07D51033BA894
:1029D000309078984F0892500AD7480296268E2059
:1029E0007F0249E7C6800524941119D95B4915A6D1
:1029F000CB568A8FF3EBC8FD98086819A111AB4438
:102A0000EF12BBA81912BA088D5EA50A40C9F58B52
:102A10000437DB28FEE6B6B0E20657B662EFCC0616
:102A2000F19CD45C9C6BC07D2E12FC774D2D7FB940
:102A3000C486B27A8A038DE03EBFED4FC2E09110AA
:102A400078FDCC0C049A4272DDB30F04FA24A090F6
:102A500014102DB3E54B0A0866215F093D58524F0B
:102A6000FB1F02BFB0349410E28F0811C509227613
:102A7000F169044092FD03B930019F50E6FAF90470
:102A8000113AE216A44CC08B8B802466FD16C2025C
:102A90001805A3DDD1BC515AD0B1BB174ADE2FA017
:102AA00019D7C0848978AE80AE44FDB8C0881808B4
:102AB000236DD6DC30AE586B300D80CD9839302880
:102AC00077A298F0AE7A5018100FE8EB545EBD6014
:102AD000F807830AE0197A85F0371EC8039839236E
:102AE000E41E3C800131EE62301910AF1A6BE7FC36
:102AF000D19EF0B5A0E3305F2F98BF30C598F89A0B
:102B0000FFA28074D48F18DFC34299C808F3699B71
:102B1000BB08B3C821AEFFF4AB114644BF5E02B49C
:102B200004F198FEC80941B13E88053011133723DE
:102B30007B5711F094025C300B60FE8C828930016F
:102B4000174104091F5060032084F921B00030FCB4
:102B500068A634BD021A5DBEE520E598AD4C824002
:102B60006A9F0D51C4A3A2B340E7AB623B288E20FD
:102B700057C4BC981341222C6F01A0812429CF3B5C
:102B800040130A14982164A6162CB9C86BC7307973
:102B9000989275B501E52C15CFFB5237996A79F2F9
:102BA0003726040392F6D3C4DB8E79D562FBFF5639
:102BB00097B0E0F23068BECCD1BF70B810DDD866F7
:102BC000ED7BDC2BB319E88DF4B4FCB956305C0313
:102BD0006BA7CF6A53B0B27BFF482B18EF65DCDEE2
:102BE0009800909ED42268C88C4EDB4205456680D2
:102BF000DE8CEE739D7A1FE566225804A3D76084AD
:102C0000B152208933C124E408D740820F30F1F358
:102C1000F88030D042173ECA0193601240B8309F0E
:102C20003A2448080361FD048C8405300A93AFAF51
:102C300011271D387FFFF0C08258100B6223AB05AF
:102C400011FC0120C0044108AC5AFB4E502010A9D1
:102C5000FD9801AC94DAD503F03057E9057B98E094
:102C600041B63C3F19BABF220D5BC91DE5C8DEA5C0
:102C7000D688074B9BF3F9301C37E6FEE93AB725B7
:102C8000304466AFDAD7F050B678F388FCE563E4F9
:102C900020B4FACCFED9820102E6304018BC5E575F
:102CA000F38C980DFC99473FA686BB1C97304C309F
:102CB000D81604BE8802406008772F0431681D27AB
:102CC00003A27F0BF71E80F4E614083E609D5305B7
:102CD000B1086833E1A01162614C84CEB1C4FC300C
:102CE00070D782067A029250D4B12D68049281A4E2
:102CF00057D107239A2DFC843FBBAE60751943FD65
:102D000073E400EF899012E34002287F20248404BA
:102D1000928090030349F2084C2421AB77FCA8FB76
:102D2000F9D2FC30717A65C8E63099C8DE0190B3FB
:102D30005B874F19475F73427EB548C020DAB10206
:102D4000396DCFC079C8FC302ECAFBCCFC984EC67A
:102D5000700460D38230A42C10B8F3E6F3B3FF2BD9
:102D600028E65533455D30FF0698B3D50E5DCF0D8F
:102D70007D55AF931FEA28FD9A0C9D41CF2E9804F4
:102D8000119A24A2A2F1989FF4885A2003A49222B7
:102D9000E1FDD066FED2F155660833DF66018B6037
:102DA000020D908187391441887D333C24DD083A37
:102DB000C778F9CB8AFC982483977664A66684A6A4
:102DC0000BBBE881D749209B1FF32C4695C073703D
:102DD000ED0532017D9842F38C02043091C19918BF
:102DE000A622F63FD384201050FC5EFC7F9698BF4D
:102DF00002100F24012C80BF059A5D1A10CCC80C5C
:102E0000368766BAB3031D4FF6CF3C08D7C098AFDC
:102E100079980D9007F0E059BB8020EE0930FCDF77
:102E20008441C530E4D2A97A66C412EA37E230FBA5
:102E30006996B304C7B3B5FA3020D66C4657C86854
:102E40001718F36BDB84D99840FFCAEE8020A0F7F7
:102E500098036124DD4888B2D6E360C25363040856
:102E60008AFEB739DB46FDDFB25E30FF080C910900
:102E700062102C90898112F916E0400809C6C680BC
:102E80004CFA85B000C8FCD4020A1F90029244FF9D
:102E9000120C82812805348AFA2452008240D6A17D
:102EA00021105FB2E2DE75D5B23B5C318406FF577C
:102EB000980A0F52F2348426F2D2829240A379E427
:102EC0008105246CBFFFC2C53FC59846E43E6259E8
:102ED000AA28B5C1D0B30509FE84EF15FF74F57DAE
:102EE000C0FFF944F6192DF3F803B3C8FAAEE0AF0A
:102EF000273498CA7BD98001B4F2DDE00C039A68CC
:102F000066B912EF07EDC53F79F830978E0EAE9691
:102F10008135C6CFC848F9A017800873662112FF13
:102F200044108CB090300402AFD04232200288BAF4
:102F30000CD86686AB04C5746688200D7F1730BC3C
:102F4000980888802085F3915A18928400C20F7ADD
:102F5000FB80A205D6FF32021160FF120C5001B0B7
:102F600008C4C04ABA8AD0C3E422BCAC66538B0FF3
:102F7000818DF23F200884EED7D998800CCE31E9BC
:102F8000C0E348F1042262758001CF30B8FCE04113
:102F9000842C57198A98A7F7E2013C800EF0BCE216
:102FA0000143F20FE8413C24D3773A90FEDC4B0515
:102FB000E87D0AA79F98EDB51DA07998CBF320F383
:102FC000C848356641D79175FE7CCCCEF101F3043B
:102FD000C0BDA1832E73F99F4969DB89D0B649E052
:102FE000B06DB83065F20CE0DC3047D90996655811
:102FF000CD19FD33B0C8D1987E4160114457CE6BD6
:10300000DEC4E0A218FE4C5C04311257F035A5CFA7
:10301000B3067F6F8404B581E0302419C0E611FF48
:1030200014C0221805016241E7848811B9A8FD2C5B
:10303000A268FFCA7BB3EE6F70041B6BD360FBCF3B
:10304000F45D4840E6A371F3AAB011E78EC667BFEE
:10305000D87828D8D318FB0C78FFBA64FDFBD4C409
:10306000672F741C76D668FA2C111C66F8F64C672C
:10307000AFF83839C4E8FF63C666CFDFC6E76EF045
:103080006389D6801947A0F91819A0BCDA6C666B61
:10309000BE412E0E40CA0073E373CDF39BC6D8F930
:1030A000F898D4B1032844F3B1279630026A78081F
:1030B000CA3C96C605F98DFDF99C37638DD398FF00
:1030C000A9DABE841E640AC5DA3C39F7CB4AE52486
:1030D000C536340E35F43D08ADB45B77F991C5E1E2
:1030E0008FACFF2060E59B8F78FF3BE8FAE9D4F1D5
:1030F000CDEDE4029BFB1E0173D27F5998FBC6D530
:10310000E4A8B46DFA1A8031C1E23F68D7ACFCD8AC
:10311000DCCB0584C6F65A2F28DBE4B0A466497BD5
:10312000DFDB67B64168F8249ABC10A1CA2E3ABC0E
:10313000AEF3F38DFC6DCC3D1D82B0BDFDEE4109BB
:10314000692819F17F32B2048DD4BE0BB498D01621
:1031500056F7DA51929083829BF7C0FA737B75F72A
:10316000201111E018CC8F6F95111B6BE7216D2298
:1031700045A214A37579CAA0F8F57BFE2214048831
:1031800081C0A18ED037E9507FD4248067BDB34081
:10319000801D35134EDB2A2080038BC64BDF334D59
:1031A00012A64C23CF6B58FEE3F27F0C0102C00441
:1031B0006A400A080F056080064197A2C566C447A9
:1031C000C43B3571C481050DDA16F5A01904819F41
:1031D00002908028500FA2C0FF14A001246008D8DC
:1031E000F9465CA646DEC4A141FCD746FB23FBCCD6
:1031F0004077F60801806BF48765442BB9C518FB4E
:103200007906E7C0F594BFD1C2F39EFF29498B44EC
:1032100044FB9628C3FDBFC4025A9A49D040C6D089
:103220003CFDF7564F400166FAC340C5FAA6CA5E98
:10323000E50871DBD0FE11E59AA65816E9B7B95B2F
:10324000C07DD945D794C8B76A279650F6C6E85AC4
:103250001E10C60DAFCF5976BBB8F940C66769BD21
:103260007DEDA009079196F69C9AB301BB31B0B2EF
:10327000FC8E2C3306CC6C756802B5281DF6A4A80C
:10328000F98F99CAE79FAEC482334A796040B6FE8F
:1032900036673648D3FECCF4556E2079B794FBB927
:1032A00001B230BCF8A8C70C73FFD8FB02A6F6C960
:1032B000B8FB4A8E10C21DDA5D02E9219C47A68048
:1032C00029B0F9C438E88FD3584604EF99EFED8D53
:1032D00070FE9FF68299A00D847F7579A5BFB6DC3C
:1032E00028FE38CA79A7E6218ACD425EFA40BE6C34
:1032F0009164B6F6D0FF3C80613F7D9E082041F886
:1033000091F6A5142CB21051CB88D8F88255EB0B4E
:10331000201BFEBD18FCCCFB621F2259D3F0E7D660
:1033200008CB8880294AFA6FFB740414FB841F5B66
:103330005710EB3950F962C6433CB823BF339B8228
:1033400058FD532AD07701DBE5F7E15598D7C6DE63
:103350006C16DA0880B6CEE0FD4A1E08CD3193FF28
:103360005A4608F6A030D1F198B9FEA0046B9665D4
:1033700023F631EB7F0810FD610392DABF4085CA66
:10338000699AC6B1027F595C40AB9A4223FA1D1874
:10339000106570D8FFF69FE7F1690CAFD8B7C20986
:1033A00040D4EF6DBA1481315CFAE97E5B7BAE8666
:1033B000015BB30802A36AFC2CDDC55A08C0CEDB52
:1033C0001F5AFD7D58FEEA7C415BC0012D63010D53
:1033D00062914D10CBF3C57AC37BF120107E5C6007
:1033E000426CD4B640DF3458FC026E0746E0A73585
:1033F00084A6B58206F38FB1E02008AB2048AF8FDA
:10340000A8EAF7F3507F265BF3ACFCFDCC0322FA6D
:10341000880A0A39D06D035E344D940168E360F682
:1034200006BF40FE050C032018048523F412EE802D
:103430000690FC81093E05800138A57AECD8A805E4
:103440001DE8FC0D1380812B8490FFF90281620737
:1034500049A601E1225242F369FEBC1804C0D5B36B
:1034600060F718802510226BC04FE7113C8178056A
:103470003C0F341007E5FEC8184101200470B83035
:1034800096B301DD3D6566A3205EF60DEF02208058
:10349000742A01084086682C2539147DE8EBC90898
:1034A000B465F5F5F9A1E3C2E89351F1A6AFDE2EBC
:1034B0006978BBBCEAB3742E4010B278E0A3359BA8
:1034C000B20D4997AB627FCE9FC6A0FB230B3B207A
:1034D0005068A1626DE344FE85FBF45F6565A9E079
:1034E000114B407AF5D8CD59B30166F539AB1405C7
:1034F000CCF496EE08FB0AFBF923ACB325D01DAC47
:1035000044186FBF78FB7F1031E5FCDB80407CFB0B
:1035100022EBDB9BD490FB65DD20B1EDF902B40416
:10352000EB8F1D35A4EAF73FBE7BB588F80C364E0D
:10353000F59120A955BEC2675E8FD8FF02CFDF424A
:10354000D6D7BDAB68556666F181F111FC6A07DA22
:1035500030FD19509FC75DED638B65487E37EE15D2
:103560007B53CB30083F377F048BF6DE09FE72D4E5
:10357000C9BA17D3CCAD2B51FF016988BBB040CC81
:10358000FF30A2C7D6B818A6D75E565D5CDBA8C0D0
:1035900050FCFF1085A040148202410209258DDDF8
:1035A0004A10E2031A41EE680859D342AFB4A011A1
:1035B0003482BB46D2C560D7B62278F310D002EB76
:1035C0009FBD22812050841446DEE57ECBBEDA55B5
:1035D0000E048B7ECE40D7E563BEA65180F7A2E7EE
:1035E00084EE7F19F8400128A005B2F90018C00246
:1035F00061BC2FF3E98DDCAE03769360013C21F4CE
:103600008C697E68CD60BB9AF305E013D220648894
:10361000FF812810E8FA20800400F1EA4890603F1A
:10362000408220228430180B02B7D06243C6A31117
:10363000673AB2848008E9E21EC212444FB582881C
:103640004014FE241801080C20414EBA08A0F910BD
:103650009E300006C029DB830322CE20826641060D
:10366000893386825B63B1301EF9BF0A10C008C07F
:10367000388E808CC4950906ADC5180285600C276C
:10368000E6D348FFFFE0413C8807F1201EFAC083E3
:1036900078000F67F38007AF1E441678EFD95D0CF2
:1036A000DCBC79E034D3C403D399E2F3A0F327D38D
:1036B0008B7A103FF3013D0860FA6A665FF95ACCD5
:1036C0004AF3084D66183E60DEF8679A6602D32218
:1036D000E0B472D3200640D33502C566A93D101967
:1036E0000712059FA2ED59045160FF108890283001
:1036F000010208590DE4037022C6B319F92209F535
:1037000022421404FE3E0B6011BF4620F002A2804C
:103710001002062117049009F81005F0FF20183454
:103720008103FC420251206A4F21280400E2C22694
:10373000D15742A8FE0295DFD63C24A8F8321F8458
:10374000A01014021E4419AA9F21C6848006D033FB
:10375000EB61D322E781A0119CF8FA5D055ED26B84
:10376000D764E5D5110C6E97AB970C56F80680C957
:10377000E1A3914BDBC15EBBABE31DE6FC806808B7
:10378000BD9814030220F8100A84013C60085DF320
:10379000FEBF0F600159C9AEB34681280705C2209C
:1037A0009918D350ECE4824128D3E2861EC8C35155
:1037B000800A410BF058FB0811EB82DF9802600889
:1037C0000104C381805F14408C4F962141A46FE2B5
:1037D000E5D4D4F8B32F905B6D3AC2080C0671742F
:1037E0002610C85F007E428124178410DAA6FAC52D
:1037F0001146EF4CC523B98CC9E0310EAB2BF3D386
:103800008B8C8BB0B3205FB38511300246A740C2CA
:103810002360045FCE2BF3A47ED33C640486C67D74
:10382000F398F9E001AF97C59798BED20C880710BE
:1038300040BD981836162221D7B1FA6BB105167B18
:103840006B100B5D913FF3314006C40229F3C63C77
:10385000F308E0FC0433105E9847C379D278F297FE
:10386000E3F3FDD88B79981C66D37066077A6B04F6
:1038700088F30A70F3D9FAB045A017B898890251B5
:103880007C41448132531CC0F113200350338C829D
:10389000D712673CB3281005A2FDE0580451200A56
:1038A000784BCCF324A8986A83EE2010217AF33861
:1038B000FF30E03019D004B403680CEB41A0099745
:1038C0003012FA9810BAB1CFDAD4FE8389102F42A1
:1038D0001843EB200822C39975812611E9A993F3B7
:1038E000FD4D2088340280FC307EAB4681ED61B90D
:1038F000300862D9652D9517F8828BFAADB6FB5C5E
:103900000CBE4DCB50FC74EA0905EDAF149A8F063E
:10391000C0F7A505C48042F33D22F0986CEDAFE4FA
:10392000CCCC05C11EEBE05240C44CF339C1FAE7E0
:10393000D003504F68813FD448FC2C90049291E70B
:103940006C372100128F2844D3B08035820272BABE
:10395000A025B09E19EB04A1A0F0F9827A220801FB
:10396000D849DF111040085822A64A20FFF0C05C59
:10397000FE8405C9CD16E9ED3DBC4240107AD21651
:10398000BE9F8546CD79989D9C6290050941E026B1
:10399000F24C642F8C824100827F63D308CE60A7F3
:1039A000820576B368FE9C30B400E25DF78B900729
:1039B0001101FE9876DB492C1908BE1230E026BCB6
:1039C000A5FF6B5EF040923079F380E6F778FF84D4
:1039D000F15D3AC3806020FBA84F34C5EB0A23B6E3
:1039E000B102ACF88901B8A8D35DA3E7A50BF34BEE
:1039F0008F89E123CFBFFE8030FD08890223407705
:103A0000EB21800B02C8779D98A1A55BFA9814D58D
:103A1000F88A9B2806A29786A3FB983002EB24C85D
:103A200008E33078804890283F0478FEA0010E8299
:103A3000B3C89A13230AE74121288DC206376C1AAE
:103A4000E82EB3E6F2C879ED348010A6D70A4235E5
:103A5000300120A5A195C8CC300A12FDF31004094D
:103A6000F0FC69C27DA1BF1E406F5CE85B4946392E
:103A70007219018C9A9F82BDECBC70EA57CEF2732A
:103A8000E0FF19EE90DDE02B035D0240813C715DAB
:103A900071A47C722988F36ECB6AF8D788400E0334
:103AA000A61E8025511CF2C695F0F3F3BFC664C173
:103AB0008130CAD0F966C9C845F88044A00821F20F
:103AC00024B9B3CC884094DDA642D9C86E755FFD99
:103AD000D181207501AC4F9E06814018CE2802E2AC
:103AE000448283EA674202B34830F80126C004806A
:103AF000DE4060024C1409E9F310C0A00332984C78
:103B0000B459F3A319C8019C06D324140A1368D32B
:103B10008249C669AD98AA4243C6A5F8AFFB34D224
:103B2000CAC8F2C5CAF5E230F49840AD9D8449B2E6
:103B3000C8CCDDE3E5FC030212B830EF3F98CB5E62
:103B4000974D7AE4BB1ED8FE80D7C5988CAFB2D211
:103B50000604F3BA7A8C19434F15CDD5C0DD446CF9
:103B6000D359C8775FDEEC8B89FA4B09F3C811FF94
:103B70000142200A448128B0AE08783010020320A8
:103B80006807DFD64B04CC1111225BA2B4DDB8303C
:103B9000B9DE105E5E135804E22061025790AE7EDB
:103BA00050E73088401429DCE1115E987F363002FE
:103BB000489E986CBC2DF2F2C0B90311E128024274
:103BC00071082221AB44C79888184359C8AF2D7497
:103BD0009802A0FF5C6BCB4540FCB6DFC8F62CC852
:103BE0003721F2973C625DC8F2983C19EFBD3BFC6F
:103BF000D740812E5DC0CCC8620218B9A7057EAD42
:103C0000EF524C6DC56684730306C2D12016E0F9ED
:103C1000C83CC6A0801EFC955020044281F00B9049
:103C2000FB2C23A0E74082FF48100B8421F32008DF
:103C3000308247805B2FB928C430DA4203F2850115
:103C4000D5AB21EE841012FCCC22559203A479C688
:103C5000140418EA1DFB2FF90182FA8449C4812655
:103C6000048D99932E57F7C52026C15B775E98E1A6
:103C70002C1004D912DDB1E40832098B75DD08641B
:103C800012DA629A09D324D9FBF3336249F398B468
:103C9000FAE56A00DE98B440E55D10BFA5983C9156
:103CA00098B27AE0B4BC98BA91B2C8F2C6F2A8DD74
:103CB000F6E8679BC0F8B684E16A2EB410F2C53608
:103CC000CBF3983F4EAFF2D2166677D9C8B9C0EAA7
:103CD000612ED3DFE9A1F980123202E75D8802513B
:103CE0002BE0CF98E6309820BD980C4AAF12326E88
:103CF000B45706051032F40E086B135CD0C8A2A7A7
:103D0000F75C20802867AE88FC9920FB8209157932
:103D1000987230A87859C240119A1A4557D02CA0F1
:103D20004442331CB3A051845F16C418025C307641
:103D30004AC8643BB48B308B23DB986CFCF58C0158
:103D40006E396FE2126658F7F8FFB69156F684F5B1
:103D5000E998F8D0EABA06A280F2981F647E3C1077
:103D600006C0D7400896B8BDA2813C8008A99CB87F
:103D700011AE32D12416D365C821F3063B8B307CBB
:103D8000F68081281CD0F89A106844445C60890849
:103D9000010640657124E37251285766ADC5118D47
:103DA00019805A578672BE280891FC9AC8C642F9F3
:103DB00017B6830C21CF880464CBFB80CF45B0C2FB
:103DC000C02258FE048B60112C024874F320C4CC2E
:103DD000AD03489488E6B60277C932E06216140251
:103DE00074D30C8251C6CDC820C610C0C68EF3391C
:103DF000FEFF57C5F29A9866C80CDFCF98E59A0483
:103E000099C6CA9E6B1612D0D3DFD7987A20F33D9D
:103E1000DFA8C030575A71F25D31569365C8107DE6
:103E20002D2481F830DBF45E88D3EC02C0208E05AF
:103E300030C101A65DC8ED7E31FBD9C8C31641AFC4
:103E400089AE80CC1811ED16C01910BB0385B5F3EF
:103E5000B91AB15E730384C0097130AF9398699841
:103E600004CE20213E90116BF3E08130E280207F70
:103E70008242442308418D5FB8773D30424021089B
:103E80001295BD01CCE5CA2177241004D7421284D3
:103E900098F78C8105857130669B683781A4051F72
:103EA0000298772930083A106FE7678BC333306E7A
:103EB000D0F1BCFED9A44065F03002EE9BB8D8FA30
:103EC000B93006A6A2060150018C0CBBED8E235919
:103ED000F30F3E06B55015F8D3CB3D20BD9860F4E6
:103EE000400EE001F3B8B4B3BB84C0FA412810A07F
:103EF000F9E630204400D090FC8808814030B23090
:103F000080BF4C0B8E292F418411311199C5CBD123
:103F1000D4EB91EBF9DF9844044122502B0CA4BA66
:103F2000B325EA64217C4240FF845180E1C5C0286A
:103F3000FC08886014404F51B000465F5FAF05E653
:103F4000578C824C10CDD7FC835130990AE0224621
:103F50008CA3E38B88F3C6829D93FEF358B3FA7D5E
:103F6000983CAFA01098F3179198F39DD674BEA516
:103F70009716D3F23D3DDB8F30C8BB3A70FBE33080
:103F8000BCD25B5AE4F5177EBF40B61C1B3F8D3098
:103F9000739B147F36038841FC3024D258E7F3D852
:103FA000FFFAB2089846F3993F12240A288869C29A
:103FB0003047BB874C5FFAB3128EB3C9D5C03F44BC
:103FC0005160018C80B609E0307E042C1021BD9D2B
:103FD000FACEB045CC0614B93010FD094101285085
:103FE00000A79D9897C871309AB35D24FF9226C0B0
:103FF0001840481069BB0CD098882BC0DACA936867
:10400000E80A10053750F92DDD064FD432BEBE8FB9
:10401000CECA7BF22DD3AA24A4B6B4022E0C2F8EC6
:104020007551F0F980BF8D07A0001497C0647CCC57
:104030005E2005C45FF3E5A6C6307E9DFDDA64E12F
:1040400007AC21030FC04DF305F07527DB1CAF440F
:104050000D51FE070804F81106104802C7A2208877
:1040600039153682E6144E08232A6CE0248E363049
:10407000F4DD28FC66414010240243EF12FF812248
:1040800048209140D800E6580803822846CAFF42DB
:1040900038FD0450300840E0C42018708360108C54
:1040A00030315A06F69804136B984CE55242A9B386
:1040B000A82581ED213862085852835FBC9870F3BF
:1040C000060129981211E7808141C770F97785C5EB
:1040D0007E5AC86A0288FF5698835DC8CBA7075CE2
:1040E000B52ECD26E8A733301EC4D31069EF983023
:1040F000401EC8C600797FBB9848F984278B30EDF5
:10410000977D9803AF4091BF666D051BBBD0026ED3
:1041100000305AE097D38778598E7F173097987080
:104120002AB8FD57175D1FFCC330C091B400F0984A
:10413000D224E16099B0B5E3CA6711842830E32244
:1041400014C41EC051408257D32B03A2E46B1A59EA
:1041500004A6AF28584BFBE6AD3404FA16C217FF8D
:10416000BCFF205F17771F68E65871F39CACB12243
:10417000B6D3B8F9030485FF988E1966C6D138D333
:10418000D8ABFC24B66689FE78EDAF93B05ECDB3B4
:10419000C8B1FF222434B133F3D6D0013417D80983
:1041A000FC24FDCC6A15028D76CD1FC91EB8C04611
:1041B000E579B1657F882D9EC41BF7F0FE378C4AE8
:1041C000F3FF2FCC4A73F6B23823E29844C356FF6C
:1041D00018FFFDA3F80C2C47C556D20138B3DBB845
:1041E000FB1B22FDE2BE5E05EB1999E6CB79431F6E
:1041F00088F700FECCFACC16DAD957EDDF284CA3AD
:10420000D56B80AE99D7CA5698FBCC3C1ADCCCCF84
:10421000FD6D409FAB984055F78436A668FECBDB1A
:1042200084B663DDCE8162BDF8E7812090CA1008B4
:104230002997E4480E04453C6FF313CFF8681999A9
:1042400012E450C4BC41B3F3B9BC751F28A1156674
:10425000A0B4606E15A0D164AFBB0AF8FB0D855702
:1042600024BA4220014468A6E8FB330A50C289A45C
:1042700057E7FE84C012025386DD4940B3A8DA66D0
:1042800021A411B487342A45BBCF6120C6446053B2
:10429000F12E400508CCE6445938B3657A4F048EB8
:1042A000B31666B339EB5F087FAD36B74BFF42A05C
:1042B000FB0879E592FBDC0241DB71F719D9FF7F3E
:1042C0009109998AD915FDFEF7BF00DFAF0491EC83
:1042D000EED2A3F8C4B60E03CFA735852FAFB78EA5
:1042E000F5EB0218DF9F769510FF7F5B498D59C86B
:1042F00001B93C88F4E0B6713CBCB2FF314B5ED9E9
:1043000067084BC4403C11C4F9E3F096FB81091ADD
:10431000AFB3FECC8C7F38B820404FFD57449DCDC5
:10432000A1F0FF91B659CBD1200DB973E8B6FA17B9
:1043300070FDF9361BBF835F2C9B7F8D124FDD090B
:104340007EFA6FEBF50143D67DD93920DF06B70140
:1043500004F4BE18DF52ED18F16EF8126CC658FB6B
:104360007D4302629DFC1D886F1138FD676EB5406C
:10437000CF16BD502FB67E67BB7970F90811FD3797
:10438000208C6AA440C57636039319FCFC0541864F
:104390007102408EBF0D2091EC04D9AB8F1455F8FB
:1043A0000A74350A2437D3FD0414AECE8CF00428E9
:1043B0004DC8FAFF7531B905846BFF032BAD41FC85
:1043C00080E69CB0FFC92359987E59A368E62E6FFA
:1043D000596EFCE23BD088F908967302126A15A860
:1043E000CAFB3233CC0430EE4BA0FFC7FCA5C22C75
:1043F000A262876D1198FAB6F9DF8C6777AC66FC1C
:1044000096D2CCFD6EB1FC1F4BB902CE2FC858EB33
:10441000D34C7C751990B1FD234D7D330E3E45C7BD
:104420009BB0F8FD1AFDE6088A7DB1FFF1624BC82A
:10443000FD17D8FC8CE3A3332B1B8CC7AE9A8AA143
:1044400030E77D0C01807E515CE71F1FD6B5149EBE
:10445000FF5B9B80FA28D637FC2DEB73803C68C647
:1044600057AD20B74D18FA995C7CEF595B7F91C826
:1044700095889B9DFF0E048465FDA737CBD0F899E6
:10448000F4A96102CBAC08B1561F8E9DB726244912
:10449000C080AD002981DDD70210EDDB01378BA094
:1044A000C034FBD10510B8C858502F2D976B82022D
:1044B000809E9043092808CBED670821E58043A042
:1044C0008334D238EC0340D26CC54DF3B354E8C802
:1044D000221D04207868621011A27E740253EBF74B
:1044E0002942A081E462424CF7A0202528FCEEB6C8
:1044F000CFFEFF8061E44F323C9206F384A203209A
:10450000CB5CC00410884271F389812014ECC8F898
:10451000EFE3ED0801B24CF3E11960B710F96D61FA
:10452000657EF741BFFEFB6BEBA80833B2AD81E6B9
:10453000C4F415829695E8F2D9FC8B2DCEE720F3D2
:10454000D40ED72CB0FF906FF273121B1EE3D47EF3
:10455000AFFF0A63D5E8106E7BECC4FD125B4FCF52
:104560003754DB2D2CAB8C214BDB661CFF12F12A60
:10457000E8B40433F8CFB03315CD045BDA88FA73AE
:10458000ED1FD3A91F6DE190FF02AAB6E4080476DF
:1045900038B35F89669EA5A17EB77298FB1DE4DAE9
:1045A0001910EBBA4F9678FB31B44892B408FDA5C8
:1045B00048E5A6A653C4ABB2B8F9EDF3A633969E70
:1045C0000131B5F4967E405D35E6EA8FD50804B832
:1045D000FE62E67C1272CC08D8029DA878FC408866
:1045E00018E0A9C58FF216D0CC3066AFF636017A46
:1045F00093FED9EB10765B06713718F6B79A9B8B52
:1046000008D373217FECB9FCFB83D52D0F80672C79
:10461000F708451240663F6098FBA0090482FF102E
:1046200012004250130844C421289F36F314021A82
:104630004102092D817D609E36327791E0059ACF47
:10464000A421221005E08220D4780A432308FF0D1C
:1046500020043502D2C0FEA110BA1CDC7D5FDAC492
:10466000F7F7CB02012C14FB1BCF59E88E77C00D56
:10467000C2D90CCFF3B0FA804081280587C216F862
:10468000108150200A2B985105A25F08800251200A
:10469000F60C84012872B56064CA80D3BF4DDFA8D0
:1046A0004081281006EB02000E80704F0CC63800C7
:1046B000C8A7FFA2A220804279E22E212406818889
:1046C0000710024088447D1D880009068877A434BD
:1046D0009077D0D4E893A9D3B94433F892FD62F12E
:1046E000040C20843F09F0F90090301606B4595CA0
:1046F00053899D013E06C037D3036072FA30CFE67E
:104700009A09323389E0F5149704D32BE042EB3653
:1047100049BEC642E198FFE07F3C8807F1401EC4D5
:10472000FF0378100FE2413C803EF3201EC08392CD
:10473000F3E4E6CEE1DCD348E0111A1E08748305E9
:10474000E041C6803270C68328F203E8F31892FD78
:10475000ADD566037B6630204D861810EB66803C35
:1047600066DCD3BFC208686626F8D340E0E621E6DF
:1047700050FA9E1237A2C004C18902FC21804481F4
:10478000002201E1489F8401240A2CF68205104092
:1047900078B3E02F02C84910DFFC30B3283005861B
:1047A000038B500AA144E6C6FA0450FD2010D7E757
:1047B000D202828040EF47980481A21448F308F1A6
:1047C00041E520D4B7AD982458F812201991167DF0
:1047D000FF1A40A1080421A001FC34802610884A59
:1047E000E7D30A02D304050F7CFF2EACF8168FD254
:1047F000D9D34F8981F3817140BF0BCC0055F806A6
:10480000FE954A1902FC5B085A3022F35DCB49F948
:10481000E2F081FD8193307EF3145EA525503927A7
:1048200045C0F308039A52F340F39835B3663CF65B
:104830002002C05818ABE4DE195931ABF381400EA9
:104840008468102916D3B891FC33A780DF284291E1
:10485000485F1775BA0682ECCE03017808592130FB
:10486000F76DAB450A57F88511B600E29C0418783D
:104870004208224CA2573089ED05B593602EBB0447
:10488000E111DBFD880F4046003F93012360048C5B
:104890005EA59902F344F3C92061F3E62CF3E6B375
:1048A00089B060FBC15780882C9622261241827005
:1048B0002A23205ED3EF41FCE0F3A5BCD2EF3F9862
:1048C000D68B00DE8B625E9827E01E06C0DD0358A3
:1048D000EF980C90077069E798B5D338FEF412E3AF
:1048E000B440F198F56DE7B8F98B8A7998C0512EEC
:1048F00062F09808F3FF349848D381B39C320AA23F
:10490000332002D70124B5985110EFB8280820A30E
:104910001B0A04819010621B2C5D48B9C008605FBF
:104920003B9411B214805131D95E5E851290FCF92E
:104930003010B48826AFE63F98BB130681FD980B74
:10494000AF09589848873830203480B510DC70891A
:1049500008FF7822103580161204FD4250080A2202
:104960000178984D40FBFC3839F80804DD40B1DD92
:10497000E28BA8FE58D288968A15334772104015EC
:104980005BF975E4FCC6E4D8FE4075C544A1C318C4
:1049900080EB60400CCB8B8730F388035C23D8809E
:1049A000818F0A3054F278F298F354D0C680A21660
:1049B0009405535D2AF250FD2C04047FF382886035
:1049C000084204CC2830A091C63944CC40885641D6
:1049D00088D4333FEE7FCF8A4850609D0A654C21D2
:1049E0007FC52081CE0242D1610167C88461D0F9C0
:1049F0000E05BDBAC1389E080B049A23F321E716B1
:104A0000C002A12064CD012CD4B2B1BBB7B243899E
:104A100005B550E0AFC694242BD3A3DA831825C67E
:104A2000B870EAEFDB58FEF598F0FC3DED000FE8BA
:104A3000B830FF2E9833307565E4EE810488E63097
:104A4000D003B830F6C671405DA3C430F30F78F8D8
:104A5000BB84D5C5C4FAB003EB145D9096F31DEB8F
:104A60008B407F3698EDF681C7D31DA3E798F203FC
:104A700040ED86F6BE5299C630FA4D91A255B81453
:104A80001801E7260C82C600325C30EE190142F3B1
:104A90009823963014FDA92BE0923058F7FE1C3075
:104AA0002124421D19057A9820BD5102AE903B3059
:104AB0003BC8249AB8304C9568A2BBEF9F300900E0
:104AC00041A2051E0ACFF69804802D117A6003BC1E
:104AD00098B91089F340D4181AD34A39362050FCBB
:104AE000CB98FC2581213F973008E4980764B647AE
:104AF000F11A9C19BF0124D0264A035EF808E07F12
:104B000051843E7F2F78F95A0259C8DF801C97D50F
:104B100032F306A42AFF1B8B9E306F36E575F868CA
:104B20008030D7378DBCFB48FBF600AE760730826D
:104B300059BBD218FA19A19A0E02457C758828042F
:104B400084405810B842489341D404099FDCFF8246
:104B500001F1022408029C3D9344CFC810D70204FF
:104B600061CF6049206619F8D2FD8009301226C64F
:104B700069B213ED904FF340C20498C6001380242D
:104B800096382286BCE3F8E031346DC257D608640B
:104B9000640909E883C64124D31AFDA7043201C081
:104BA000FA79DFFC3D7E5ED5F35E8BAFC41C8BF3E0
:104BB000813C366EE6E3E08080EE573050EDD60B58
:104BC00077F60235D358E598ED6B30F8FC5D47A6D3
:104BD000E5D5FC3DBBC1C0C5BBECF9FECB178519C3
:104BE000F4BCEF5A6B08F96BFE98D60C02B5EF21B6
:104BF000F9B53B92C83F0AE6300C88BF0A463FE54C
:104C00000920016404822CC8DD4904BAB132BE7F98
:104C10008BB0EB32D398B06988D744181330791130
:104C2000100BE0F9F0304484802B118230F96901D7
:104C30008DA2397F17307F174181A811050066F6D4
:104C4000B103EF1D98881A497B782128AF447A5E1A
:104C5000D1084248FF4841A005130110BCFE4A1A82
:104C6000F5A502C02B1EFB28F331FE005DD78FD2C5
:104C7000365D3F59CEAAD2154AC6C0DCD8F265F2DD
:104C80002BC6C050FC2CBA06A040CCD52293D9E04C
:104C90002305AEA0FFC20352200AC041305B646509
:104CA000AB6664FFE6058280080448860C2EF46B30
:104CB0008498AFD339120AF87AF318FF0C6433449E
:104CC000144F3A22C9FB8B9E84951244824C666C29
:104CD000219BB58F095F35ED4D5E88D489E865234A
:104CE00084F475EF6B14C022183F20481221005045
:104CF0000742C088FB1F320940E0C424983FBFC967
:104D000044300926C14FF32061124C5E76B322B9BC
:104D1000CA09813026A0411AF2603AB27B65C6C248
:104D2000FA72238167D340F390F85EDF5C30AE0007
:104D3000573D799B9897F39098F3366F4E63ED0546
:104D400080ECC0D550B918D33D41F36D0ADDD3B026
:104D5000F804DC4A77ABD2809A3D8481F38B60F310
:104D6000847FB3FEF64903B83DB586105ED07F97C9
:104D70006B77482140E7C890FD3FFA1005164414B0
:104D8000F888020B40827A0011CDC8487A9803B99E
:104D900030103B2C080553BB27C598E07C13A6B305
:104DA0009305113706E01427B3C60144304D12B7FE
:104DB00078F8F230D2BCA5B9308DAE246D30161023
:104DC00032C8B9F9B52CCDC1B3C08A044CD0DF616B
:104DD000EB97004DC778D7940813480BEB2A002DAA
:104DE000C35E5FE4C730F9A591C44BF36FE653711E
:104DF00019EB081053016E060813FD5E6099FD5D06
:104E000028183EF614900251BF0C01952C89EE989B
:104E1000888350B58601DA1180ADCB40FF7F302604
:104E200063161887875FC241AF28138BF7D33824E6
:104E3000D36DE2B968FD73840481F6245C1F860893
:104E4000062290B798111A4224087E8421286D8882
:104E50008A966E04FF7FFE9210D04290208B02470C
:104E60006C048992C0CF2418D34811899F02B800DE
:104E700013FB80F845B0081601BE58048B6069BA70
:104E800082F300CFC122F3206411922CF319F36E48
:104E90002BB0B5313516C1EB9D01BFE72049C6C126
:104EA0007C4CF58124200EF3C1FF5F4697C8F9A51D
:104EB0009FE698DD6CB5244BB472B2DDD340011887
:104EC000AAD37003FC9803B2C825FEF9C87F1D6AF7
:104ED000E7A528F3C2F30343F36E3230BC9089D3C5
:104EE0004E605D6401E5C6FF72204004824DC60934
:104EF000FEFC300F4488AE0264302890F3BBE88F8C
:104F000030CDC82871F399CA2F012DC04AFE99FBF4
:104F1000E8581C2110050CE880C9B34257E077B56A
:104F200098FF30E9980607FE4250236804412800A4
:104F30009FA206D0001A5C230F0DB0EC110401DD16
:104F40006B6290218730F292605AE9C04D205E98E2
:104F5000CF1488B513280C3F6304B500F8F97F9788
:104F6000989EA5F87830A3E7774F1683DD676F64C6
:104F70008ACBC7BEF98FEF20DB0D7B8040468EE8E1
:104F8000FF4F5D3202A400B916BC0A9360F3C8401B
:104F900030E084D1AF79C5B7AD065254F86019E955
:104FA000053240A3180F04429C81C605C002AF051C
:104FB0003803CB3CF8C8FA2C38064BB1B543A050A7
:104FC000D2111985BEB329955C2F0F02449684DF58
:104FD0007747FDF8A010D00288DD83680026108492
:104FE000D7887859102048A4768DD060FFFA845174
:104FF000300A40C028E7180508588C8270F399A43D
:10500000B4A3674292F3CDD7AF8411320246B8D72A
:1050100072C3600CB29AD34641DCC080F3642C8822
:1050200051B3D8BFFBCFD2CBC86F5F98F1E798F1EF
:10503000239C67B460F7980640014BD3E44F326B72
:10504000393058BFFAD698C45FA89840F3BCB8E38B
:10505000E610EB17FCA53D022FD388F65E8010B456
:105060004CFE77301050FB7B9804405C3007418247
:10507000DD4481E3985090F920014400883F2CF3EF
:10508000E5B208FE989245FBA8B2C8BD98C818338F
:1050900064449501B3BF1D78FCA01159C8F51208EE
:1050A0001A41C730F8980F14248260F40368018114
:1050B000D40D9C66BF05C7988A40080B81B0EB09E8
:1050C0000482582A0242B02A7C8D200405DF96F91A
:1050D000C435FB5F8F7F9F1CE78F1FFC96C76F282F
:1050E0002885198DD632C8F5C68011A9F70EC3736D
:1050F000B0FAD335D540EFF650200A602571F3752C
:10510000577D1571301964BA625C3022E0BB63B719
:10511000FA200C88402FC61A98C638EA7CEF37E888
:10512000F800E02804A1FF12024044080A01CF4120
:1051300024898520841311013F9D1441210884098D
:105140009BD9B1886E3088D2BA9010232D66C5E005
:105150009183889881446935E924FC77EAF8FAC19B
:10516000300806C1F755836010E80C8241F3BF8315
:105170002008BCAFF3D46D5A56A411106984D30A29
:105180002D12DC5550D34CAB83209074D37C1290FD
:10519000FBE0264F193DF9C8B507ED1F03A3F868DA
:1051A000807FB7980E487230E8F5D3407A9858D38C
:1051B000D56B60A6159C30B708F298F989F3866123
:1051C000E0F3AD7515D0B702FA773BD3E4BB3927CE
:1051D0009DD3F2FD96B28E984489FF1505CC3040E0
:1051E00014AE373F30CB98D7C59875127230101374
:1051F0005EB6B85A11047230810271F08C1011D76A
:10520000A79882B35140E18108804432CB10FFF46B
:105210001A32FFB87DC7DBFFE8FBF9941044753CF8
:10522000B3018CF3E5AC228DB0D3B8F918243BFF61
:1052300098FF2C1A33938CD17139F288F9C1216609
:10524000D8B0FBC4CBDBAF3AF3312919FCD8040149
:10525000C9449CBA6AE001C6E0FA866ED3C451FB29
:10526000608FF5CCF67F2838632B1C08D62404C445
:10527000D7B55D9169F8CCFC2C23F14BCA610A8E3D
:10528000F8C2DFD87F4093EB018019A3E3FB220330
:105290008210B508FAEEEA433C393558F691CA8BCC
:1052A0002D9C203FFFFF345248DB18B1C3F3CED60C
:1052B0002560521E48CA1DCD4BA8F98B7DDB1BDE35
:1052C0001F61E7F99980EBD4102D60FC5B826E546E
:1052D000B80154C73ECDD34FC1D27ED3BCC1A121AA
:1052E000FDF22CF59EAC17B2D18F1E089DCFCF7B5F
:1052F0004010885FA58008F01B5204CD2B8DC65B43
:105300007618FB6174C7AD1ABCCDBFDC24CFF74B58
:10531000E0281D81A530D68002A11B0AC32CD00D28
:1053200030DD81BC220168AFE6B3D0FEF36096B2F7
:10533000389FDAB702146AF5A5B390DF667BD40113
:1053400004C1175014FE42600C8C88F102B53A3843
:105350008508E0EE05030A6564CCF8FAB7D9F8C20F
:1053600075E933102519DE411DD8DBA740C5CBEE0A
:10537000BFB9FF38F90A7867FE5702CF37A6200475
:1053800074C99B8116108EFB34DBE8062E65FDC4C4
:10539000FA93C61FC6BAFF4D6BF95802C56C6C670D
:1053A000FABF02CEEEF1B0FA03CDC5CFDB3FA78F37
:1053B000F231171E357C2384B6B8D25EC5917F04C6
:1053C000C5B5F93387F8E4C7BB6E01B308DBC6C8BF
:1053D000FF43E609742F68791203F3F6116CE28833
:1053E000FF28E3DD3C64CEF7FE98FE406517C85900
:1053F000105BAA62BC20B101563D48FDF32170B29A
:105400002D1BD0440145C6088D1E4F164B0B40C6C0
:10541000BDD2085B1928EB408EC53F730265AF29EA
:105420000863E00104310FD85518C7DBCC9B26ACCC
:1054300012A0F5E48499BB49F91D33B5CD54B88B5E
:10544000CD3D4866FD7157855F31B3104CDDA71621
:10545000FB8001AF052F1001C002CD4009F011DD26
:10546000949918F02AF5EF280120FDB10CAAD50671
:10547000C8FE2E2040DBF21124FBD7A770D2D0FD4E
:10548000626B7280257C0263CB488066DBB8FE03CA
:105490000F96FF012DD2FE48C6B21FDFAC8A5BF625
:1054A00098FB59498FACFF2163E775FFE8F961FA72
:1054B0001902DD4BA8B0FFE0BBCF6CEEB8FD8D3616
:1054C00015EBE23CD2FDB2F879F2206AD6B304BF04
:1054D00021FF5BDF636B900217EB9E3DFF94B7F9F2
:1054E000EAD2DB7E406A2C7BE5236CB08002C4C923
:1054F000CD47681CB3B167987EA6ECB2C0F35C756B
:10550000D4012CBAFC83BBFAE9C4D6B28026C067AA
:10551000B63C68FBE5D3E6C8BC18628B60108CD83B
:10552000A6904840CDF69390F86DD408F22E85D21F
:10553000F2C6B17970B942A0C327741A82D6038D1E
:10554000D3DBD850FC6274D3446DD07920B7467E4B
:105550009E0F5A1D21BA4473021080DA011E818108
:10556000E1201E89CB844D7134F866C290898EFE8D
:10557000287A5F3001D65FFEAE0A34A5001DCA78D6
:10558000B3A8092514FF8002180012E14A432DCC6C
:105590000DBB053A06FA6A26C3ADC8F9EE5C33C006
:1055A0006FADE0C0D581CC6088911CEFF6E1405E24
:1055B0005A0C61B420FFB5041020C4A071F3AB1CD9
:1055C0004190BFA2FD481440022390E09221A07CAC
:1055D000088C012430BC19B3DFCF61FBCCCD0C3477
:1055E00061CEF1E3A99A10E02121DBCAE26C4BBF46
:1055F0008066D9FDB8DB2F2ED68B0402F3A618FAED
:10560000CC249B8C2081DA4041DCDBF8E9C9F00234
:1056100099B380FADF968220FDF4B5041678F03550
:10562000D71F9BDAF6CB0276B714F9C68D35C6DFE5
:105630007A5D5051D072E5E7F6B4DEC9D860FBF967
:10564000BF9FB5FCE6E929DB93E0CCB37FAF6A31BD
:10565000448DDF7228E77D75B1878BFF1025F9989F
:10566000B4FE22112C3BFC62DF2F3F24E5F8F38BC4
:10567000ED9E7D05AAC9022BBCDCD5F318B4FB2F27
:105680002936EA3735DA8E33ABD7FF248B9CE360BB
:10569000E50F38D7B5B7F3A862D9C8B38056F7106D
:1056A0007FCB64A93F96F1FB20DB69E6032C9EB219
:1056B000200CF2EE5EA6686679DD896AAF04CB3312
:1056C000968CA8E6B358FF96CB40FBE50DAFC0CA59
:1056D00079D7FCA46793B79E24309B408110728BCE
:1056E000E325DBF9A0FC45B703B17A1FAFF223B77E
:1056F000CDDDA6089DDAAE2138E0D8C84C549866B6
:1057000084E7BAC65062488037E72C731216C4DEAD
:105710001802B246E67F9733F1334201B91A4003CB
:10572000E0CC4122C090A485A663F3A7018031D3C9
:1057300018ADFEB2F1C504E28D1EFFD32CCA51E4B0
:1057400090C8FF40E07A07C04E1B03750F02B956A0
:1057500007AFF0B1725ED7C580E8BA06B05CD3136C
:105760006A05D2C0037FE09B11D8FABF3810EE81E2
:1057700088025FD541E508AAF320E9F39B622CB0CB
:1057800088B00B449D6843600820C7063BF8F16071
:1057900080694E40086CF8F94909C529F74601C9E6
:1057A0006104AAEBAF41F8D019012360BE8C8011CF
:1057B00030CECA662EED691308986644E7488031FA
:1057C0009146C0F308180120A68C244ED329F96015
:1057D0009F352694001ED0F30278100FD13C33F38E
:1057E000F4F3C4FF8378200FE2813C0867739B4188
:1057F0003CFFA00430201E48007839B0E201F3E7F6
:1058000007F120D3037ACF000FF33D0840C2FC809C
:10581000953051D45B51020C8B5159922018D644CB
:10582000F3E6671C1AEDDD02C0F97F603BE98201F7
:1058300031D380ED18108358D370FE4BFAC6164250
:105840004EE053110C029BB3A6C0BEA64344AF84E6
:10585000B39295B345C3EE261997119371C3019383
:105860005FA34386D309FF011050FE3040140607A2
:1058700052820A0875FF012C9A23814FBE42F260C2
:10588000142123DFB7E3D354F832F3C5902212ACCE
:105890004068915F9B1E0257D3873F40846CDC9E1B
:1058A0009617A5FDB644918B6FE4090079FF7DF052
:1058B0009BE7739BAD731A90FAE5808130EE789880
:1058C00055FDF90F42E3C10C04CD8378BF42190C9A
:1058D000C4B3F611CBF98357EC06C12028D3A4EF4B
:1058E00099DF29F9ECD220914802E5A221E8990834
:1058F0001241E11D12DCB6BC0ABDC867F88550E054
:1059000014C443688608BF0C8FDD1A3BF5407AF358
:105910000193FC84CC9026C3EF58E00B2220F59035
:1059200081B0FA5F02F8C1FF11048421101D9AB3FF
:10593000EE051080CF371801033E324C8009B05776
:1059400088C3A1C30B6024D3E57F81FC6001F524EB
:10595000800792E99803B0DD0FE0EEC5F2201664EF
:10596000B078A3D9F32CFA33FF800C8804F0201E02
:1059700050EE007840F67880054D83D383CCD34138
:105980002CEB20FD842F28F69803203F0C84017710
:1059900085984966618025F3939CB264789807F9ED
:1059A00098E566E7E5B2D319FBA3D8B36BED8CCECF
:1059B00085FBF681F3B13F734B043222B32472E0CE
:1059C00014B833BA0AF1A6869A0CE530DC49201CDB
:1059D00014911F50808204357221E7407A98048B1D
:1059E00092BB4E24103F5F13A00104800281D28A33
:1059F000DA48037898277A99481828D3248015968E
:105A0000C85F17E699981ACC5B6467F5B1DC8D77AF
:105A100099C0E4CBB9DDF8FFE098175E9EEE946084
:105A2000D8F3B420F14CC6661BCBF8940A1EE3CA27
:105A3000FA37F261340C68D3F0FE4466EF88FA510D
:105A40008BB84FDBF398F49D767B280423B996043A
:105A50002F5FC5DF0B61EB9885F749900A0A67D382
:105A600048D3C8FABF80CB98FF3F1360108C84FFE7
:105A70008530212641405804C58360F68C828030F1
:105A8000DAD2B5124EF8099D1204692E146641F15E
:105A90004C804510EE46EEFE01211D0C3BD308F074
:105AA000FFFD98915ED25C6A778C98F3B09539F3DC
:105AB000C230E6DF803037D4AF3CC96A10A446BBA1
:105AC00078953D2CB41CD3AF02225ED3F9CB6B7F0B
:105AD0008BE5666E173DF378E514F32D93F424DB24
:105AE000ADB13D98146BCB30114F23E566D3D3F0A5
:105AF00019111CAEE53430E36ABDA5C201CBB380F9
:105B00008CA6ED654D8A013304B345D3F0855FE67D
:105B10001EFBB63552FCE898849551EBD288B2C88A
:105B20002480EF0F0442CEC88C211E3006CECAC896
:105B3000CED502116B6C48FC6024840574297697DD
:105B40005BC1B58E0406F4F8C47CCD037F3798336F
:105B5000BB0F5E59ED04B9193AB0B8FBF912066DE6
:105B60009AC8405A5007B5C60F82F6AC6FE3CC8195
:105B7000D00C269A43D318FA523C267FD98748770F
:105B80008E989A8110FCEEC82122C9BB397E48C884
:105B9000E1A1D909BF3226658BA406248851FA26D3
:105BA0002FBF21CBC884B0A8E6CF3BFCE0206187A3
:105BB0008257983FD7128090053204F040C0229857
:105BC000FC9360028096FFE776657C01BA6D6CDE1F
:105BD00098060A3410F8FF26C124581F0360122CBF
:105BE000823F590999FE60808D2405BB90D6D278FA
:105BF000BE98B5F4F49868B6F3FBD46EC0F525B53D
:105C00000CF498182909D3B42DF5988316C64FAE15
:105C100095FD8001AE10356AC9C8F364FD12782B7A
:105C20000669B37D9F1F52E098390A8441667E5B06
:105C3000C87AE549B3C81269CF301301204C4053EC
:105C40000846AFD5372C2CE041D2195AE022FB98F8
:105C500044842DE0B2C80B4CE99B30FD98020652FB
:105C60002BB3C8142BEFEB87FD7F0244880DB1DF07
:105C700004B6DB047A902802E43014F3AC080A6915
:105C8000BF84E7053186D328189043CAAB8C269A87
:105C9000CDFDDF8872C2EFB3343889582CA1FF7D67
:105CA000EC9EFF32C3FBEAC8CBC8F6F19D7A180818
:105CB00083FEC56FF2CC4FF3F98E33EA64D28FD2F4
:105CC0004EFB52B3C81E0DD98E0D64C81CFD0C1DB1
:105CD000A0907AAE03FCD26230C8400D02E75C2D82
:105CE000B5C1FA6CD5AB90CFB010444888449C2124
:105CF000A2052020EB08C3A9C805767081533B603C
:105D0000FED0840973C3C6988043BB04119D10E381
:105D1000C208DA62EB208C888CEAD719810130192D
:105D2000DCCA22D857248A98BFD1FD7C9B8BC680C1
:105D3000B923489AFC5325E3305CFFC8E4810CA0EA
:105D400005F080B516F58B2C9DF5C4CD3088037811
:105D500098C3E01A5E989B3DD3B055C6E838D3305F
:105D6000F9844C9CD7C880CA1F66FADDCAC816F3EE
:105D700093DB9566FB9880815FCC5C5076B76318A7
:105D80000434C68201665E9871B3BF3830280206BB
:105D900025E0AF8DC5C605B7DB42EA6204FF4D982A
:105DA00022FE8468759BD3F398B3C84C767FC8886D
:105DB000FF20091421FF105240020108610C5E9877
:105DC0009C8465C2187903F3F6148C21487E4DC873
:105DD0009E3479B6A73E30202440040A99D3024568
:105DE000EDF021812250B510FC96C8FDCE67F998E0
:105DF00019C3E61930E53566F8C56AE298266FA141
:105E000078CF890801E0021E95F310C830090D7C97
:105E1000A05B471119B3DC305FE9F30A804130D34E
:105E2000F03DF60483107737410838CCFFA859209D
:105E3000C1DB33D1501D14779098391D82447E7C8C
:105E40008185FCFD9BD91628DE818614F588042304
:105E50000AF4B11035FC28F5B097B630D343FD7382
:105E600005209688768F62CE8C810530DF260890DB
:105E7000F5A3D57BAB8F113BA4CFC76A10F2980175
:105E80001B0AD7848001CA7F806BCC0484D30A1E8E
:105E9000FAE081B3C8907679C879400FF3F70C9097
:105EA00007F17AC5786BF36896230267E7DF243041
:105EB000A007AF125798832E3060CBC85F5D6B0B85
:105EC0009EC8E8FD84137CDDC810E798F130725D50
:105ED00040CAE2303735F97F734A6683E330DB66C8
:105EE000C0209766000366C3A9FBB729F1987939EA
:105EF000A62005E0B688CBF571B3466FFD7F04267A
:105F000095C330D3046435D3E0FCEE3081105132B8
:105F1000E72F00212C9828A78135C0EC9863681CD6
:105F20008C01B6D15A6E82ABB323F9761012F141CF
:105F300072F9288405C7E6C60042C76336042030DC
:105F4000BE3006B0FCDB2BD569CE86406D9BE5608C
:105F50007CBFE3A365B34D12CDE5F2B099E478FEC2
:105F6000CA6DB309EE0F5DF83AEAF020D1AFE9AFA0
:105F70000EB6B7EDFD48BE91621679982BD02086FB
:105F800030D3070ADFF68360402027523C19087E91
:105F90009C401088448021E24A5B501E904B024591
:105FA000A074B341222C6738FF84B0A004269FD18F
:105FB000DB0205204822322DC91C40AF7B4FAB0AC3
:105FC000AAFC80BF452EC8FF6C118090073002BB31
:105FD00016C4983B4880FD093140B12C91A2AF8393
:105FE000BC98425DAE126F303009CC9B2075A9750C
:105FF00041BACB10FA53F2C8D3873D703D90DD070C
:10600000F2ED981810725D3CCFE91733321914B7CE
:1060100057B097A51A30E69B5AFCFB8E20B8F8843F
:106020004CBFC8D2D20C17FFBFBF4FFCFB123CFFC6
:106030008EE0CAC8F26BCBC88DD3F6F6BB57FA65B3
:1060400073308C42A705C0C28418CE0113F94C8866
:10605000CF3FB39A3046C4F49823131680AC11D2C4
:106060009BC2C653D3C39860A0FF7C841481405068
:1060700035F5CACA3020E43D16AF8842C56024F326
:10608000EA066AB3A0EF400AD2BB928530A82EF38D
:10609000C6F26B7FC68C8131300670F97FC9F6E796
:1060A0008E7986DECD622BFF1255F809AE985BA77C
:1060B000353070FE97E2A51988F426F0415007812B
:1060C00035EE03786C2C3110E519812130C03F95F5
:1060D000300CE378D3E0021CEDC0F60ECE4138EC74
:1060E000F928634440E40248B9F7E5122010BD6086
:1060F000020340907C9BB52FD36B7251F1CB985E1D
:10610000E58588939A08B320778B40112473031494
:10611000419E22C509B0FEBC98D3F33243F98CAD41
:1061200080FDE140C010180577944C805FE06AB2B2
:1061300001B64F7BF80A10C1499763F43DE049303E
:106140000406627F00034086EFFFF598707998FCA3
:106150003D033C90779EC5F3AC64DAF507F2CA03C1
:10616000D777970165FF1DD3EA78E2E110D315FCDC
:10617000035E6BF63D2028FBFE987701B76FD4577E
:10618000F34B66905D5A15D0AC5E888F3F98A6F1B0
:10619000F3C1F5D340FE6B8EF8C9F198FA3008329E
:1061A00037460267C862107E6DC8044D2153B38420
:1061B000B3225E983CE4206244269C3029D37902C5
:1061C000FD8C88913040E079E58C9BFFF415B0B3ED
:1061D00085FFF8DAFB20FDC2FFB56719F3CBAC22CF
:1061E0001B4BD3B8660487FF98FF2863469371D191
:1061F0008E363981FE092A668925B3801084ABD199
:10620000201CFE7FFE04FEB11B60444C2A62175026
:10621000F83047FACCFB7F3BD6B81035EB9780635C
:10622000EA136D1948FA0CF810FFCCB8B1FF9FD8EB
:106230008204D2C608C43BEB78D9F810E9BD10D768
:10624000634BBB0424CECC6CD694FEBCDB0810ACF4
:10625000F20545B84001AFD10ADEBA4801C86DE188
:10626000C8FC16E711C0D31B79887D5CDFDC713375
:10627000E7C2999486A76FC12FDA80F812D5CA8039
:10628000CEFA9504E7C44B19681FCF0B2DA3087BEA
:10629000BCD0F96FA4D4C3497808C08A2189E39699
:1062A000802C89FFEBAF81206236430846B7E41BA0
:1062B000C5445EC2D6E0FDD6B0E2CB425648923825
:1062C000BD0474E814A0D69918D860F366E57A6B1B
:1062D0008405B0E2022294CE90CB40288DD1593271
:1062E0002260F55B9BC150FCE2DC860A0340E101C1
:1062F0002BA1470C5A1ABD529302CDC010B2419E39
:106300001AFF2001308C24A00510F814534012010C
:106310007B61247E94297A31CBB0FA5BC8F63ECCFF
:10632000F2A737DBFBBA29E9086BA65A7FCEAEF19C
:1063300040FCDF28EDD7FFB6A9F9FAA2623E3195FD
:1063400001B3F44521B921DB0977DB597492ECA044
:1063500084F9D2D33CE1E0CEDD0488843D93D34080
:10636000F9C6240501FED06EB044F3B85956637CDB
:10637000166773C52038B1FD1E33D5C5EED1846DC7
:10638000FF18FF88F62640CBE3DE0A05AA66FDFF6C
:10639000DC028053B4202D19513088B4CB19301A47
:1063A000CFCA4080089010D3A624D31189D3F3C05C
:1063B000B5FB5AD1087D0DE7FCFDCE863AAFDA90E9
:1063C000FD2C4120F33D0AD6AF018BBAFC1AFDE942
:1063D00010E63250CE4635FBC758B830BA6FC235DA
:1063E00080108EEF3CA8FA79ED8E23B380B08C013B
:1063F000D72C2E6B6C5855B810625B2E81FC016255
:10640000FA756A50B52857F014D8C0E295FAF31B14
:106410000A16FF069D890989363450FEA67ACB3EBE
:10642000201D3119AFECEC38FF7476CCF3E31C6C13
:10643000D888FBCFD864034DFB778012F90A6661D8
:1064400039FF8FB66198FE76583072B2B9C81940DC
:10645000B408FB5ECCFA9E170EE79B2EFAA820D458
:10646000E1D3681C87B6EEB6E9DF7BE1F0FB43D5EC
:106470000BD6161422C8D998FB8BDB420916B24002
:106480002610D9B8FE9EBA5A356CA763CB62043F7A
:10649000DAC620F83005B7F635802DEA3234EDB192
:1064A0000C8E7AAE20CFEB2518E43040749545CEA3
:1064B000A6F7777B378004082F8DEB5B6A422015A7
:1064C000E66F68FCCACA21CD09047E1C10ECBFC36C
:1064D000EC06C4B42092B4E4DD3A51F581E1F9C789
:1064E000088AFC804AB9467CE1F940851CC5824295
:1064F000E6D85009E3E8ED4D6750F54070888169B2
:1065000009652925049FA0C6A8050F27402990707A
:1065100001788DDDBA06EB6F019FA390F8A0CA56F3
:10652000FF50425A2802042122C41100048D8680A3
:106530000DFE37C52841120984BBEDBFEEF2840879
:10654000EB3F51B00985C638FF68026E6008A6149B
:1065500000E63006046F500A46A5A04CA748FBAFE2
:10656000DF2D3ACAF884E9239D4B1BE9A3191CDFF0
:106570006920D0FF11E19BF8C6FB0CEFBF9CA8D7A8
:10658000CABE6FC4722EBEEC3AEEBF8108FE84A074
:1065900044DCA3044B87E670A8FEA310F775B68110
:1065A000C7CFF598E5DED68B7E9170B1B9F1AF5AC1
:1065B0006BF4311B145CA07BC7EC9F33318FBC3371
:1065C0004DB485CFF6CB50F9CB40BD44423DC3C559
:1065D00033CF0263BA3B5F7F649848A26502CE580E
:1065E0005A02B772EFD8FBC2D4770231E0FEDB204B
:1065F00004690589AD12FF4C746062C65656046B7F
:1066000066F98077918CAA791FE7EEFD62AFD835E5
:10661000E1FF99F035CEF370F8C6D2D008CECEE3C4
:10662000CC299D10663632D0FF6E6C62025D160179
:106630006498BBA6F7FC78FC19804B96041532B31E
:106640004CD863EC7F641DF3A13CB8C8336ABB909F
:10665000E04BB320737537CC51B5EE40840D5D50DF
:10666000FDDF769DC67F18439195CFCA80637BF38B
:10667000803130063BFC3F0106904D10046D626E88
:10668000D5247FF70626C0420205F8136144018134
:10669000DE340070FBC2BC97CFB3021A7A650C04DB
:1066A00041E9FB06C4F6039360EFE63137E8F826CC
:1066B000DD07DC1ECA77CC06C0837FFD413C67291D
:1066C00030C0B30229FC4F60F8100382012C7A0716
:1066D000E067B803789EE4019A30E2FE07E21042D8
:1066E000A28FC9E0AF742081C73004677F9DA001ED
:1066F000E8200446D3E4F40D0F2184800681D040C5
:10670000A660668C8098B390FD5009BC0220C0083A
:10671000F3C4236004ED1133F346F358D12010F392
:10672000C6AA7F29C0811924E61805A0C04C4AF2E8
:10673000C04685199020BF96E15612D3FD338807D5
:10674000FFF2201EC88378100FB9E2F3F13DF3C0C9
:10675000037936F3813C770FE5BD0C900425BDE04D
:10676000399703E481D3DC0132F387180940E677D7
:10677000F0FC296006F010A303F061F3D6BC61F3CE
:10678000C47CFC4979FDE0BF83D49930FA2DD3FD58
:106790008430BBFBBC50460440B7EDF5E70220F364
:1067A000232D6C9D8930F31985BCDC24E060DF0E5D
:1067B000451005E5B320B2B3F874660585BE9802AE
:1067C000BE08FF0121200484AD806380005027F3C0
:1067D0008031046DEB5C2257B79101168190120154
:1067E000FE98FA2128800422F098FC001369594190
:1067F00039F7040860FF8BD3993381AE35D3346504
:10680000B30CAAF686FF3798EBFDFC985DF3EE9883
:10681000840111BB17E077E9E6C0C083F960100C72
:106820008241F3DD06C1A442F3D9E201A3B3F0C66D
:106830007FAF9840F1986069E0982990B30400FD1B
:106840007D0898FD2C4800DB5ABA68687FEFB202D9
:1068500056FC209AA1ADB30A51B3A54CE7168ED8C9
:10686000FFCBC52857BC980540DE98CE880126EBA3
:10687000FF631510E32640ED5800FFCE42F94018A3
:10688000210B20F33BE6B00035B305CC0882B2C043
:106890006998ED976197786B3F04445008445B7B9F
:1068A000FF1206F1FFE0812C80FC07B1001EC4023C
:1068B000F3B00B6001F305AFB050C583F3B5E6E864
:1068C000B14DB6E1D7D29840D3FF2F98346BF5B5D0
:1068D00019FE983CADFF8481C173062C73B166D656
:1068E000A120F3D66A6666F998DF8C7F6C0A30CEF9
:1068F000651C09FD5328EDC2E0CBF04B4BC54BE6C0
:1069000069DB9EB35F1B99808713E0EF448128F514
:106910009840AEFC60A020D0FF9F2965C60042824F
:106920002CCD866500504CDFF324D9DD01A319FF7F
:1069300026AF9099563742ECF1412080043526C0AD
:10694000FF56100912019090797628F9299BFC8056
:10695000531F3CB395D744C7309FE9EB98808D0512
:106960003930D0E7FBE041F707202C26CCDFFA8353
:10697000EB4C3038B35AE07330800364FA98842CBF
:106980005805E9983CF9C0FF285D6F9B1175445389
:10699000B8C5ABF411F3C89C19A420670699BA8B4B
:1069A0008AF80A212D85DE982910E90C77F2282231
:1069B000FCD5718020C08BC25EFAFE0A46C120F76A
:1069C0008B61108CC482090D9AB3D780118C98F01A
:1069D0005845D0175791BBB97BFA1362DD2208FDE9
:1069E0006A28FE78B2FA19F20016C0DC830FA453AD
:1069F000F3F00E1EC802E6F3412C1B34B35DE0EA4F
:106A00009880F3786F4998320CC6BF58D1981037E8
:106A1000FD84F8F2B3CF3CE503F830CD3F664BAFD1
:106A2000D698409E98462684EAC67FF341B9F9532A
:106A3000310326C146C051B3E3F3C530625A62A0A8
:106A400002FE33A3E028B480F69858206FD3447E2A
:106A5000B350F92048048024118292C9F97FFDD3F4
:106A60000809F348806A661DB7A7C822E09006FFB0
:106A7000D1481A4020602101FCA091041016C04E9C
:106A800042440069B32D5910D858FFE659D763B373
:106A90006982726640964680DC30DAC28017198CB3
:106AA0009808FEA3FAED37C84C61F52C08B7C67FED
:106AB0006AB3A28444F25840B478CB0C8216F2C870
:106AC00051B3F3DE9806F9571F6BA2012CF59CC356
:106AD000C8037EC2876FB649CD6602907217C0BFE9
:106AE0007D51CD0814DF48A64CC8A06437F3EAD224
:106AF000FB8E80170902C29F24469360122CCE821F
:106B000049F326C173F3118BF34C9B82E60834667C
:106B1000EF141FB3F6AFA0EB5F02484B8F5575081B
:106B2000B576EC8302121DF8607BA505F05C30653C
:106B30007998FE8B40E6D9DB96FF410C9003F080FC
:106B400002C4DE0118D35F8939D34083F3A107A3C0
:106B5000DFA0FD6605668979E5C6E625E79803E0CE
:106B600046E0BE9846D3BF8DD389F8E01006019D5C
:106B700092C8E05FF3B6E37F112F1926E0A1F84C2D
:106B800059C3B9C8E328FB10E28508661222BE8803
:106B90000F118C21C1448483102277821CF62102BC
:106BA0008404C2B3EED11831CD100486182291129C
:106BB0005721373034017A9840B5EF2038861404D5
:106BC00076F829E6A66FAD980243B3CD814706A1BA
:106BD00060E1DB5DE098090C83351F11C07D172D46
:106BE0004A0173C80FB480C8C8AFCDC84290B36F14
:106BF000E498FAA10726C0AD1AAD50AF2A80521012
:106C000010702E03F798A8F82C6BB7A937068102ED
:106C1000FDC6FE48779BC0E6C814D5B38A9241B042
:106C2000962C4095D2ECD163EBA0F15288B6136A52
:106C30009D4AF85AFD941110F5169AC804D0FD36F5
:106C400080BA62DD01A3AD6211B09FB5499595F997
:106C5000C918FB9160F6E249C808D2F540FCFB0C6C
:106C60004CCD2028D8FD714AF9C8ACC0EDC80F64DE
:106C700073C8D0AC0392C8E646CED896B50CA5C66C
:106C8000F02F3C791003E4AF2663B540065702A20B
:106C90008B62C324CB38FAF0232BC8CCA5DC8AC87E
:106CA000F3B37EA128F803BFC0853DEA7998B94EB9
:106CB000784EED6619FF7C58FCECC82C90BCAFC830
:106CC000357ED3FB73B34C9C78E02364E2FA8028D2
:106CD000DF4196C880B34EB1FA2067DE90F64202DB
:106CE000AC04C2C8816B90C8ED6333C80AB5023CDE
:106CF00018ABFF2F2918988840A6E00157B206303C
:106D00002BC59F23442C240806EC0400FA738C3511
:106D1000C166F21856FE98BF0C9A304220F5986270
:106D2000E3F35CFF7FD6A069C884580C6DAD10C03A
:106D300003A65AC8E5921BEB9F19E298E32BBD9876
:106D40002847F37998FCEA9B2CEFFBF6E5E3E58D09
:106D5000C7FA62134CC6C88979B31AC8E815BF666A
:106D6000DA9804884CA728C69062CD6BCF13E09FB9
:106D7000E004167BF2FF8051B3D5283F82A3601454
:106D8000048424F304C9F398AFF3E10C825102C4E4
:106D90007C9875900818AF2540208845A5B0000460
:106DA000DE989921AD45A40EF9D78F3DCDC80BA92A
:106DB000F37A9879B8508C46FF6B981C90CBA575E8
:106DC0009379D7BEFA9820FF789803E201247DA832
:106DD000FB80939DC8048297C530EB7E085519044B
:106DE00091E798AEF781CB2E27C898F3776651FDCF
:106DF000E5E2AEEDE38CB6E3FFA3F9E66F59A04000
:106E00005E980DDE989B60EC81F3C8228448F1B354
:106E1000F30BD8F8234B4186C7C118FF0363600CFE
:106E200020843130FE06C6C01802418078F38C21E0
:106E30004056106797985720AB98D8F65F209E98D9
:106E400097909A723064172C84019B0442FC13E3E0
:106E5000317D5A0705FA9802DBD4982146785DB84F
:106E6000BAEC204D3830BEEC70E350FDB2813CE00E
:106E7000D75EAF02E00138EE145D4EF3BB0E2CC8B6
:106E8000DFB67EF09804FDF3EB40012CD7302BD316
:106E90008D303F5290D7FA0C79CB20112826E7A0ED
:106EA0000814465004A489F3409E40F34102480B65
:106EB0006DB7E3D5AF49713039F9445108F7EB2488
:106EC0000485E9215B93BF68E05270D0FD944C8F3C
:106ED00002769E54804CD3A1FF4A094BF247FB65D2
:106EE00012E130DB4569CACA81F75E10C0187F869F
:106EF00098306928B560FD90E23F05F0801EC80318
:106F0000CC79205381FFF307F24006C0027833F3B7
:106F100068E608627C305E98F781781007FB98F18C
:106F20000069E7987330A8FC938009A5C25F125AE4
:106F3000FC3753417AE52092C861F3CE3766F29868
:106F400051FA8266FE98B7C0E4F228FCB3FA804595
:106F50003001FCC0049802136053C009E73042A618
:106F6000F314109B03F38C232CC8A2B324FF7601E7
:106F7000EBB38488C0985AC1703027733098F838C2
:106F8000FB310614C206AF635AA5817A98826789DD
:106F900061F301842CF3D6652004D722C8BB9C1072
:106FA000443480328647F377233090760468F8398A
:106FB000E69877EB7E818D9BCEE96946C18056606D
:106FC0006BB996FC9B9A38EAE0E585037AD2C0EE6D
:106FD000CC17E0E88454F346E62DE7982FFD03FD37
:106FE000CCF11BEE7330F8FB5EF69989C22453FF97
:106FF000900812412248048AE240112493B8F38198
:10700000AF2235DC5AB310B5B28889E798E4A0F313
:10701000E6410421B3405F7F0383607F1730337DF7
:107020008005A60630EF185DB6ECDE98060385F302
:1070300086797EE6B4DAA729F664C01D7F7F90606A
:10704000D1044CF0167B8AF2DBF66C412870F1FB20
:10705000E097BDA5F1801EC097EA9883F498E8ED0B
:10706000E610073BFE90B403FCCD28576B3F20028F
:107070003F7078100FE281B70CCAC8E5302C126659
:10708000F010D38F3DEB51B696FD150846C4234949
:107090007BB3D0026A196DC7300BE0448C9F9E69A8
:1070A00030A0FDC00237B348FB3B8C84BB29D24BD8
:1070B000142A6ED30A5BA6057562AAB384F2FA6B32
:1070C000D3A3606803BBBFB358B420E1309ACBB8F8
:1070D000FEF11A33FF56B30436D3DB20FFE96FDB32
:1070E000FD6701F36602B4B121B6D380FCC68C956E
:1070F000FF314BC7D980FF2C63469371B38E3B3968
:10710000FBF81409CC667DFFD1B0FA88B4C9231905
:107110005337F64D02EDF660FE8E1B4499B346B12F
:1071200060D316EDF389FD8D19B5FEF6638DD39806
:10713000FF8F8B1BD0533375604190E968420DA3DC
:10714000F3D0FF6C06639E4A018CF9E3BBE988F932
:107150006BB6711B9BFF8E775D30FFC383BC3D50C8
:1071600088B0FFB3D6A8424F9F41FBC7405FB9F23A
:10717000F228B2FBFD2828677D118CFD6D9FF2ADD2
:10718000CFBA17C2BF5A0510A8BF40E359F68DE623
:10719000E0FFB2F680C9F2B33C63CF0B3FAE35E3FC
:1071A000BEFC47B4DF74E02084FAA108D737A7817A
:1071B000E660FBC06ADA730398116A83470C2CFB04
:1071C00005EE4913A0CEFDCE0614E5801A0C290E5B
:1071D000301DA095B3B2AFA20A192A280F2078BBA0
:1071E000FCC62AFC190D440B79C22FD69D607B1B6F
:1071F0004017327E84B47F95622045284008E130F4
:107200005404AFCF8482FBC8089FFBE20770F802EA
:1072100018FD3E808F7EB220F1FD416CBCAFFDA316
:1072200049336EB32D0C784DA1024DC58480E1D455
:10723000406DEAD808F0F19B70FD53D91331BAD3F1
:1072400053FEA2C9EE9F90FAC9E0FF2DFCA3DB8C90
:10725000F26FADBED6AD04BED1D8B0FA7DDDB5803B
:10726000409066B0FBC7AC2BFFDAF02037E6F8FBA6
:107270009B26693D8FAC1901638962CAFD61626713
:1072800086DFCF1E33F733A938B0FDC39692842929
:10729000BABE08E57D0A85FF8D67F51DB7B659585A
:1072A000F99C6511A7C2DC64F07EB1FC3E6C7E8067
:1072B0000243F5CA28D44AF9ECF8FD022E586910A9
:1072C000BBF0A8FD61811B193E41644B2463A90EEC
:1072D0007D4B205C106565AE78980608E5FF967BCF
:1072E00023F6FB1B36B388FE09666627F6F2EAF63C
:1072F000845A57026B1D080163D90BB0B8E3F67FBF
:10730000086988717D9E66B140EE318D77D108980D
:10731000FB6FCDD50481BF01C86DC6BB1679376E32
:107320004940C5D63B0233F6B17F13684EF8FA6385
:107330007FAD78D6A3D8FCB2A12343EF13FDC403DD
:1073400036E868FAC6042CB32CDB6BF6C60252ABE7
:10735000A0C35FB332B292F5F8B0863D17DE10409D
:10736000439511F9C64C534110FF6A4BB7045A8F2D
:107370000165959213B1402168EBB848DD0BC5E378
:10738000F7E855FB4E32E3FB6F4228F38CC57528B6
:107390001022E72F15B9CD98D28188F74BF3F8C9A1
:1073A000E6CEF8088AE890B206690A920572661479
:1073B0000CB2D1F00D929FE458C68A0575958004F1
:1073C000EE7C60197466F398EEC050CAC16F242D2C
:1073D000A5059B40198455696076090868E306BCD9
:1073E0000C031182D8890187BCCFA03FE107FCA420
:1073F00010184202EA3EA00501991AC1885D934225
:107400006AFCBFF6F20B68FE37E6982BD4942E2D5B
:107410001014F5417569F0CC7608A0A6B3FF7A3652
:10742000ED02A2B2E0C5FFCC04BB90F7D582920773
:10743000A6811D100EE6F698FE006CBCBC33F3135B
:1074400063F31DF5934099FD1D6CFC8A2CD8056CE7
:10745000BACA0A32C9DCE3FA067169E690E85C5000
:107460000D17FC289EFCBF4725FA7142DFCFC025CF
:10747000340DF88F1934FCDE67F2B140D91288B1AF
:10748000FD8DB1B673B037B61720EB0BFF63E90A79
:107490003DDD2062DCAFD808F8D65845DEF6A820DE
:1074A000017736C148FC3BB61C3CE1B180FD31158B
:1074B000BFD96B10E411107BCCF8FD625B17B150A3
:1074C000FCD82B4092EFE8C53D4B2862EBBA0C1973
:1074D000D7A150FD0862FEEA63E6FF732B30FFC0C0
:1074E0008031174411131A21DE630896BF89B3FB5C
:1074F00082642936F314773F7AA03134862010FF56
:107500000482440A080C8D20F480008222D3F343C5
:10751000600801C651EB844080CD4B38D2CE5B8BE6
:1075200020ED809C279201BBBAF1DCF26BCAA5105A
:107530003BEA30C8E09A36E8C8835FE5EC60E08952
:1075400029B4419CA47FCB40B899D306C0577ECCC8
:10755000A8210CF748FF2044FE7589B8708B8E6E09
:1075600041E90CFC9464159AB322FDE820C4224042
:107570000DFF87E62C0228B044288728202143D815
:107580000309597BA408F7C8316101E76004B11110
:10759000300346C029EEF302EC8C841140B378B678
:1075A0002226C11B5808F4AC2CB00D42C46B5B22E0
:1075B00061482690390AC019AC81FE01F0200ED036
:1075C00003797F8EE0413C8807F1FC2006C8007AF1
:1075D000100EE0012DCE1EB4ED3C80077FD31EC0FF
:1075E000001A100FD06080F3CCCC16B07822169918
:1075F0000C70FCB65FCD3D931808831106F37CF93F
:10760000E8F30481E31A332BBBC381993096C2E0BF
:107610001805F9E6843F47621C26C64CD3C8F925F5
:10762000ABED23BFCA135FF644EC41C14098FE099D
:1076300060444C0088A0CFEA6678324640844850C7
:1076400001EE0AF67311166786981C64215EA13D4F
:10765000A5D8FA907B9814118F02613E9D012130CC
:10766000043E84103C02D7B192CDC8B524B7AD9882
:107670002452F83271B51724FE12518A4814892118
:10768000BD984089128A10F5CF812DA0AD0854FB1A
:10769000FE98366B08FB825F0A971862E875B3EEB6
:1076A0007BBB065A42712E19261DB170C5A7A98849
:1076B000C0F8E02919F9207F8EA58841301E06C147
:1076C000ED2241E4F8652CF2B3FD9FC294E9B9C004
:1076D000791869CE99B0FB2C022F708EB9B2D741C0
:1076E0008CB610D71E4180025EAB6ACAB20A354B17
:1076F00012A7104E201101F4448488282E00D7C808
:1077000011EEA58C773573FE14666142B3A30B8E20
:1077100020725384B08652F3AC61362C485962CC47
:10772000B38521C6C202268B9960378808049A3037
:10773000E8C4FF7A886040A680192091D3D598B01C
:10774000ECEF83583F0360013CDC8805F316784D6D
:10775000F3C82C887A980C7FE0F08006400239DD6F
:107760000007EA9803F39899D30FA0E60710FA2BC5
:10777000B6D5D241FBB903FDE6306995C8E098A5BE
:10778000420E19EDDC99F510020420F2ADE0922EC4
:1077900031D33A3F3A6945C6D1E9FC8011C9C07777
:1077A0003FFA6141488105B2E41016C4F33901265D
:1077B0009B80DCB010E116C0E124C0024221886049
:1077C000BA4464C046699A84F222FFEDB04090CC7E
:1077D000FD20E28263B102CA6110EBF0DBEBD399CA
:1077E00042DF03E9080401E60667F17F7230D478CE
:1077F000705010097A4D22F498269FCAD1206481D6
:10780000411310052E9FF0980EE1D91D6566F50312
:1078100065C80CAD8AE4CB46FA8BB42025D00C04A5
:107820003759C0F9ABB320D673839E4C00B66EE5D2
:107830002D817DE388EA6441D48B6B820CAE2A4EA5
:10784000D278CA800173B350F9D0120282FDBFF61C
:107850006F49F320FD988C79EA9FFD7F222035DA6D
:107860001109DA1804F2982F82409868FF8C0809F1
:107870003120E8FA800839025FE3281001AFCDCA51
:1078800080040475FE30194010A84803CDD77A0350
:1078900008109922D1286812601680043C30D7ACB9
:1078A000C1690510A60823667CA0F9E0410C3F04DD
:1078B000F4000EEFC80278F2B8E25061110338FB11
:1078C0000F20011C3B505172242D30E5E006442668
:1078D000BF0830C6B019803F913C0818F984810177
:1078E00010D002C01B069C3001794EF9ABEC0C4263
:1078F0000143863080205139A4A682C7775653D1E0
:107900003A927B5E2058BFFAF43AC0FADC0B62D39D
:107910002D110FB3F598309D9EDE8049A004A23F43
:107920008208090307442C77C2D1A5C289417E256C
:10793000817F9902D0F9204804A780A30A0108CFCB
:10794000610CD331A488767EC8610B088440BB0EDD
:107950000666FECC3101D3CC40C0B248F0D0120D47
:10796000202734F3C208E20243037C124D22003583
:10797000DE84F9871D19192432B1A101458C671FD6
:1079800066EBAAC47E158046A27CC7BA771BBB975C
:1079900028BFFF6909E488769DE9C723FADA03BEA8
:1079A0007CBD98106CA26FF47706BBF0ED295B9755
:1079B00004F05F11AD4E0DE7F868552D260869DE1D
:1079C000DE3A2BC2884DF3171301041A80CFF298C8
:1079D0004D8A3075C02E5652577428E15814DC0871
:1079E000AC0CFA5F3012D9FFFF984204C09B243ED2
:1079F000838433ED0F26C122100CF5F5120C40C61E
:107A00006668669A92E0241C7AD56011129067A38A
:107A1000400C1805C8204222C29EB3A1FA60BCA542
:107A20009F461ED00378405B56EB1CA007D5B8508C
:107A3000BC760F22D9E608BBE381653CFCA001348B
:107A4000800648AEE000034AAABDE130F3CC400F07
:107A50001B1CDF56FEC43DF09508E3D7FE69FCFE13
:107A60008B778B95D63F4D158BEDCF6BF823486602
:107A70006B5F414BAFF37F701905E4B10806C74453
:107A8000969902D309395BE2AF10D79F84DBC6FE1B
:107A90001D14D5F88AEB093104750E90BBB60A8225
:107AA000264D12F398DD54BB2C7E5270FB10844D92
:107AB00049C2226DA0A7FF6A9010C1181261EB2382
:107AC000280CDB9814013B9E7F4424121070750231
:107AD00043E20A6981211916DC0108C6F804452031
:107AE00010B01A48FDF2DFCB1B3830B6DFBC98B6B9
:107AF0008ED421D8195EB1FA64F12B17F397B8CE62
:107B00006BB9D8F803BE0EB2C8D82E64F3F1F49561
:107B10003968EB98105F375240AB859B2030A2C389
:107B2000B4BBC858FDD899BF5238AEFDAF9D22985E
:107B30006539A36D0533C628F713EB210201562FD3
:107B4000A2A04D5B205E904FA22F0481088821B82F
:107B50003D40D8BB84C8CB187FF6113601FAFD949E
:107B6000117A984041F0AF8B68C5804573570BBAC6
:107B70009820402CE5CA229BE99804B39822392426
:107B800053084E44764CC85FC025FA7F04CEBB0133
:107B9000B07AAEFAE0412C6EEFD5C803E7303C90E6
:107BA00005FBF0401E5000F9302C2CC2CF9FCCE0DA
:107BB0001C8007F126D38458FF1E98F3F2201EBCC8
:107BC000E2BA61BB549896FB1399D55E982FFB3BA4
:107BD000F3E0BF08864266A0CEEE1640203E06C106
:107BE000FEC80E40C36903C168E97E778E19FE0E98
:107BF000C04682988EDFD7FE30041694C41996AF23
:107C0000406D98A0808DBCFE998BEED97D090396BE
:107C10009744B50FC6EC022021594A3DE608F0FC16
:107C2000DD0FAC46FFC840A00814212850F03400F6
:107C30001012A7027F4841CB0121E6338B84F23C2E
:107C400031D344DFC40249EE082485F698429232CB
:107C50007F2948044D20083411DC88FDDC2CE2EF3C
:107C60006E9801612E70B1FE0CA32C6073A2CBF450
:107C7000E8C26E4C2C37FA17285322AFD3E9CCD97F
:107C8000C0768E62B30C644B18845319765E301044
:107C900005A27833BF194D087D4341D0100CF73E43
:107CA00090FE084235801695D990D07EFB503089E1
:107CB000DE830B602444B930046A656FFA2A2826F3
:107CC000D650010A60FE84C028EF094404C8275C2E
:107CD0008C8884FAA6A1FA8051DA836373210106A5
:107CE0001480FCED0846414098EB0860445B62203C
:107CF00009391B11F9310220C022D33FE010880856
:107D00000530384D0418E7A26001C58C080B0AF94C
:107D1000C2FCE0AE042F30D76902AEC564CCC8B057
:107D2000091E3BBB78C59843986702E0073C880171
:107D3000AFF43B988D107830BD987AD6200B41C8AF
:107D4000EB60FC84EBD98F30F5E604726A088FD6BD
:107D5000E5500C7E0490D7EBD42D237F82314789E8
:107D60009DE0D5EBCA51441DEBBA200CDE98D750EC
:107D7000FB90A5E0F596100B62DDF40502DE8B5E4C
:107D80003EEC70212C9CDAC844BFB384043012A0AE
:107D9000400B10055E0E7FBA981040427AE96104EC
:107DA0000C81EF8438FC209E40BD26C0184CBB0AD5
:107DB0002175DD0F09C6DE8B5EB8D7212807306636
:107DC00067C8A131F92492401204E076C4E4441952
:107DD00068D60A49B86C0D2030FD0218FA9BE69867
:107DE000A7C2ADBA40F5151468DF59557F19307B2D
:107DF0003649DC6219017FDF70FCD68001EE09E4B0
:107E000002DEEDAFF1B97FD0034EC260813059ABD5
:107E1000DDB142FB18BC6B035F4A9832CBDAB62F58
:107E2000CDE97FF0FDBF01EE061024E16B5105D9CD
:107E300001B811B32781808236A2226FBFE6822863
:107E40002022A0109802CE42B52492C8CD837E7F16
:107E5000092260048C84289C34F2F88077641B6BC0
:107E600098B4AF02D2AFF2B8C8BB51603088408B33
:107E7000B337DFE59011312224CAC42887E73020C8
:107E800088045F7FE2C402484C61B34CC0CDB0EEC1
:107E900068F860F298E73DC48378FC1007E8413C3D
:107EA000883DF20067E83810D70F241930AAFFE0A8
:107EB000F078AECBA87CF8C8F02016C07038F40378
:107EC00028190BFE8409DE985FEB6DD564CB501842
:107ED000BCB8BAFE59E1FD189B31EDC06E2230FAF4
:107EE000F2ABEA8EF36BBF281085F905778A78EE3E
:107EF000D2BFDC1D01EB2E26C0350E03F2F9E033B4
:107F00003DB4059E80BA44841899D3014C155DB1E7
:107F10005B99F09108710AA981797083FF84C0147C
:107F200082E0C4181A7F63600C01803130E709C613
:107F3000C0F361035EB836193473B4A001DD04895F
:107F4000CE30400B2C250DDE98834408C71A40C75D
:107F50004801E2200486DD78E098899CA06BF797C1
:107F6000F90BFA1D366840FDFE6671C32C4F028C7A
:107F700093C8C6B640783B4AFEE163C4A6F4F60354
:107F8000706BFBC8BB2407E0B2C8EF2F753398C9EC
:107F9000FF32B045F997A8F9987D2F37A662103BBC
:107FA0006D08F0FB9CEB421028F502800812B252DB
:107FB000462711249832EE08A23C10B3D67415BAA5
:107FC0009171DB1410460B4400D04C01CB1B148480
:107FD000EA1C24C2E102B0FD51112B295101F980A4
:107FE0000E0886E6F31800EB30BB41A03033722E4A
:107FF00056E35FD6C00374444C69348BC41FF5212B
:1080000064228CCFEA04B0FFE0AC41EBF5F04030E5
:10801000C879C5EBE0810C20F56B1ED020BB7860E1
:10802000013C206D7D530368F883681C7FB998C0BC
:10803000033816AF68817FF0EE2006D0E503E27EBC
:10804000DF80BA64856D93AFA098813F9270086617
:10805000577A363B80058BBBD0565E8801B810CA74
:10806000F69802C4E5E96017E67417B8FEB370C06D
:10807000FE9A136224448809BD98C205EAA6206DC1
:10808000D412044D215AB38421FAC2F298E130E3AC
:10809000BB818930A609D62262D30FB930F82CFCF7
:1080A00069FF046F962E10ABFFE8EB32A86416B898
:1080B000CA5975C6F372AC22C6D8D3B8F90C121DD2
:1080C000FF98FF2C8D1993C6D13839ECF2F91412B0
:1080D0001866C8FB08A0EFB29E74FF8F9331F93287
:1080E0006637FA0573806CD344F319A3FEBE30EBF8
:1080F000F0A44F31D13380CDE0F44BD4D3F6F3016B
:10810000FE23047FAFCCB17F5F58B901BF9797962C
:1081100009987B81FF7A4BFFF3CE34B7C77C5BCFE6
:1081200020CD11A5CD7DCC9AB9B2024CDFF3F5FF7D
:10813000A202661E71EB6BEB98FDFFC20244D000F9
:1081400079901800B751BCD5AEEC9B08B5E841A3B7
:10815000F970FD62AB3908163F20EC07F3D3D898CD
:1081600018F90CDF36E4F8046CC5620196B2B3422C
:108170008F4FDE7A60FFD4F5CBD329639F11E6AE33
:108180002090D0D303BEEC216D0DB9C57E32FBF13A
:1081900081C45AFC456CA7998BF063CCAE43D74A97
:1081A00081A8C908B8F0234D7BC7400074F0D0887F
:1081B000FDA86720A0C4C1C2C01920BBA13E2902EE
:1081C0009006421F406100B309C768ED1001C880E6
:1081D00082E01818A0B80C2D72B888EDC79841D667
:1081E000010AB3E058FCF3117B4704704DD4170823
:1081F000EB6D30BFC1480F419067BF662120060E6E
:10820000C48887B007F340288442F254D080D06EEF
:10821000342830FEE0B6F0FEDED4B308FCF359AEED
:10822000FFCC6DFBB602BE581B5FB783EF6090FBBF
:10823000126EDA71AEBE48E1D2964022B6C740084F
:10824000860266E082AE40FF96C31E4FB64058FAE3
:108250002BE2B1D88CC563D67D01C2BF6EDFF16859
:1082600040EDFFBAD18DE88849F3C57C46B8DFD828
:1082700093DB6DFE781EE28632B30C7E578F3F375C
:1082800094E9BDB96284DB02AE38B1B133B5703761
:108290000CEF2F2C2FAAB3C43A9F5F9FF8BDFB4D64
:1082A000F6CD818DBFAC18607EDC1CF15A1E79DAE8
:1082B000E50FE30FAFFC61476C1D0493B263232FFE
:1082C000BB3F58F81657B58098B4AAFF20C596E86A
:1082D000FDBE85611AFF01C71DE1A8F902BF0B7E33
:1082E000436E307EB1FF406E2BB8FF01230A3EC7BC
:1082F000DF2CC1F1D3ACD9B8FCBD6DB504112FE5AD
:10830000585F9D2ED8FD99F60C51F6B21114D4A0E9
:10831000C7F54E20A3F85A3F4545F3866DFF58FB3D
:108320008B7DAA8E187C9EB6A05CFF59DB878B6183
:10833000982D6610468C122CC8024BDB7C98FC1AD8
:10834000582604BF81ECB20832DE5AF3FA3148C431
:10835000CC196B227F3431782687C0FAD7CB066DD3
:10836000557EB4E08C8CCF37713F6877E21099C4AA
:10837000FBE236FE602DBB490808BA55CDFEC42885
:10838000FFF3993BE0C923516327C5D0F1843D1029
:10839000DE28FECD627BFF652C990267D67D40CD3D
:1083A000A1B0FE8C2D3C02FCD803C8078CDF61799C
:1083B0005B50F6C710F3E3D6B3FB576CB1084FD64A
:1083C000ED08E668E7A2FD59B14BBB0660F9B39230
:1083D000CF6CCB82B2C9CFC92EB31D6979FFE70537
:1083E000C6A86EB693E8FDC26FC7F0D82E3FF35112
:1083F000A104D1E6E2E2A3DD2E804B6E042FB66924
:1084000020800453A678FCB640CC7B06DFCB01ADC0
:108410009B02603CF112401948D9C620AFB340809E
:10842000059098A1F730D90A11E5F8A0A8A2800E0E
:108430005494E1A609BC28A10FF8FB80950473931E
:10844000BFFCA248CC038EECCF18D0F7F08C97DAA3
:10845000E49EBA92457AFF7D61105484144E28043C
:10846000694E77F2E08906D090729E0206C23F8084
:1084700069700B98FA3BEA1088CF80324AFEF98C7B
:10848000A2B3B3BFDA117FEC8284FF47DC8059B31B
:10849000B6FF51E944B02FC81016C4EF29DDF8200B
:1084A00080651D6D2DFEDA43FDD2415D78057E9F0E
:1084B00040502C190610F6C841C23DF6C814DCFF26
:1084C0002BC78AFD729C6863BBC87E8D625A099D6A
:1084D000ACAF8884062FD5B1E67F29BD1DA0FB8AED
:1084E000E64E80C7B289C4776B60BFF8EC982AD398
:1084F000FFF83DCC355651EA78B3845C46611B4F9A
:1085000090FE6DE6AEFCEFD80240B25F10FD35FB89
:10851000EB262B4FFBEAB34BBAFDF715FB0919CD40
:108520003F08989528A7AA9B9568FB4EB467DB2265
:10853000B9F5882CF3A3731616219570DAEE64381A
:10854000FA59EA03CD2A8001897AA010CE59014058
:108550008D95E0F81FEDD68124C22CDA6B56A04031
:10856000776CF1F05737C804ACC180D46D08B7E818
:108570005BA101FDE0A881E0CD90FCA7DF40C01821
:108580003F1263600C0180AE31FA15C21840081624
:10859000F3D227952EF396C0485D769B01F405949F
:1085A000F31AB2AC82DB95067898B0F49CFFCFE565
:1085B000E71890F67EB56206F49C248378DDD8E057
:1085C000C9A8F08D71F38A34B42C1061D10680BD36
:1085D0006D6F7EF5309FF60358200C60AF815F4BC6
:1085E000FAE95A10DF8B6008A101F5AB42F3F951AB
:1085F000F31019F1FFB4BD02754069A762E9DA3ED4
:10860000F1220180900470EB98FE7211B0CB3E080D
:1086100018EFC1DD4CF350300226DF5877E4E38CCD
:10862000E6B3F349B4ED08E346C0188323FE6104C2
:108630002C8045302240F39B58B050B84E7FD31861
:10864000FCE0413C88FF05F0801EC4037A40930F94
:1086500019F3079BF4F3D092F3E2E6CEF1EED338B0
:10866000BD07F11F1EC0037810CA0FE4D366F340A4
:108670001E5948BE2431D3E440FC80ADE766C220D9
:10868000538360E9100C88F3062E1768F3400CE65C
:10869000CE251AED08ECE0036032E0F2D335EA1B98
:1086A00066F9FBBAAA53ED03136024EEE074F304F9
:1086B0009BD3F304FCFACF25B2A0D279F226B30DF6
:1086C000D33460F3C22D5F1720EF6D1048F9308D61
:1086D0000406071200BF42E6ACEA8409F37FFA877A
:1086E000012120D37B55FF24ABF83204379E107D47
:1086F00067FE980124F3D01C76BE9813BCFA6FA6CF
:108700002F6F68C740CDDDF30C6AF8DB0640786B4D
:1087100036ABCEC171DCF7EBD8F980E999E618B435
:1087200004EC0F30B5F3F4640CD99130CEB386412C
:10873000086BAF21D878021A120BCE86F3D21ED75F
:10874000C798D370FE044D04822ED981224BB8CB3A
:1087500023FB880C4B65447EDAE60AB5F80510C4A5
:10876000ED19593D6E328580109821CF8447D39BF7
:10877000FFCE9480E446C429E2FE0B60010C889190
:10878000103C46E4895800F33D04847DE19AB3FC33
:108790008580301002C20F19039360028C579687B0
:1087A000F8DA8214FC32E7D329FFBD3CA0F507F0CC
:1087B0002016D0BED79798A0B8F2681EC4F396A32F
:1087C0002C7E9780B2A505F0266490789092F1C631
:1087D000550512AF8E98D3E8FC5F67E3C566037F4B
:1087E000ABA511C1E53FCFB83366BCE63BBC6BD748
:1087F000C59813E6F34266F1BBB131020649F4E0D5
:10880000A2CA020CACF378F93361018A7A4B346066
:10881000E0D0431A99A3B34CF144F37901FE984C8C
:10882000A690FD0E84040144A2E7404810EA8C2182
:10883000153C721204824487F320EC840581E266C1
:108840002FD33578F498A067ADF3407D9832E806D1
:10885000C8F9DE5E19A4656D4AFE0363BA612C593E
:10886000ECEEC8FB40F5A5C0272583F20F02775A2E
:10887000F97464EC81E001FDB506EED9169085DD52
:10888000D4ECD340160D0359DE98FA3C0858FB2867
:10889000F79C1601249702759764170857C3C35BAA
:1088A00036CB482FB649BDF729F3FC880B10209032
:1088B00001BC01FA02B0FE8041F0A59F40180401FE
:1088C00061C70280FE21300A16444008635421F635
:1088D0000C0210FDFEB5127EF88949302006C19FBA
:1088E000D30361114C90FB21B00046017FA53235C6
:1088F000FFDEA516B0EF2EC55D5DE8C95DB0397726
:108900009748AC8B3DED5C16E0E095F0E0C230E0BE
:108910009BF390077F1198F37870FF840BC8B266C1
:10892000216677AB9831AF334E6620F38130CECDE0
:108930004089AF2B1004CD9800D3B71D663990F84D
:1089400078B2BFF68710CD0C045E9864720305CF31
:108950005AB3887A9858DF8830B3DFDC980150FE2C
:1089600081F79035F442FC38091208214BDEC5022C
:10897000421803476559E81D9DA220A0B2D585DEA7
:10898000817B98808977DB72F8984E10F8F9C5BC26
:10899000B5D3EC4FDFD97F099DF166FB73D8FD7A23
:1089A0005824E7586010036B9A081E348E33B1F4D4
:1089B000AFF52B04F9C85F453DDAC08016AF08302B
:1089C000E635FAC71F705DB5B5FDE2C0D9D0BF442A
:1089D00028A0B0CDFD32211C06B87F9143661DE66C
:1089E000E99824F60935E69AFCAF020840C100F583
:1089F00098048320FF3F49300926A2C262D7622C27
:108A000082052CF3DFFE7F0810300426C178B109FF
:108A10002360128C7C76C626014FF732B0FD78C5F4
:108A20005DF02065F579A5FE984BF3D0BCB8B2AEE9
:108A3000CEFF32E2013D2FE043D379EB0F68008C8B
:108A4000039F1D98ACF884DC974293065F66E6C5E9
:108A50005E59E8AD19844193E7C569CF95E0983731
:108A600091FB66F546ECBCC8E013F3BB580CA2F3CF
:108A7000C6FB5235B382D9093419C844B34C64F3E8
:108A80003048FBEE9031046BA24244F1A18C82FA93
:108A9000848810C018F3C5F92384099DCF9B050174
:108AA000C0108011FF1498C2902DF3FC98765BD013
:108AB000FD7FCB01003CF45988BE7D628AFFD0E97E
:108AC00017FABF0726C82C0F579EF7F9F420FA06AD
:108AD0000FEFDAEC049A19A0ABC42F6DB6B1403C8D
:108AE0009866AC0CF3C1034E6B306481DC7AF82CD1
:108AF00050234601427DE58504F67608023BB955D0
:108B000081051F31E7391A39F998FC1D6BE598E7A3
:108B10004321CE884208E10140A01F4F02FE1410FD
:108B2000F8B00826C12281F98B601480FF73B50864
:108B3000989900F311F4B745D56220B7475C9F3090
:108B4000E1C2281801C00360EE0C8085CBC87F9D70
:108B500032B9C8F8714A91CE5D68012CB2E82E1E78
:108B6000C4E5F3E865F59BE497D3D788053503D0D2
:108B700083CE03E2013C59F35E98F7D8FC8041FABA
:108B80009808FF65E5824084BE67E8820E9008671A
:108B90006915D9D5B620F3782C667DF3E9FD8009F7
:108BA000FD2B2BE03BD54C80F9031429F3954C5E4B
:108BB0007E67FE2A29ECDAD5027A98A0CCE2307ED4
:108BC000B9F92050040A26005E4048A00895CD84DB
:108BD000C223EBE0F35881223080EC01FD2EAF2E52
:108BE000323FF6913005ED09B3C8853E26060AB03E
:108BF000FBE0DC0CB1CCF36326FF4F163DD90FBF71
:108C0000FB77C3CCD707C0ADA50372E88946F360F4
:108C1000FD200C82810880A79798DB0A25CF2C5372
:108C2000AF33300BE4F610599B7F35300468ACCF7E
:108C300018FA87308843C0D2904A082250B840B50D
:108C4000BFF3E8FAB5CDEEFE04025EF51A5FD694E6
:108C5000A066E8F948880450200D1CF79F0889F9A0
:108C600078A565AA6205CFC84C8451D73008B5B83D
:108C700098009FC804848030D98A0280B33E51B0E6
:108C80001046C1BD780B8B608CFB0220B0400623E0
:108C90008430BA5DFB60919BC840B2F5BC98BCB80B
:108CA000B2C84BD0F3651924BF2F302CE530C479FE
:108CB000982DB03CB830B840BD6B70CAFB8449FBFE
:108CC000415CDFC888EAB8802DF36D588440FCE52C
:108CD0005B886815B746E1304A5EB80592669C200D
:108CE000191131B5F5CDC840FE982EB95FD312E603
:108CF0006B86BBFA0B00D606025FC8EA988CE4F7D5
:108D000011B2D3B930FA5EA5F51006C4189FD5612B
:108D10000C0180F2313086409EEC88BB178405310F
:108D20005FED65F464047DBFC6F47E68B54BA3C6F1
:108D30005C98C88A099D1088FA89F1302D77100C4B
:108D400075CEDA64049B55E833065FEF10FCE2B29F
:108D5000F9ACF2BB70B53738DDD1401864BB3A02CC
:108D6000D3AF6FDB3A44F664082E072051DDE012E2
:108D7000A0C607D7C298BB3DC8F0FB287FF71611E5
:108D8000E4080245E5217D22500409DB6B051774D8
:108D9000B66D040AABBB14644B50E8D34011145EAB
:108DA000B33FC28020C242889240FA99BFA9C0ACAA
:108DB000F8CAD502F34C6203E42C15F1F1F54240F8
:108DC000CEBD20214CEEB37C0B34F3A0B0B7C0F184
:108DD00002180113BE412C001031BC42D3FA320CF0
:108DE00042F3A1F3C888AE072E3D3B5DDE983DA05F
:108DF00005B0B9238359BB4BF32035B36073D3F46B
:108E0000205C109818E062A9F3147F8A98F36DE64D
:108E100008F873C880DD1804EAC588C9C8669720B9
:108E200066E7BB8130019DF199D79FC5959BB71A25
:108E3000F9B8B166DC30DF88FA93954698777F24DD
:108E4000408011301206DAC008F003D9F301C5B32F
:108E5000CB3D26FC9879F40D8085F3DF4604E59838
:108E6000A4C0B9DDB0FFE3A5F142FE180363600CB6
:108E70008C8192F320F33E046363E38C0530B306E8
:108E80009DB305014078A5A3DE6FBC91DFCB988729
:108E9000B5D340FB62D9C8B1402E58260AC1E53A85
:108EA000FFA0FCC0F2A56B581C804EBCE8177806EA
:108EB000221218F3668E0ECC38D8D95B3569AF7B99
:108EC000A5B040AD0499466960E95BF6BF4029C88A
:108ED000F33830E2FF2B48D3A51857445C57C24102
:108EE00002E9040A4039519980CB41AB2CE6DDEE12
:108EF000A12890F1A5B85A8069E99840A2AC88846D
:108F0000C253F3D3C8F9730506C0BF282EAC2CCAD0
:108F1000CEE824D52060BF465146F3ABB301555E81
:108F2000107F6CC044FF9804A360124C80495E8B94
:108F30006BFE328C814977D370FC7BA507F15C3DD9
:108F4000EB037A402BD5CF98CEBB7A109DF33C2013
:108F500007A2BB90D72926E088DF07B4C003D65B01
:108F6000C8F998FFDF3A7FFE80DB43B95D10DF036D
:108F700062E5C5B4963B6B91E86D0516BBD0AD5E5E
:108F80008841A0D33B835CB5C8DB96DDF31008FBBA
:108F900033FA4100C0581213B93D886AA60F236105
:108FA000344688E6B50435216BB384113CD5C4281A
:108FB0001A3B0B332FC876B30238F935A6297F1A2E
:108FC0007DEDF8FD4B5F7D66F79278FA5F886FABB9
:108FD0008F0138F3CE51AC22B595E6D362D38858D1
:108FE00066243BFF98FF241A33668CD17139C988F7
:108FF000FAC1206658B35ACF478483732173B500F2
:1090000046DD19F82CEB6444CF37B42FE0B77D0070
:109010000AD5D3C888F9C11FEBCCEC7F5132026A64
:10902000C363860C6F367588FEE60E78C2B189532D
:1090300097166CA770FD708DDDAE0863C75D9866EE
:1090400025F94B854AD210311C9FCBFCB0662BEF23
:109050006959F3105F5C019FB20CD3D8A5CD6CF3B6
:1090600020B02DED6401126DC704CEFB17DD56C094
:10907000FC02C1F7A42064B2FA7F278162A3B3D7B0
:1090800010651C09709408A6EB09309DE8FA11DE02
:1090900013262942416ADCA514A9062CE805F4B47C
:1090A00040F9EC28018041C5E1064021F4822814F2
:1090B00061D19802B66D463052E0FD7770208F9BEB
:1090C0005E8801151C0B605F23F63011EDB280FA4B
:1090D0006D3CFC29624D0F522802C872A01109FC98
:1090E000AD082D336C13FA1293231FE5BE808C1349
:1090F000E5B968FD971246AFB808F1235E64FA1629
:1091000080C482B3B45BFB119FECF2CC0499C6908F
:10911000FDAD659CA025BC0197F37973A331D908F7
:10912000625C65592E0193C2FFFFCEE3F23C348CA2
:109130009557A718D328FF63FE0A7154849CC3B0C7
:10914000B89BB4B180CF63CFDC08FE4080121042E0
:1091500026F004880011B61044E8F321570219F3F1
:10916000BFE9B840ACCAF967F36FC36BD328B3FC4F
:109170007EECC3A6FFD8FBC2D5CF08B95AE5FCE602
:10918000EA47F67978FE11E96FE6C93E48D8D8FD7E
:10919000FEDB6D98ECFFF67FA8FC162C1A8069E3C5
:1091A0009080FFC326B28240C91B48ED2045E8F0FD
:1091B000842BB30827EFC4CB8553BA3FB6AAF86710
:1091C000D832FF1BC11AB5F58699DD58E0FA97D65B
:1091D000EB12EAA906D51A246C85D0800956D9B3BA
:1091E000FE86323EFF61A7EC7F08FF31E5FED8D74F
:1091F000D0CEAC62027BEC69EE6CB038FD283FBC8F
:109200008C0F6BFA9DB8FEDDFB20A6DEEEFBBB40AB
:109210008DF6F6E1CF59B7037FA45AB665360480C0
:10922000FF3DF64527EBE88075E240B9F39FE24B3E
:1092300047C3A6FF98FEC383C43F7830B8FD0C2710
:10924000DB1DD62F10EBBB0110FDF7FDE6F035DB83
:10925000B12063CB1F2E919664C63C6F2DB0CE9F7C
:10926000FB07381CFD9191E80D19FC9FE49CD24D41
:10927000300A1089389B208010B90204C66AD4B520
:1092800011CA2E569680689A90B31A6FE8205068DB
:10929000830805DB12D95FB342E3C6D3C81487F055
:1092A000CB29B30DC0A0A128DD0B3F0182288E057C
:1092B000E1ABE9F0142001242109BBBDFE600814D4
:1092C000177A520B440147D142E0EC71FC8801F659
:1092D000102667CFC0893181049122B853B3A448C6
:1092E0000F2880D25504F6023D41C955B0C4B7FCE1
:1092F000F9A571637F0363FE749A087EF817B47A48
:109300009FF4BB831043D29661427F0C69E381A333
:10931000FC8A61AB4576ED9184341019CBD1FC30D9
:1093200038A75D78D65E50F3D9E104FF1546CE2DFF
:10933000A3A0D62CB8FC6ADD192062DEDCB0088759
:109340007E7F80C0FB04D0F6C77C95588D42FFD845
:10935000F9FB69DB680112D689C8FECFDDEC88868F
:10936000F96AD830FFFE971D986047A4FE79D9FFAF
:10937000801F352CF783F3CCA7D2BA3FE0CC0EADDB
:109380005993102BE27016E37DFCB0C7B9CC806610
:109390007B2158FF63FCA246D672B102CB5BB5407D
:1093A00076ECC0C7F696F3BB13596180EB57FE18F5
:1093B0003CE3C1C6F211CE5954FD7F33B1016319AC
:1093C000749144B5FDEC8A1807E965B7DF22B696BB
:1093D000F9DCC2010A17883133F312F3421B630828
:1093E00032DC22E6CF7CA901848010D2F0D3482061
:1093F00049F30921E1900BC022CE124448022CEF20
:10940000EC02A8FEFE47A502630F2A800111102F6F
:10941000C0F6B8400CEE3C06F39A630C025BC050F9
:10942000ABB3C03C530BE001CFD007E516C0835966
:10943000436268B12116069CA81D12AEB8F0FF70F9
:109440002C400F60263CF6F8BBC111F4200244808A
:10945000E7C9240490F320A9B8935C1BE6621F6E51
:109460009422702991410FB9881005BAA4C26623CD
:10947000E0330C204034FFB0FF8005300246C0E7E7
:1094800008188193800A24E6F3ADDEFE39106004EB
:109490002C801159F3CC1949B09F9A2699080B20BA
:1094A000FF244C8441B0104001F348080920578044
:1094B0008584300B48FAFFE0413C8807F1201EE725
:1094C000040238BAE081893C04E6F080100C792669
:1094D0000FE859E6DFC481E02CE08805F4781EC06F
:1094E00083787F0760013C801630E7F31810033E55
:1094F000C6380860F9E4F006C093183B66200A9C61
:10950000F305C040E0660362510CF39C1B7BD3C2A1
:1095100020F318040360E08468E040F36820E676F6
:109520007568FDFD2331F204CA26DC29C06E0840AF
:10953000136EE00C33E69EB385300826BFEC00E6E0
:109540000B610AD34593A608B301E8A32002B366D2
:1095500025506631BCC564BE42B1E1E10128A2F3E9
:10956000F39882A44422B6845ABB24A7F8328E8290
:1095700020CC92408408CDBB218684CD914050649C
:10958000A6E0848904D668DB96E8B6BCBDF3FF3F4D
:10959000988DCAFD900C6AF8DB868174F1CEB00418
:1095A000193108CBEF74A8FDE09F414606C1201891
:1095B000A5C4BC0B6FD288055E985966325380E60D
:1095C0000335B306C0010940641E975E6B594A77A4
:1095D00083884879412766FF24B510C9D7FA9911C5
:1095E0006288F9AF02129868F985EA06C6BE4BF8A0
:1095F000050829DD3B18C21152F922848801306028
:109600008BC003D30013338004F2B00811FDC6FFF2
:1096100085CE8848EF0AD205F3FF63981320EB2C20
:1096200080ECC1D7B3850931C906201F865F60D0A1
:109630002C021B85C8582E8627B37211FEE0CF81FD
:109640002CBDB0001634EF1846CE412C88F040BD3A
:10965000985A030F649601F37F9798A2A5B2E01E73
:10966000C4461AC00B60F92C9001F020F3C90339ED
:10967000B10C9E3C70FB8041D3C0E60760AF100880
:1096800098BC982AF19833B10C0F1AE68081FAB988
:10969000F26BF9DD655F9FBD08F303B440F67E38D9
:1096A000FF1709B020FC16C4825810011C02049058
:1096B000ECF3B4C04240E761410C4FB12067EC0BC2
:1096C000E3CD42C4685804F8431983A046CDC228AC
:1096D000B353731A8029D730052D30083D9948F9C6
:1096E000000A210128F3BB90CB98A735F380312CD9
:1096F000E6FE783086802412C070400248738008ED
:10970000E290473BFB9801A05E98CB28FFF33B2CEF
:10971000EC6F9230104657DCAF2D22DBFD28E6BD02
:10972000E5FA0A41D3D94CC002B6990BED0823776C
:109730001D30F9D1E0E6623C30C82006E0ABE89A83
:10974000ABF18CF37AE882BB17E896F9EE9B4945BA
:1097500099F9CC48FD779C98D8132410B304BC4BDE
:10976000BBE702FC2244041A09A1B8277E62F1C4B7
:109770005702223084130BF76084FF0C300F46C170
:109780002818CD8402A20AC9F305DC5E98EB6110AB
:109790004C8C23ED669F9045ED26BC4B1E21610449
:1097A0008CD73C31BD3E1018089070304C09B02D5C
:1097B00018FADC6AF707F0001EF99800F369C83060
:1097C000781A0FE2E323375516E4CE3007F280BD56
:1097D000A538E6400FE8D3A02AE123D3C51840CE30
:1097E000E0411988FF5B1C7130791717F382982EBE
:1097F00066E050368125CF302006C240779FA5C550
:1098000010F4ECF382831BFD98C8A3FB53C1B3FA99
:10981000015022043FF3EECC08B3B803CECE748AD5
:109820008557ED0F30221321247BB310C8D70818B9
:109830007F84022C90910409CB38FBCC5C9FC868D4
:1098400044010810B505E730600C81F6028430064B
:1098500077BF9811069224122233D30AAF8C71D3AA
:10986000B7A7B62C0F1441D954FDA6D1679998CD4E
:10987000668101E589E29EFAD7EF1E1BF20C02BF5A
:1098800061F8B640CBC8B830EEB49BE73078100C26
:1098900085423C671698EBA010CB9825ABE365D5C5
:1098A000DD6134F3C8E7A40F0C084AFEEB814CD706
:1098B000C8011C6CF369C93009F45EB8098867C82F
:1098C00002A2F84004582009C15E0D6891D2CA3541
:1098D0002304FA72495674FDFFB00926C124988406
:1098E0005E495CCA33F305371430E804C6DB8451A3
:1098F000F5D0B7BD42821130047B984008E1432087
:109900000CD388D310C05E1F9E03D8808149446663
:10991000D9FAE01E98AE403730F698200B96E61044
:1099200077283040D3BC9857E090E2D3FE83F120F3
:1099300006C4831819F35C03CB08F8F02BD6980102
:10994000FE98DD1004F6F976DF9697C8723D41EC7B
:10995000B5D5E123D369DC17B9FAB6FAC8C89421A2
:10996000C001F9C85C305EC55B1C66F7FE8485FFEC
:10997000304026C08298101301AE4C6EE681EBFD9C
:10998000648427AE0CB0FB9F20DE88101122C00239
:10999000459B6A052886F36C430D63FCB5621E98EF
:1099A000E209029015759FC848244980C51134EE1C
:1099B00000C422C89BB00C43823459B30BD6601844
:1099C000F59884B7D17F331026FFCDC30CF331C592
:1099D000F3B0DC5A77A4D0F92DF7B3C8786D90C8EE
:1099E0003B16C003FF3D3CDA8801F8EF06A0112BBF
:1099F0000DEE9FF06581BB46BCF8F0FCBB3CD098F7
:109A00003D7D28F904881742CD12EE6011C1F37034
:109A100075CCE18085409BF36F055EDB6C0165C80A
:109A2000FFBFFC181150200280D796341230CD139E
:109A30004C466609E0F352FD5B45E7C8810AA38006
:109A4000F3B830B97311E50C81459F9DCCCA313014
:109A5000A29A86FEEC010CB5D712922086884EA7FA
:109A6000A6840908D958F8536564C89BF3D530BD5E
:109A700098790054396C21B780C9C806FE05D440D6
:109A80001EC8013A1E0762BED69B631ED0F9300184
:109A900039B2D8FBF06F90C89F94C8267F1F30CB97
:109AA00043046FB76BCBC8FC986DE941F635BC98A1
:109AB000D5F6C196F8DFD9C82D4633C8A0F74808B7
:109AC00040236F1E8030B3024566F87030D7F99896
:109AD000F299242CD2908908E258E30321AE44E0A5
:109AE00006F7F0FE2050E7C81843D7000AAE9840AA
:109AF000CDC80867C80A14E58C2140D19AB3BB20B1
:109B0000D7A5946864F12B2180113110469FE3B6EC
:109B100059224576A6624F9A6DAC2D406736C83102
:109B2000C3A596888E015E0C9203400C8A8092ED4C
:109B3000FDE0EF2D1360E90260560B45BB7F97985F
:109B4000973E97C51A6BEDFEB752A8B306FF254B9B
:109B50008FE4669B07FF523B40D381745928F99DDF
:109B60007EE54905C5DF9159C859FC77F8F2210215
:109B7000443611865DE2ABBEB70942CE4018E822FA
:109B80008252C9260634424C444390D86661B06B79
:109B900062FE35D50AD3FEF902106B0A86F3668899
:109BA000B930201E40E3F33919058F02220DCD286C
:109BB000200C7E32B2116A9928F1A3663367096AD4
:109BC000B8B6FCCFC8080258B440CAC87383C08373
:109BD0005846642DF3806EB7F7980C88059A94D395
:109BE000C8F6EF0B68053CFCC759BB8B10E09D81A4
:109BF000C678FBAE56C8772E602065C8AFA5982002
:109C0000C9C6F3C622BF2AC0888135D342EA98026A
:109C10000665D0E0FCBFBB9B7071FF5CD7C8986D38
:109C2000640232C81D44D9C8FE412C8405011002CB
:109C3000CCDD488834FC2640C0C01032972CF5EDAE
:109C4000E37E4224EF78983208B8FE2B3FE2C6C08C
:109C500082404827BAE88831E3308610E9484295C7
:109C6000211382315CFB68FF6BC528FF5D3480C027
:109C70009077F0344824A7A4519002F71480124141
:109C80006A4B2022E3DA1BCBC8756E12AB5E818073
:109C90007126DE78BF226856FBD4DCBBD110EB9076
:109CA000FE4039E207E0F37E56C889DC50DF59C830
:109CB0005ED3EDE00130966640C7A4EEF080BDC0F3
:109CC00042CB2003B3738CC281F3C8FB28DE8AE841
:109CD0002011241C98D42010B20AF633B2C8BEF466
:109CE0008D06CD53BECCEF01981A1165950966AB70
:109CF000D0C28240D023029228325A98FEEB9EBBFB
:109D00002B58BB844E62D9CA665A62AD2318AFACD9
:109D100010ECCE9A971941D910AEFD58046160013C
:109D20008C7ABB06EE2EF105034473E2A8FC4F26A5
:109D30009007F240BF1EEBD5C5D294168340C89B56
:109D40000FF32C3BE5B1BD723D90BA842F38400F24
:109D50008B623C5C301706D0E2037A10FFE8402C9F
:109D600008D0F98459E264E7C831086DC430C9B13C
:109D7000100EBF17EBBF4F60E330FF7210DF088398
:109D8000FFB2301040F95E920316C2DF0019F2CC28
:109D90000C70F302A02B0929C8B345D9B020FDB13E
:109DA00039DA2542F883A020BC24B34AB6CCD67851
:109DB00042407DAC210250FA6D29DE98D71843FE4F
:109DC0005E0908103186B92252F80063600C817B6D
:109DD00084803965203C8D821054537122FE092401
:109DE0000D2004148027C122402EDBE48888EEA7D2
:109DF000A4FE33DC3CAAB29D3BCCF8478E305DB06C
:109E0000C0D7A1F491201F96BBFBBDF7FFC001385E
:109E100076171C0602106050404938368859C8969B
:109E200070D34EEDDC125AF805811C23190608AFD9
:109E30008FADCC01EFF0774274AD202DBCC03FFE5A
:109E4000FE4804894011288216016857FCEF160964
:109E5000F498A05E122024DF85D33EBF9398EDC016
:109E600010831A51D12008666632C297370B8EB222
:109E7000E6FBF98F81D2C3D262FD32517898DDC5FD
:109E800014DFFF048405302CA6CCFA2E880930207C
:109E9000DF5F98040B24D3F7F8660A460418F40130
:109EA000B3AF8007AED9AFFF3FA5C69846181D0ACD
:109EB00065D5DE98AC14D7C82057A45A972DBB900F
:109EC000753268E2013D80D77080985EA5AC62E78C
:109ED0008E0730F3C48359C8CE6080C690F981A044
:109EE0002DE4961888660B0AB86ABECC4E66D6205A
:109EF000048BF3EFBF6DFFD0024566D3AF9F9895FB
:109F0000A8A7AFF23060E4E4310DA1FA79A5FBE334
:109F10002BE6EED4C9884D071040FA2360042C903C
:109F200004A6D7AD3952B38419062444BF2D01C20B
:109F3000648441C6B40608B333DA84D3084B99FA73
:109F400014D32C3768EBF0C216FFBCFDFEDA5510B7
:109F500066D301D8F30B50F30CD5AC229ED36EF32D
:109F60005ED5C070F96090FFEC98FF246493596F40
:109F7000DDB1636DD3EBF891E567CB1D08F61802F0
:109F8000EB6C0C9BFFC9FE3CED8593B28A97D11117
:109F9000BA73FAFA65762F08D37B27E0FE113651A3
:109FA00016D1F322B16DD6A2C617FA7E3BF3F1FBB0
:109FB0002BE03F3630B5CBF0CC0C7628FA4F1EA004
:109FC00023669B1C99B0CBEB2072E334776C19D8D5
:109FD000FFF3D61BF23AD9FC797FD8C78A91C0DF4C
:109FE000EF7F331A7E77CBD06445EFB3AB124029B5
:109FF0002DD10166A68FA81942B7A701DEA1209F27
:10A0000071F3EEF84480103B72F3373C58A412CB46
:10A010004278FD621EE761BBFF88FE611FD9D46BE9
:10A020002D0437CD76D6F4D8CD6608881A3296C17D
:10A03000D831B2FF80BBD7405EEC868248FCDA2B79
:10A040006C509FED7EE0FFCB91E1DABDBA414BD37E
:10A05000011513B3E4B182B5102D74BC0783977A50
:10A06000017A6568DB93CA06660AAD6027452F143E
:10A07000C0048E50B75D816203B4B505F090A13481
:10A08000C023C84911BB80F80928A120141508BEB7
:10A09000DE450105372070F86A23FE700481C01286
:10A0A0001403046069845E77560CCBB2FD3CB2B7F2
:10A0B00057FEC0C01FFC0562B0102C82DC7481C248
:10A0C000CC14E206895431DA38FA81B39448451940
:10A0D00061179241CF044DB8D384A79BCAF4602D79
:10A0E000B8F997EB4D02BA9456505FFCEB6C101127
:10A0F000CC2E880D8120FD8664288741F39BAA1011
:10A10000483BCD988CA4EF5C88803F63BE6CB1C0A7
:10A110005D37AFF3A6115EBC20BA6E1C0DB7018D82
:10A1200096601924D262EBFF04634CFA85C84A8713
:10A1300021E6FE15FF10CBF537208CAD0E08C2B31B
:10A140002F3B4EE37623B9279B75DCFE2F76F84034
:10A15000DE796BC60B2463631B2BB1189D59154028
:10A16000C61D6AB801CEFEE5D0FCC44CBA7DA02065
:10A17000629B7C5E9867AC4120D3BF3076FF8AD16A
:10A18000C4D6B320FA626ACF44B6F46DA6DA29B415
:10A1900001B36AF5DD8014D686CD9650FA1BE69899
:10A1A000A6FF99E505A0C658471EA5863BF930FDD8
:10A1B000255A41610FED7808B647FF33561BE6D8A4
:10A1C000F80A3F050267B10D0810D94B92A8256621
:10A1D0001063E71A93961608A06EF1B728C83CAB37
:10A1E0004C154BF69D1135D7B0915FBF88F6D4FD65
:10A1F000C7FC538CEF231D4DFFF8F98DFEE004CF13
:10A2000031E8AF6C2ED8FB77ACB522DD8504B166A2
:10A210009419B0018F3B790140104C5D2082800180
:10A22000B6B0FC678B13F3552084FCC846A6BED598
:10A23000B4080A51F392156C4478FC5481CF3783EB
:10A24000DBA56E96F59577B66450FF24B6634BEEAA
:10A2500010CD477C8DF3E47F6C1B48FE28E304702F
:10A260001916047F9FD79D2938FD8C6993BF9A7476
:10A27000ADE7040CBFCE3FB36F5BFAA0D414F9B0C6
:10A2800078B1FF806FF6B47FB678B8FBEA6F013C17
:10A29000FD4E1355328288E94875687AE50281D609
:10A2A000323201DF362EFBDFF2B98497027AE620E4
:10A2B000BCD52B757F089668F1102002045AF6640D
:10A2C00040ECB6CA1A99CD88F9CCD27B63D050073E
:10A2D0000A033EF5A080010228DAC0506DB0464066
:10A2E00016B310FF6D5E65F015B00124CFBC5002AF
:10A2F000E03FAB2801250094FF16082006410B40E3
:10A30000255FC2D130FCAC08DBBF1251C94F3DF212
:10A310005232C0F42D28024EBB2C62BE93A429A950
:10A3200080E0D3020E1FAF182F0160CF3205E81175
:10A330005680C34A42831D40E0465200FB215A200A
:10A34000F875D101B7CB1A3663BA30B3883F2A23E8
:10A35000925384EC05041EFCE46DBE410858F9DC00
:10A360003CBEF9BECC2B45E081DFBF627E305F7F13
:10A370001F041047309CC0EF7FA9CE40FB68D7FB7D
:10A3800030D1BA8CA1C6B65B2665198A6EE101C4CC
:10A39000BA659BEBDCF827F6084012F996B0D616A2
:10A3A00086BBED8C10F81F22C6C7A693DADE69F6CD
:10A3B000017EEDEB80BEE0DCB3FFBCC8F76C19FD9D
:10A3C000CF5B37049983FD59B22094F9026D668EF4
:10A3D000CCB390FDC54C35C3BB3DE540794B9BDD0F
:10A3E00028E8FF8E75179EE8B30116A10453446850
:10A3F000FF61B6EC040143B7178899B3ABAF011105
:10A40000D570108AEA5D50C96CF498FCDFB39DCD1D
:10A410007FB28B8FF631F79D6C8FA8FF4B8DE4CC0C
:10A42000EE7CFF837F389DF60D38F9C716C11022E8
:10A43000E5631BB1B2FF3ED53AEBBD4DB3B5B2EA11
:10A44000CD59A6018690E396662277444A708381AF
:10A45000BE885C4E5DEF26DFE04176EF04807FE84A
:10A46000BA44C322EA1338F9E4E5818C28FC487425
:10A47000777AE0F8762F8500EB97CE60F6220C9B7A
:10A48000BD1040BA9F05019EB441E0CAE0E5E982F3
:10A4900004E07AE08047F326F47601FCB07B486E56
:10A4A000FF98FFF43B30B626E18B7169D708754001
:10A4B0008F7D2F9CE0C0B0FDE7148002B30A40C33B
:10A4C0000128D005A0F30B50C0F36004B040126720
:10A4D000EFE016C0C00258FE0BE0012C8005B06D05
:10A4E000F34094F307F35AC6FFFFA00C9481325354
:10A4F00006FECC4019280365C07EF329335006CAF6
:10A5000043F3FD8364200DAA419DDF1B0C900132B3
:10A51000FF4006C804192003643BF3A44155F3131C
:10A520003EF3140190FCFF3B0080FFFFFFFFFFFFA5
:10A53000FFFFFFFFFFFFFFFFFFFFFFFFFFFFFFFF2B
:10A54000FFFFFFFFFFFFFFFFFFFFFFFFFFFFFFFF1B
:10A55000FFFFFFFFFFFFFFFFFFFFFFFFFFFFFFFF0B
:10A56000FFFFFFFFFFFFFFFFFFFFFFFFFFFFFFFFFB
:10DFF0005465737426536572766963656B97E72B76
:10E00000F89404B7087011F00C940000FF246AE53E
:10E0100011E0E12E1FEFD12E11E2612E10E1712EE1
:10E020001FE111BDF1BCC798BF9A1FEF1DBF10E1E2
:10E030001EBFE0E0F0EEEBBEC0E0D0E187D631F7E6
:10E040009F9B1EC07ED6E1F41E9818E111BDFFCF44
:10E0500024D6E4E9FFEE23D674D661F4E8EAFFEEB5
:10E060001ED618D6E6E9FEEE1AD6E0EFFFEDD7D5BC
:10E0700011D6EACF01E305D6ECEAFFEE10D655D66D
:10E0800019E718BB17E817BB18E01093610010934D
:10E09000620011E01EB910E71DB9F092980015E07A
:10E0A00010939900F0929B001EE010939D0018E0E1
:10E0B00010939A00E0ECFFEEF2D5E8E8FEEEEFD523
:10E0C000E0EFFFEFACD5E9D5E6E9FEEEE8D5992023
:10E0D00021F0EAE7FEEEE3D503C0E0EFFFED9FD5C8
:10E0E000DCD5009BFECF05E021D6EEEDFEEED7D5C8
:10E0F0001091610011601093610013E91A95F1F716
:10E10000109161001E7F10936100019BFECFE0EF34
:10E11000F0EFEBBEC0E0D1E010E8079009920FB835
:10E12000779BFECFD150DF70DF5F52E04FEF110FD2
:10E1300011F41791111F441FD0F75A9549F402E0CA
:10E14000459580F00395439551F053E04FE3EFCFB1
:10E150005A95B1F4469508F35395E9CF040F54E06E
:10E160004FEFE5CF4395D1F45395479558F1551F9F
:10E17000110F11F41791111FC0F7050F56E0D7CFFB
:10E180005A9511F401E00BC05A9529F4439531F4E6
:10E1900055E04FE1CCCF5A9509F7542F47915A9546
:10E1A000A42FB52FAC0FBD1FB150BF70BF5F0D9036
:10E1B00009920FB8779BFECFD150DF70DF5F0A95D1
:10E1C00099F7B3CF029BFECF10E51DB91E9AC79AEF
:10E1D00064D5E0E0FFEE63D5E2E1FFEE60D5F092BA
:10E1E000B406C09A10E24ED3C0982FEFEAE4FEEED8
:10E1F0005ED32A9511F401E044C20130B9F7E0E59D
:10E20000FEEE55D380E002FF80E414E03BD307E745
:10E210003ED312E037D309E630D3082F2ED33ED3B6
:10E22000002341F002FFF3CF01E431D30023E1F7F3
:10E230007ED30AC07CD3882339F00AE728D31CD3C5
:10E240000093B40615E01ED3A0E0B0E0C0E0D0E03B
:10E2500084D377D311F003E014C2EEEB00810F7783
:10E26000A1F4E2EC0081013051F0043041F00630BD
:10E2700031F00B3021F00C3011F00E3031F4E6ECBF
:10E28000A191B191C191D0812CC0E0E0F4E035853D
:10E2900000E010E028E037950F1D2A95E1F70A9578
:10E2A00009F4139506850784002909F0139503895D
:10E2B0000488002909F4139500A101A0002902A0F7
:10E2C000002903A0002909F413950589007F003F68
:10E2D00009F41395143009F0BECFC0E0D0E0A0E0FF
:10E2E000B0E0A0938D06B0938E06C0938F06D093B6
:10E2F000900633D326D309F0AECFE0E0F4E00385F7
:10E300000023D1F704850230B9F7C0E0D0E0A68938
:10E31000B7890B2F0A2B21F4A4A1B5A1C6A1D7A1BF
:10E32000A0938706B0938806C0938906D0938A0687
:10E33000C0E0D0E0A389B4890B2F0A2B21F4A0A15F
:10E34000B1A1C2A1D3A1A0939506B0939606C093A4
:10E350009706D0939806A189B289C0E0D0E00B2F30
:10E360000A2B19F000E1D4D3ED01DF93CF9300899C
:10E3700000938106A0918706B0918806C091890616
:10E38000D0918A060A95AA0FBB1FCC1FDD1F0A95E4
:10E39000D1F78F919F91D5D38685978580938B06F2
:10E3A00090938C06CED3A0939106B0939206C0931F
:10E3B0009306D0939406E5E9F6E0ADD3E0E0F4E00F
:10E3C000058500938206A4D3A0939906B0939A067C
:10E3D000C0939B06D0939C0602E0DD2359F4CC2326
:10E3E00049F4A53FBD0530F401E01FE0A53FB107AA
:10E3F00008F400E000938006A0E0B0E0C0E0D0E0C8
:10E40000002331F00A9521F0A4A5B5A5C6A5D7A58E
:10E41000A0938306B0938406C0938506D0938606A6
:10E42000A093A506B093A606C093A706D093A8060E
:10E43000AF93BF93CF93DF93A0918B06B0918C06DF
:10E44000C0E0D0E0EDE8F6E073D3A0939D06B09372
:10E450009E06C0939F06D093A006E7E8F6E068D337
:10E46000A093A106B093A206C093A306D093A406DE
:10E47000DF91CF91BF91AF9111E00A2E0B2A0C2AA8
:10E480000D2A39F01F93B7D2A4D21F9110F413951F
:10E49000F9CF1093A906C0E0D0E065D2C0E0D0E08B
:10E4A00006C02196B096F63011F45DD2B9F403851A
:10E4B00003FDF7CF04FDF5CF0081053E91F3002366
:10E4C00069F0EF93DF01ECE5FEEE0791002341F0E8
:10E4D0001D910117D1F3FB2FEF91E3CF04E0D1C0E1
:10E4E000FB2FEF91A28DB38DC489D589A093AB0684
:10E4F000B093AC06C093AD06D093AE06A48DB58D97
:10E50000C68DD78D0A2F0B2B0C2B0D2B09F440C079
:10E510008FEF91E016D3F3D21197CF09DF09009165
:10E5200082060A950A2303950093AF06009182069E
:10E53000EFD2A093B006B093B106C093B206D093C9
:10E54000B306F092AA060CD30093B606F092B50675
:10E55000C0E0D2E0A0E0B6E09924AA2440E8099106
:10E560000D9301D44A95D9F79A2891F479D181F481
:10E57000A0E4BB24CC2428E03D91369550F08D2CAE
:10E58000FCD3E9F1C79AB5FEC7982A95B1F7F3CF46
:10E5900077C0AF93BF933F932F930091B5060023AD
:10E5A00061F4C0E8D2E0A0E0B1E0442709910D9306
:10E5B0004A95E1F7E092B5061BC0C0E8D3E0A0E0C1
:10E5C000B1E040E809910D934A95E1F70091B60654
:10E5D0000023F1F2C5D20093B606F092B506C0E072
:10E5E000D2E0A0E8B1E040E809910D934A95E1F747
:10E5F0002F913F91BF91AF918824BFD319F6BB24CF
:10E60000CC2428E03D91369528F001D4C1F12A951B
:10E61000D1F7F7CFAF93BF933F932F930091B506F8
:10E62000002361F4C0E8D2E0A0E0B1E04427099102
:10E630000D934A95E1F7E092B5061BC0C0E8D3E020
:10E64000A0E0B1E040E809910D934A95E1F700910F
:10E65000B6060023A9F084D20093B606F092B50660
:10E66000C0E0D2E0A0E8B1E040E809910D934A95FE
:10E67000E1F72F913F91BF91AF91B2D341F6E8CC32
:10E6800005E00093B506C09A1FEF1DBF10E11EBF45
:10E6900004D3EEE9FEEE03D301E3F3D20091B50615
:10E6A000013021F4EAEAFEEEFAD211C0023021F480
:10E6B000E0EBFEEEF4D212C0033021F4ECEBFEEE00
:10E6C000EED205C0043039F4E0ECFEEEE8D2E2ED23
:10E6D000FEEEE5D203C0E6ECFEEEE1D2E091B50637
:10E6E000C79A05E010D3C79805E020D3EA95C1F793
:10E6F00018E110939A00D1D2E0E0FFEED0D2EEE123
:10E70000FFEECDD214E11F9303E4C0E0D6E07CD04D
:10E710001F9119F41A95B9F795CC9A2891F008E150
:10E72000DAD2D9D2D8D2D7D2D6D2FFD2E8E6FFEE0B
:10E73000B6D2B3D201E3A5D2EEE6FFEEB0D2F5D267
:10E7400081CC8ED061F7A0E4BB24CC2428E03D919D
:10E75000369528F03DD3B9F02A95D1F7F7CFC0E030
:10E76000D1E006E051D021F4043049F005E1FACFC0
:10E7700006E04AD029F4043011F005E1FACF33C0A5
:10E780008824FBD249F7A0E4BB24CC2428E03D91A7
:10E79000369528F41DD331F02A95D1F7F7CF8D2C7B
:10E7A000ECD2D1F7BB24CC2428E03D91369528F05B
:10E7B0002ED3B1F02A95D1F7F7CFC0E0D1E006E033
:10E7C00023D021F4043049F005E1FACF06E01CD053
:10E7D00029F4043011F005E1FACF05C001D351F757
:10E7E00006E079D281D2043006E029F008E173D244
:10E7F00072D271D270D26FD298D2E8E6FFEE4FD2C9
:10E8000027CCC058DF0905E166D216E0C79A10FD93
:10E81000C79840E050E7E5E041505040E04021F427
:10E820001A95A1F70027089566D2B1F30430D9F301
:10E83000013091F7C79AB1FEC79856D255D29924A4
:10E84000AA2440E851D209938ED24A95D9F74CD2E6
:10E85000102F4AD20915A9F61A1599F69894089519
:10E86000E8E6FEEEEBBEA0E0B6E007911D910117D1
:10E8700011F40A31D1F708950FEF0FB9779BFECF4E
:10E880000FB108950FEFF9DF1A95E1F708950F938F
:10E8900012E0F8DF0F91F1DF0027EFDF0027EDDF57
:10E8A0000027EBDF0027E9DF0FEFE7DF08C012E00A
:10E8B000E9DF16E0EBBE0791E0DF1A95E1F710E221
:10E8C0000FEFDBDF0F3F11F41A95D1F70895C098D1
:10E8D000EF93FF930091B40606FD07C0AA0FBB1F7C
:10E8E000CC1FDC2FCB2FBA2FAA2715E0CBDF01E5F9
:10E8F000C4DF0D2FC2DF0C2FC0DF0B2FBEDF0A2FAE
:10E90000BCDF0FEFBADF8FEFDADF8A9571F00E3FD1
:10E91000D9F7FF91EF9180E092E0AEDF019301978C
:10E92000E1F714E0AFDFC09A089502E0AACE0BE74A
:10E93000AEDF0023E1F7E6E5FEEEB9DF0023D9F70D
:10E940000895EEEFF5E001910535008109F40A3AEA
:10E950000895E0E0F2E0BBDF0895E0E0F4E0B7DF27
:10E96000E0E0F4E00895CF93DF93DE01C0E0D0E073
:10E9700000E1CED0AF93009182060F93C9D00091F1
:10E98000A9060A950A1738F4CF91CF91DF91CF915C
:10E990000FEF00230895C091A706D091A8060A2F73
:10E9A0000023A091A506B091A60629F00F9323D0CD
:10E9B0000F910A95D9F781D00F900A940F910021F9
:10E9C000A00FBF1DCF1DDF1DC8DFDF91CF91002736
:10E9D00008951FE000918006002319F4A73FB107B6
:10E9E00008950A9519F4A73FBD050895A73FBD05F1
:10E9F000CD05D107089500918006002339F10A95CD
:10EA000079F0AA0FBB1FCC1FDD1F0A2FAB2FBC2F25
:10EA1000CD2FDD270AD03196C191D081DF700895C6
:10EA2000C0E0D0E00A2FAB2FBB270F93CF93DF932B
:10EA3000EDE9F6E07DD091DFDF91CF910F91E00F0E
:10EA4000FF1DE00FFF1DA191B0810895FD01EE0FA4
:10EA5000FF1FEA0FFB1FF695E7950A2FAF2FBB2785
:10EA6000CC27DD27A6950F93EF93FF93EDE9F6E012
:10EA70005FD0AF93BF9371DFBF91AF91DF91CF9123
:10EA8000D170EC0FFD1FC191F63031F4CF93C0E08F
:10EA9000D0E0119662DFCF910F91B081AC2FC0E032
:10EAA000D0E0069540F4B695A795B695A795B6958E
:10EAB000A795B695A795BF7008950D2F0C2B0B2B1E
:10EAC0000A2B59F4E1EAF6E0A0918706B091880696
:10EAD000C0918906D0918A062BC01297CF09DF0911
:10EAE0000091820604C0AA0FBB1FCC1FDD1F069534
:10EAF000D0F7EDE8F6E01CD0E1E9F6E019C0AB2F65
:10EB0000BC2FCD2FD0E001E0D695C795B795A7953E
:10EB10000795D0F7089501910A1BA02F01910B0BC7
:10EB2000B02F01910C0BC02F00810D0BD02F089539
:10EB30000191A00F0191B01F0191C01F0081D01F52
:10EB40000895A80FB91FCF1DDF1D0895D8DFE7E88E
:10EB5000F6E0E1DF0A2F007F0B2B0C2B0D2B089525
:10EB6000E0EBF6E001911191012B1191012B119134
:10EB7000012BE1F1A091AB06B091AC06C091AD06BE
:10EB8000D091AE069ADF0091AA06A00FBF1DCF1D3F
:10EB9000DF1DDFDEA091AB06B091AC06C091AD06E3
:10EBA000D091AE060091AA0603950093AA06109193
:10EBB00082061017C9F4F092AA061DDFA093AB06D7
:10EBC000B093AC06C093AD06D093AE06E0EBF6E092
:10EBD00000810150019300810F09019300810F0909
:10EBE000019300810F0901930FEF0895A091AB06E7
:10EBF000B091AC06C091AD06D091AE065EDF00913B
:10EC0000AA06A00FBF1DCF1DDF1DA3DE0091AA061F
:10EC100003950093AA061091AF06011B089502E325
:10EC200030D02CE00791002321F01AF054D02A951F
:10EC3000C9F700E250D0ECEFA791B7910A2F0F71FE
:10EC4000E1F01B2FAA0F111FAA0F111FAA0F111FEE
:10EC50001F7099F01D3088F42B2F26952F732930C3
:10EC600060F024D00EE237D0012F20D00EE233D056
:10EC700000E228D0022F1AD0B7FD0895E0E9FEEE99
:10EC80000EC00F930BE127D00BE525D00F911AD0C2
:10EC90000DE621C0EEE6FEEE02C0E0E7FEEEEBBEC2
:10ECA0000791002311F017D0FBCF0895005D07FFF7
:10ECB0000053085E06FF0851045F05FF0C500A5F11
:10ECC00004FF06500F93029501D00F910F700A3088
:10ECD00008F0095F005D1F9310919B0015FFFCCFAA
:10ECE00000939C001F91089500919B0007FFFCCFAB
:10ECF00000919C00089500919B0007FF03C00091C4
:10ED00009C0098940895FDB814E6169A1E9808D0B1
:10ED100016981E9A05D01A95C1F70A95A9F7089575
:10ED200084E695E00197F1F708950EE14EE15EEF7C
:10ED3000C895C895C895C895415050400040C1F746
:10ED40000895E0E0F0E0FBBEC0E0D0EF9D2CAD2CDC
:10ED5000079109D0079107D0C79AF5FFC798219767
:10ED6000B9F79A280895A02618E0990CAA1C10F467
:10ED70009624A7241A95C9F70895EE27FB2DCBBE3C
:10ED800065EA03E04BD0839491F0EE27FB2DCBBED8
:10ED9000C0E0D1E010E80990199001E03FD0329630
:10EDA0001A95C9F7EE27FB2DCBBE05E037D001E160
:10EDB00035D06AE5882061F0C0E0D1E0EE27FB2D78
:10EDC000CBBE442707911991011729F54A95D1F730
:10EDD000BE0CCF1C1C2D113011F41B2D103E0895BC
:10EDE000C0E0D1E065EAE199FECF1091680010FD26
:10EDF000FCCFCFBABEBA09910DBB653A71F4E29A65
:10EE0000E19AC79AB4FEC798B39469F76AE5CE0C45
:10EE10001C2D103108950EE176DFF8C81F93109174
:10EE2000680010FDFCCFF894E199FECF00936800D4
:10EE3000653A99F7E8950000000000000000109185
:10EE4000680010FDFCCF1F91089540000000009560
:10EE500048000001AA875000000200FF5A5845569A
:10EE60004F5F465742494E005A5845564F1A0D0AB1
:10EE70000D0A1B5B313B33376D001B5B33316D4239
:10EE80006164204352432100626F6F743A20000096
:10EE90002062657461006D61696E3A200000534420
:10EEA000206572726F723A20000043617264000044
:10EEB00052656164206572726F72000046415400B1
:10EEC00046696C65000057726F6E672066696C65F5
:10EED0000000206E6F7420666F756E6400000D0A6E
:10EEE0005365742074656D706F7261727920636F01
:10EEF0006E66696775726174696F6E2E2E2E0000E2
:10EF0000547279207570646174652066726F6D202B
:10EF1000000053442D636172642E2E2E0000525364
:10EF20002D3233322E2E2E0D0A1B5B306D4E6F7735
:10EF30002C2073746172742066696C652074726130
:10EF40006E73666572207573696E6720582D4D6FFC
:10EF500064656D2D4352432070726F746F636F6CE4
:10EF60002E201B5B33306D000D1B5B4B000044619A
:10EF7000746120697320636F7272757074212055FB
:10EF800070646174652069732063616E63656C658C
:10EF9000642E00005265636865636B20666C617364
:10EFA000682E2E2E202020004F6B210055706461AA
:10EFB0007465206973206661696C7572652E000046
:10EFC0001B5B303B33303B34306D1B5B324A2020BF
:10EFD0001B5B313B33316DDBDB1B5B33336DDBDBC9
:10EFE0001B5B33326DDBDB1B5B33366DDBDB0D0A0A
:10EFF000201B5B33316DDBDB1B5B33336DDBDB1BDA
:10F000005B33326DDBDB1B5B33366DDBDB20201BC0
:10F010005B33376DDFDFDFDFDB20DB202020DB2011
:10F0200020DBDFDFDFDF0D0A1B5B33316DDBDB1B3A
:10F030005B33336DDBDB1B5B33326DDBDB1B5B3345
:10F04000366DDBDB20202020201B5B33376DDCDFBF
:10F05000202020DFDCDF202020DBDCDCDC2020DBCC
:10F06000202020DB20DCDFDFDFDC0D0A1B5B3331FF
:10F070006DDB1B5B33336DDBDB1B5B33326DDBDB4B
:10F080001B5B33366DDBDB202020201B5B33376DB1
:10F09000DCDF20202020DCDF20DFDC2020DB202044
:10F0A000202020DFDC20DCDF20DB202020DB0D0A1D
:10F0B0001B5B33336DDBDB1B5B33326DDBDB1B5BDD
:10F0C00033366DDBDB20202020201B5B33376DDFE8
:10F0D000DFDFDFDF20DF202020DF2020DFDFDFDFBA
:10F0E000DF202020DF20202020DFDFDF0D0A0A00C4
:10F0F000FF1F627FC23C006088FFFF8008900122F2
:10F10000400488C60011850302E24410015C41F30B
:10F110009320F5E6101A00CD6EFF0C1046D3086C54
:10F12000E033F306D398E9200364F301FFD8FD0030
:10F1300015E0025480F00A50012AF30468FBA0DEB7
:10F1400002B4F3E64005A8E6A01B39B312B9A0D378
:10F15000D00DB0E0CEF30BD374C005B838F3027015
:10F16000F84C121BFF98FF0229B38048FC40ED1DAC
:10F17000F458FF06848BCB400856A82106BFD8CC94
:10F180001FA6B307E9B3FC866AF8639DD1D870FD6A
:10F1900046B36DCB28041B76DA50FB08090D1981A4
:10F1A000FE824FF6CC89FE097F7FB004486CB3FA2B
:10F1B000F90FCF304B7FFE7FD8FBC12CB3C12C1988
:10F1C000C127B6B19004BFF632DCFB071FB64BABCC
:10F1D000FC0C9C3060FE19607E713083FF7617B2A4
:10F1E000FD071EF649C9FA07A718301FBC30607E1C
:10F1F000F23010C958F4884CB3607EDF60C00264FE
:10F200002CF4183EAE92F040C858F4287D4B11C043
:10F210002A70C4FF18242CB3580F2E3130FEB1CB06
:10F22000CFD852B3EE5BC87ABA01C2258DB98EF23F
:10F23000CA04D56602611266E0C73515806AB3B0AC
:10F24000508DB31BB0FD8C6658114419D8F8FB25BE
:10F25000A6B320CF80BF5202A5403C019CF36718A3
:10F26000D1D9D38277AC982811CC6613A677C12365
:10F27000ECCC137649C096FB320ECCB30FD3B3035C
:10F28000F4B3C0FD30B33F56B310090BB3CC04CB7D
:10F29000B0AD370CB30FD3B303F4B3C0FD59B38093
:10F2A0002DF409FE9AE3607EFDCC81FAB3B240AA48
:10F2B00092C129668961F7AC982095F4B881C3F6AC
:10F2C0003207EE18E13F98B31FA6B307E9B381FAFE
:10F2D000B3607E98B31FABB30C55F8068DB6DA70E9
:10F2E000FD11ADB30856F80436DAEC50FB08121BDA
:10F2F0001981FE077C3147FFD87F042436B3FAF921
:10F3000004062C94404DEA88604CE2940CC121B371
:10F31000F2B0F9D3F6324324EBD8A8F866B4D8C0DB
:10F32000039D6CD3F834311936B3F1F9030486B375
:10F33000A8FCC127F632DC0725B62CABFC0F3C300D
:10F3400060FE1960FE669604B304CF989824E7C85F
:10F35000B2FD608EB5EC300288123F323CD61020F0
:10F36000D8962300668EF9C12019C34E30303F6D08
:10F3700079BAB0FD260C190DFDDC9620B360C7F6F6
:10F380007F0FF5DFD8D8FB22B9B3800501FB608C75
:10F3900019A0E0B41BF80804526660B308FE3048B8
:10F3A00000B3CC30B33F6E60DA6CEC73F652B33B13
:10F3B000DBB10255F801844D8DB9FC8EE172AA666D
:10F3C00002C22666E0FAC73E0FD5B350611BB31BDD
:10F3D000FD611866B0118919F8B0FB4B4DB320CF11
:10F3E000807F5202404B3C0138F3CE31D1B3D3047D
:10F3F000EF589828242C6690130C66123ECCC13B23
:10F400006C4912CC660FCBB0603F6EADC6B7868834
:10F410006040DE6080C53489C0FDF3E503F4B3C00D
:10F42000FD30B33F4CB30FD3B303F4B3DE365BB858
:10F4300004AA1940AE60C0CDFD7F408A18B318669B
:10F44000193F8D8254FB8395D860FFC76D01824FB1
:10F45000B29808101558662398B2275E6010C12133
:10F46000B3CC6099E64B06F9B381FB36C407EFD8FD
:10F47000CC1FA6B307E9B381FAB3B50C58F806DB85
:10F48000DA70FD61265AECACF8046DDA50D8FB084E
:10F4900024361981FE04C6ECE304121BB3FAF90307
:10F4A000EFCC4B1FFE7FAC79C12CB3C12C19C12707
:10F4B000B6B190040FD8321FB7606071DF13BAFD88
:10F4C0006072F9E58131A6AF069F18307F86E107AB
:10F4D000EF98981FBC30607EF13081FB766007EDBD
:10F4E000D8601FABB31053F81CFE52A2FCC716BA6B
:10F4F00002ABF80108968DA83BCBCA04556602847E
:10F500004D66E0FA8DADE18056B35011B6B339FFC8
:10F51000118B6611089B19F8FB04B4B320D7CF8078
:10F52000F45202403CB3018CF3E3D11B30D34EF5CF
:10F530009824823966826F183024FDCC8277183087
:10F5400024186615FC7D607E98B31FA6B307E9B347
:10F5500081FAB3607E98B31FA6B307E9B381FAB30B
:10F56000607E98B31FA6B307E9B381FAB3B0104821
:10F570006CB3CCFB12CC660DF3B303F4B3C0FD3017
:10F58000B33F4CB30FD3B303F5B30C6AF8B106B66F
:10F59000DA70FDC235B308AAF804C6DDDA50FB08FC
:10F5A000824319B2FD604C7E7F04C121B3C9B0FA19
:10F5B000260C190E3FEC7FD8FB12CCB312CC1912DB
:10F5C0007BB19060FFF63207EBB3BAFD6071B619FC
:10F5D00089FE0FC66607EF3630FAF9071F2C308117
:10F5E0000ACF30983F7A17C1FF8CCA0FDDB0493F70
:10F5F0006E60C0FDBB6003F7D69810A6F839FD52C7
:10F60000C0FA8E2DB30256F80111368DE8F938E0B4
:10F61000B5045866024466D8E0FADAE080D5B35003
:10F62000611BB320FE611866B0118919F8B0FB4B5D
:10F630004DB320CF807F5202404B3C0138F3CE3196
:10F64000D1B3D304EF30984830664ECBC80257EBA5
:10F65000CC2CC80953660623B303F4B3C0FD30B302
:10F660003F4CB30FD3B303F4B3C0FD30B33F4CB33F
:10F670000FD3B303F4B3C0FD30B33F4CB30FD5B3D6
:10F68000108243B3CCFB609666606F98B31FA6B33D
:10F6900007E9B381FAB3607E98B31FABB30C55F89A
:10F6A000068DB6DA70FD11ADB30856F80436DAB03F
:10F6B000504AD66289FEC188B3C1FFFB32BAFD044D
:10F6C000B3660395B3046090B3D8D8FB2598B325EF
:10F6D000AC19081216B39007D6D8E3F9FF81FBD610
:10F6E0001705A6D8961FBC30607EF13081FBC67D21
:10F6F0000FFF7FB08163BB6007FEECB1FAF90C2FFE
:10F7000030E53F7830C0FDE33003F5B3106AF863AD
:10F710009F52D8A2FCE2BA02D5F80161128DA8C7A7
:10F720006F13046A66B0028966E0B1FAB5E180AA97
:10F73000B350C236B339FFC2316611611319F8FBF9
:10F740006096B39A20CF80FE520240963C0171F33E
:10F750009CD16366D309DE98B024472D6630AF4A4A
:10F76000E330049FB0CC4EC3E104836602BF8C7DBE
:10F770000FD3B303F4B3C0FD30B33F4CB30FD3B3D7
:10F7800003F4B3C0FD30B33F4CB30FD3B303F4B3B2
:10F79000C0FD30B33F56B310090DB3CCFB825966A0
:10F7A00081BEB3607E98B31FA6B307E9B381FAB3F5
:10F7B000607EADB30C56F80636DAD870FD46B3B5A8
:10F7C0000858F804DBDA50FBB004486C19C9FA1287
:10F7D000CCB312FF7F086090B3D8B2FD1D1E4B6002
:10F7E0007E98B31FA6B307EBB389FE60C4B360FE77
:10F7F00019B0BA23B930406CF7B0D8267C98C1272D
:10F800005615D808597BB52358F8F820E7C8C00327
:10F81000B4016CF748FC1073C8036AF8C090FC6030
:10F8200090B39698B3090BFFDC0638B05C7FC647EF
:10F83000A3FCC18B8C301FFBB1EBB0F8397415C041
:10F84000FBABDF07FF2A98305E5830193F7D9810D8
:10F850006AF8638BD3881DE57D02AAF801C2258D65
:10F86000A88EFA4B04D56602611266E0C723F680C3
:10F870006AE2B0508DB368B0FA8C6658114419D85A
:10F88000F8FB25A6B320CF80BF5202A5403C019CC7
:10F89000F36718D1D9D38277AC98281216668109FC
:10F8A00094F86091F6CC099C30D8FAF912BF326016
:10F8B0006018B31FA6B307E9B381FAB3607E98B3AB
:10F8C0001FA6B307E9B381FAB3607EB6B3DCFB06CB
:10F8D000DA1904D8B3C13019C0DB5AB380ACF89040
:10F8E000090F5A9801C5A9822A6604C12BD7E502DF
:10F8F000ACB3FD12FF32106090B3B0CCB819C0FDAC
:10F90000DBE303F4B3C0FD30B33F4CB30FD3B30319
:10F91000F5B30C6AF8B106B5DA70849A15B608CB5F
:10F92000941B76DA50FB04090D19EBF8824BB3C92E
:10F93000FA6097FB7F080486B3A3FCC0FCF34B0777
:10F94000FFEC7FB2FD09831904BEB0FE7E30193F83
:10F950005BB3BAFD038D1989B0FE260C190E3EEC7F
:10F9600017FAF9125BB3D8FB025B76498107479817
:10F97000981FBC30607EF13081FBC530C67D071F0B
:10F980002C3090167E32C0FD5AB31098F8E7EC5236
:10F990008077B61702ABF80108968DA83BBBE3044D
:10F9A000556602844D66E0FA8E1A47ACB350236C5C
:10F9B000B328FE23166611113619F8FB0969B32026
:10F9C000CFAF80E95202403C016719F3C6D136D36C
:10F9D000609DEB9824048666EBF8C12E6C2A123EDB
:10F9E000CCC1339B30A3FC04836602BF8C7D0FD354
:10F9F000B303F4B3C0FD30B33F4CB30FD3B303F440
:10FA0000B3C0FD30B33F4CB30FD3B303F4B3C0FD69
:10FA100030B33F56B310090DB3CCFB82596681BE9B
:10FA2000B3607E98B31FA6B307E9B381FAB3607ED3
:10FA3000ADB30C56F80636DAD870FD46B3B50858A3
:10FA4000F804DBDA50FBB004486C19EBF8125BB336
:10FA5000C9FA04BFD87F082436B3A3FC07E7984B44
:10FA60003FFE7F90C099301949EDFED883FD98C6BE
:10FA70001FADB389FE8311B383FB19BAFD607E7994
:10FA8000E583FF7617FAF90C5CCA60FFBD4981FE79
:10FA900081CBE6E50717D77F1830131DB160617978
:10FAA000E581FB766007EDD8601FABB31053F81CFF
:10FAB000F56B808EF27D02D5F80161128DA8C76FBB
:10FAC000FA046A66B0028966E0B1FAC34755B350DA
:10FAD000846DB328FE84626611C22619F8FBC12D1D
:10FAE000B32035CF80FD5202402C3C01E3F338D1E6
:10FAF000C6CCD313BD9824608E66609B7660093FA8
:10FB0000CC609D86E1090666057F187D1FA6B307B8
:10FB1000E9B381FAB3607E98B31FA6B307E9B38156
:10FB2000FAB3607E98B31FA6B307E9B381FAB36056
:10FB30007EACB3101216B3CCF1A9607EFD7F81FAC2
:10FB4000B3607E98B31FA6B307E9B381FAB3B0DC04
:10FB50009356FC0CABF8061B6CDA70FD235AB30805
:10FB6000ACF8046DDA50D8FB04243619EBF8092DF3
:10FB7000B3C9FA825FEC3208121BB3A3FC03F3ACE7
:10FB8000FE1FFF7F90604C981924F6FED8C1FECC72
:10FB9000C60FDF6C98B2FD0E2F2D98B09625CC19AC
:10FBA0000E4EEC17FAF918B8CAC1FFBBB181FE03BB
:10FBB00097CCE50E3FEC7F89FE098EB0B130BCE5F5
:10FBC000C0FDBB6003F6EC600FD5B310A9F88E7AC8
:10FBD0006B80C7797D026AF8B001898DA863B7137D
:10FBE000B5045866024466D8E0FAE147AAB350C2A9
:10FBF00036B328FEC2316611611319F8FB6096B363
:10FC00009A20CF80FE520240963C0171F39CD16352
:10FC100066D309DE98B024472A66B0DF4BAB920466
:10FC20008FB0CC4EA31104836602BF8C7D0FD3B37B
:10FC300003F4B3C0FD30B33F4CB30FD3B303F4B3FD
:10FC4000C0FD30B33F4CB30FD3B303F4B3C0FD30AA
:10FC5000B33F56B310090DB3CCFB82596681BEB3D6
:10FC6000607E98B31FA6B307E9B381FAB3607EAD97
:10FC7000B30C56F80636DAD870FD46B3B50858F816
:10FC800004DBDA50FBB004486C19C9FA12CCB31289
:10FC9000FF7F086090B3BBB2EC7F0FDF304B3F4C6F
:10FCA000B30FD5B3DC81C96D2CABFC824BB389FE9D
:10FCB000606698191FBDB16093AD15FAF9824BB318
:10FCC000D8FB604B66C881C1FFACFE0FD5B3BA81CB
:10FCD000C98B478903F7CC981FFB179060726E4958
:10FCE000D8C166ECFA0FDBDA601098F8E7AC6BB3BA
:10FCF00077963002ABF80108968DB93B7BFA045534
:10FD00006602844B66E01C954380AAB350C236B3AA
:10FD10001BFDC2316611611319F8FB6096B39A207E
:10FD2000CF80FE520240963C0171F39CD16366D3B2
:10FD300009DE98B024486C66EBF81279CAC9B0FAAB
:10FD400048FBCC04CDEC49A3FC095FB032ECB3C056
:10FD5000FD30B33F4CB30FD3B303F5B3106090B392
:10FD6000B0CC78BBAD03F4B3C0FD30B33F4CB30FA0
:10FD7000D3B303F4B3C0FD30B33F4CB30FDC30E179
:10FD80003F4CB30FD3B303F5B306608AB6FB04014F
:10FD90008021FD1540E440810801B120D4BF20DB63
:10FDA000BD8027F401FDD0F9604CFF7F15A0FF0254
:10FDB000B4800A50012A40D005A8F33B54D0F3C0C8
:10FDC0003EB80017E002CE22D0D343E0D068D33D46
:10FDD000E05C800BC0F3E4A8D389E6FFF080081054
:10FDE000017F410488001120064483F36F22407E86
:10FDF000F30364800C9001CD38B4D381E00CD0D3F0
:10FE00007BE032400699F31045D3F2140128FFFF3E
:10FE1000C020FFFFFFFFFFFFFFFFFFFFFFFFFFFF10
:10FE2000FFFFFFFFFFFFFFFFFFFFFFFFFFFFFFFFE2
:10FE3000FFFFFFFFFFFFFFFFFFFFFFFFFFFFFFFFD2
:10FE4000FFFFFFFFFFFFFFFFFFFFFFFFFFFFFFFFC2
:10FE5000FFFFFFFFFFFFFFFFFFFFFFFFFFFFFFFFB2
:10FE6000FFFFFFFFFFFFFFFFFFFFFFFFFFFFFFFFA2
:10FE7000FFFFFFFFFFFFFFFFFFFFFFFFFFFFFFFF92
:10FE8000FFFFFFFFFFFFFFFFFFFFFFFFFFFFFFFF82
:10FE9000FFFFFFFFFFFFFFFFFFFFFFFFFFFFFFFF72
:10FEA000FFFFFFFFFFFFFFFFFFFFFFFFFFFFFFFF62
:10FEB000FFFFFFFFFFFFFFFFFFFFFFFFFFFFFFFF52
:10FEC000FFFFFFFFFFFFFFFFFFFFFFFFFFFFFFFF42
:10FED000FFFFFFFFFFFFFFFFFFFFFFFFFFFFFFFF32
:10FEE000FFFFFFFFFFFFFFFFFFFFFFFFFFFFFFFF22
:10FEF000FFFFFFFFFFFFFFFFFFFFFFFFFFFFFFFF12
:10FF0000FFFFFFFFFFFFFFFFFFFFFFFFFFFFFFFF01
:10FF1000FFFFFFFFFFFFFFFFFFFFFFFFFFFFFFFFF1
:10FF2000FFFFFFFFFFFFFFFFFFFFFFFFFFFFFFFFE1
:10FF3000FFFFFFFFFFFFFFFFFFFFFFFFFFFFFFFFD1
:10FF4000FFFFFFFFFFFFFFFFFFFFFFFFFFFFFFFFC1
